S3150000000030F5FF1F61060000690600006B06000060
S315000000106D0600006F06000071060000000000007B
S315000000200000000000000000000000007505000050
S315000000307506000000000000FD0500004D060000EA
S315000000407B0600007B0600007B0600007B060000A6
S315000000507B0600007B0600007B0600007B06000096
S315000000607B0600007B0600007B0600007B06000086
S315000000707B0600007B0600007B0600007B06000076
S315000000807B0600007B0600007B0600007B06000066
S315000000907B0600007B0600007B0600007B06000056
S315000000A07B0600007B0600007B0600007B06000046
S315000000B07B0600007B0600007B0600007B06000036
S315000000C07B0600007B0600007B060000F717000099
S315000000D07B0600007B0600007B0600007B06000016
S315000000E07B0600007B0600007B0600007B06000006
S315000000F07B0600007B0600007B0600007B060000F6
S315000001007B0600007B0600007B0600007B060000E5
S31500000400FFFFFFFFFFFFFFFFFFFFFFFFFEFDFFFFF9
S3150000041000F002F800F068F80AA090E8000C8244A8
S315000004208344AAF10107DA4501D100F05DF8AFF285
S31500000430090EBAE80F0013F0010F18BFFB1A43F0BC
S3150000044001031847D0440000104500000A444FF04D
S31500000450000C10F8013B13F0070408BF10F8014B1D
S315000004601D1108BF10F8015B641E05D010F8016B62
S31500000470641E01F8016BF9D113F0080F1EBF10F8C6
S31500000480014BAD1C0C1B09D16D1E58BF01F801CBE9
S31500000490FAD505E014F8016B01F8016B6D1EF9D56C
S315000004A09142D6D370470000103A24BF78C878C16D
S315000004B0FAD8520724BF30C830C144BF04680C6064
S315000004C0704700000023002400250026103A28BFAC
S315000004D078C1FBD8520728BF30C148BF0B607047B0
S315000004E01FB51FBD10B510BD03F044FB1146FFF745
S315000004F0F7FF00F0EFF903F062FB03B4FFF7F2FF3A
S3150000050003BC03F063FB00008546084780F30988B7
S315000005107047EFF309807047684680F309880448FE
S315000005200078C00714BF0220032080F314887047A8
S315000005300C410000DFF818C0EFF305831B0618BF57
S315000005406047EFF31483DB0708BF604700DF70479F
S315000005507B300000DFF818C0EFF305831B0618BFD9
S315000005606047EFF31483DB0708BF604700DF70477F
S31500000570B3300000EFF30980816911F8021C39BB22
S3150000058090E80F10E047EFF3098C194B93E806004B
S31500000590914218D059B10CB44FF0010381F82130C3
S315000005A02CE9F00FC1F824C002F091FF0CBC1A60D0
S315000005B0D2F824C0BCE8F00F92F821308CF30988F9
S315000005C01BB192F82000CCF800006FF0020E7047C5
S315000005D010B5084A1268914209D8074C54F82140D0
S315000005E090E80F10A047EFF3098C8CE80F0010BDC0
S315000005F054E0FF1FDC3B0000DC3B000002F006FF7E
S31500000600114B93E8060091421BD00CB44FF0000347
S3150000061081F82130EFF3098C2CE9F00FC1F824C0E2
S3150000062002F055FF0CBC1A60D2F824C0BCE8F00FEB
S315000006308CF3098892F821301BB192F82030CCF85F
S3150000064000306FF0020E704754E0FF1F02F026FFE5
S31500000650D6E7000002F021FF02F020FFD0E70000FD
S315000006600948804709480047FEE7FEE7FEE7FEE740
S31500000670FEE7FEE7FEE7FEE7FEE7FEE7044805497C
S31500000680054A064B70470000A10600001104000051
S3150000069030F2FF1F30F5FF1F30F3FF1F30F3FF1F4F
S315000006A059484CF22051C1814DF62811C1814FF4B1
S315000006B0E971018055494FF4881048645448002177
S315000006C0017054480173242242709A220270C27843
S315000006D002F01F02C27003220271417181798907FB
S315000006E0FCD58179C1F381010229FAD10271402139
S315000006F0417181798906FCD581794906FCD51A2193
S3150000070001708179C1F381010329FAD18179490602
S31500000710FCD5704730B53F4908783F4B84094FF404
S3150000072000404FF001020FD00C78B2EB941F58D165
S315000007304B78DB075ED0087A3849C0F3420002FAEC
S3150000074000F0B1FBF0F055E04C7964063ED40C782D
S31500000750640710D40C7BE40700D118460B78C3F36A
S31500000760C20302FA03F3DBB2B0FBF3F04B7813F0EB
S31500000770300F00D04009C97801F0E00111F01F0FD9
S3150000078038D14911082935D2DFE801F004070B0FEB
S3150000079013171A1D00EB800005E000EB8000000235
S315000007A028E0C0EB0010C00124E000EB800040020E
S315000007B020E04FF4377148431CE04FF4B761FAE785
S315000007C040F69501F7E740F67131F4E70879497983
S315000007D000F01F00401CB3FBF0F001F01F011831C0
S315000007E0E9E70C780225B5EB941F0BD1097BC90705
S315000007F000D118460549496C02EB1171B0FBF1F0C6
S315000008000749086030BD0000002005400080044014
S31500000810005006400040064000127A0000093D00E4
S3150000082000E0FF1F00F0C9BD00F0D3BD35490968DF
S3150000083008B1012000E0022002F066B9002464201D
S31500000840DFF8C4C000DF204600F0F7FD24B1002425
S31500000850DFF8B8C000DFF6E70124F9E70024DFF887
S31500000860B0C000DF274E00231A460F213060AFF2DA
S315000008703300DFF8A0C000DF706000F0DEFC01F09E
S31500000880DDF9012001F0E6F900224FF6FF710320A1
S31500000890DFF884C000DFC820DFF880C000DF00205A
S315000008A001F0D8F9DFF878C000DFC00701D00A25CB
S315000008B000E03225DFF86CC0706800DF204600F0EB
S315000008C0BBFD2CB100242846DFF850C000DFF5E759
S315000008D00124F8E710B500F093FD00F0C4FD40B91F
S315000008E0FFF71AFE00221146AFF28F00DFF838C07C
S315000008F000DF01F02DF84FF4A04003C8FFF704FE17
S31500000900002010BD04E0FF1FB9380000C938000000
S31500000910EF3500006B360000612A0000B338000096
S315000009202B2B0000D73600005B370000FEE7704730
S31500000930FEE77047704710B502F059FE30B117490F
S3150000094000EB400001EB4010603810BD144810BDAC
S31500000950144910B50246086800B1FEE71248106057
S3150000096001220A6002F0B6FB012010BD10B5044654
S3150000097002F03DFE002805D04FF6FF71DFF82CC0CF
S31500000980206800DF10BD10B5044602F030FE0028D6
S3150000099003D0DFF81CC0206800DF10BD8C0E0020DD
S315000009A0901500200CE0FF1FCC1000208B310000BA
S315000009B0E530000000207047002070470020704797
S315000009C000207047002070470020704700207047C5
S315000009D000207047002070470020704700207047B5
S315000009E000207047002070470020704700207047A5
S315000009F0002902D0DFF888C000DF7047DFF884C026
S31500000A0000DF70470022DFF880C000DF704700F08B
S31500000A10C4BA2DE9F0411D4C1D4F002525603868EC
S31500000A2038B100231A4603211A48DFF86CC000DFEC
S31500000A302060DFF85CE0194E00240EF1080E00BFBE
S31500000A4046F824505EF8240038B100231A460221E5
S31500000A50DFF844C000DF46F82400641C0F2CEFD9F1
S31500000A600F4C25607868002807D000231A4602211B
S31500000A700C48DFF824C000DF2060BDE8F0810000EC
S31500000A80992A00002B2B0000612A000044E0FF1F7A
S31500000A9040410000000000006B36000094F1FF1F8B
S31500000AA030E0FF1F00000000FE4900228A61CA6193
S31500000AB00A6250B14A62487808B1072000E008206F
S31500000AC008610A724A728A72CA624FF4A0400A63C7
S31500000AD0C860CA700A714A718A718A62CA71F34A19
S31500000AE0F1481060012008707047DFF8C4C300DFCA
S31500000AF0EC4DF04F4FF6FF7A4FF480694FF4A04665
S31500000B004FF40038A863002251460C20DFF8A8C332
S31500000B1000DF0228F7D1DFF8A4C300DF0446000790
S31500000B2005D5E14A4946E86803DF00F076FA600732
S31500000B30E9D5386800F010FC3446204602DF04F59B
S31500000B4080644445F9D300F068FADCE700273C46A8
S31500000B50DFF85CC300DFD34E4FF4E0487063002239
S31500000B6064214046DFF850C300DF022810D0002C75
S31500000B70F5D0DFF84CC300DFC01B40F6B831884221
S31500000B80EDD906200024B070204600F031FAE6E7E1
S31500000B90DFF828C300DF0546C00417D50120F07131
S31500000BA03220DFF820C300DFF07901280ED196F855
S31500000BB02000C00705D0BC4A4FF48061F06800F001
S31500000BC031FA012000F014FA0020F071A80404D5CF
S31500000BD0DFF8ECC200DF074601246804BFD5002415
S31500000BE0BDE710B5AF4C606A01280AD060790128CC
S31500000BF009D000F00EFA0420A16B01F085FF012058
S31500000C006062002010BD0320A070002000F0F0F903
S31500000C10012010BD2DE9FC5F0024DFF8888207461D
S31500000C20A146A24601940094072904D198F8010030
S31500000C30012804D00D2420464FF0010B07E00C24B8
S31500000C40F9E707EB4011C97AC9067BD4401C102886
S31500000C50F7D3254612E007EB45166946304600F005
S31500000C601BFAF0B101281CD002281AD0032818D08C
S31500000C70042816D0052878D020346D1C102DEAD310
S31500000C80B9F1000F09D0D8F81C20D8F810100020B0
S31500000C901144C8F81010FFF707FF0198012862D029
S31500000CA034E0F1694346C8F818100029E5D0728B84
S31500000CB06FF0060C0CEBC20201F2FF11490A1A632F
S31500000CC0D96131785F2907D02E2905D0E5290DD1C4
S31500000CD003280BD0012809D01869904201D14FF0A2
S31500000CE00109C3F818A0C8F81CA0C6E7587A194627
S31500000CF001280FD118469B7A63B9046B836AA34215
S31500000D0008D304228270002000F072F94FF0FF3001
S31500000D10BDE8FC9F886A08B30B6B98421ED2101A76
S31500000D200A6A121AC869824218D381F800A0C1075C
S31500000D304FEA500500D06D1C00244FF4A0464FF436
S31500000D40806707E011E006EB8420574A394600F039
S31500000D5069F9641CAC42F6D30120D5E781F808B0E6
S31500000D6000982C4648612046D2E788F802B0CAE7C8
S31500000D7070B54C4E04460D463078002834D05248A3
S31500000D800068002830D04FF40071284602F074FE47
S31500000D90092C32D806F13C0000EBC4014A6850F831
S31500000DA03410284602F023FE012C1ED0072C1BD13E
S31500000DB07078002818D106F13C0000F13804C06BA9
S31500000DC020222844414902F012FEB17806F194002F
S31500000DD050F8210002F0ECFD626805F11C01505448
S31500000DE0062061681A35485570BD70780028FBD119
S31500000DF0FF2068720F20A87270BD112C07D0192C25
S31500000E0009D0212CF8D1BDE8704000F016BA2F4960
S31500000E10A022203102E02D495022C0312846BDE8EB
S31500000E20704002F0E4BD2DE9F0411E4E04460A462C
S31500000E30307800284FD00125072C01D0082C1CD172
S31500000E40E1B21046FFF7E6FE401C16D0F07810B16E
S31500000E50012802D011E035710FE0D6E9071088426B
S31500000E6002D1726A012A0DD0336BB26A9A4204D15A
S31500000E70884202D9706A01287ED0292C2BD330797A
S31500000E8058B10BE0F079002825D1F571716BBDE8FA
S31500000E90F0414FF4805001F037BEF570F06AE0B1D2
S31500000EA0401C15E01400002078E0FF1FF40000202D
S31500000EB0EF35000000E0FF1F612A00002B2B000029
S31500000EC0AD380000B3380000DC00002028440000E4
S31500000ED0A04202D0B572BDE8F081B07918B9306988
S31500000EE0844200D93461FFF77CFE0128F3D0706A92
S31500000EF00128F0D1B07A002720B13069844201D1AF
S31500000F00B77277723069A042E5D8B17951B9A0427B
S31500000F100CD1B5714FF40050716B01F0F5FDB46260
S31500000F20B07918B1B079012805D00FE03069A04238
S31500000F300CD0052029E0B07A40B9B06AA04205D0AD
S31500000F40316A0844A04201D002201EE0F07901284F
S31500000F5000D1F771B07920B13069844201D1B772FE
S31500000F607772F462306A401C3062C007704801D064
S31500000F7000F500706F4900E009E0086000F05CF8D9
S31500000F800128A8D1307A30B10420B0700020BDE825
S31500000F90F04100F02DB875729DE7674810B5C17A2B
S31500000FA0012489B9654AC47200234CF60501AFF2E3
S31500000FB06340DFF88CC100DF00231A460A21AFF236
S31500000FC0D540DFF87CC100DF5E494FF41830086079
S31500000FD05D494FF4007008605C485D4904604FF459
S31500000FE0987008605349524808605A48046010BD1A
S31500000FF070B5514D044668700120FFF755FD204637
S31500001000FFF714FC696BBDE870404FF4804001F0B7
S315000010107BBD51490820086070474F490820803938
S315000010200860704710B5FFF7F4FF4348816B08204E
S3150000103001F06AFD002010BD70B53F4C4FF480658D
S3150000104094F82000C00716D1394A2946E068FFF710
S31500001050E9FF20B1E06800F58060E06018E0D4E9BF
S315000010600701814203D10120FFF7C2FF12E0E068C9
S3150000107000F58060E060D4E9071088420AD1C00715
S31500001080F1D02B4A2946E068FFF7CCFF0028EAD0CA
S31500001090012070BD002070BDF0B5067A437A827AD1
S315000010A0057800202D4F14E007EBC00494F801C02A
S315000010B0B4450DD194F802C09C4509D1E478944218
S315000010C006D107EBC00252680A6017F83000F0BD7F
S315000010D0401C17F83040052CE6D1A6F1610400202B
S315000010E0192C02D9413E192E1FD8A3F16104192CDF
S315000010F004D92034192C01D9202B16D1A2F1610371
S31500001100192B04D92033192B01D9202A0DD1A5F189
S315000011106102192A02D92032192A06D82E2D04D0A6
S315000011205F2D02D008600520F0BD08600620F0BDE6
S3150000113078E0FF1FF40000201400002078F0FF1F65
S315000011406B3600000C010020E8000020EC000020B7
S31500001150F0000020DC00002084E100E038450000BB
S31500001160F0B5064600200346054617E03478A4F19C
S315000011703007092F01D830230AE0A4F14107052FD3
S3150000118001D8372304E0A4F16107052F00D85723BF
S3150000119000FB0240C01A761C6D1CEDB28D42E5D3F1
S315000011A0F0BD2DE9F041674E2420674F3070707016
S315000011B0B0701820F0700425796800200A5C72551A
S315000011C06D1C401CC0B2EDB20428F7D3002405EB19
S315000011D0440081194A1CC4F10300C300F868D840D2
S315000011E0C0B200F058F8641CE4B2042CEFD3083502
S315000011F0EDB2002405EB440081194A1CC4F103003A
S31500001200C3003869D840C0B200F045F8641CE4B2A7
S31500001210042CEFD30835E8B200213154BDE8F08143
S31500001220484810B5001D02F0C3FB022101EB400047
S31500001230C0B210BD43481D3070477CB5424D0024F6
S315000012402878C8B905F10C0000F022F91022042113
S315000012506868FFF785FFE968102248402861082181
S315000012603A48FFF77DFF296948402861FFF799FF53
S3150000127000F01DF80120287035480021354D8DF805
S3150000128004100090684600F039F810B12855641C27
S31500001290F8E701207CBD2D4B10B5113B03EB101474
S315000012A000F00F0024780C70185C107010BD2DE94A
S315000012B0F041244C201D02F07BFBC3B2022004F156
S315000012C01D0500EB430028700320022268700021F0
S315000012D0084605E0CE070BD05618A855491CC9B2DA
S315000012E0B1EB430FF6D302EB4301C9B2685495E75D
S315000012F004EB510657183679EE55EFE7F0B5114B6A
S3150000130001261B1D104C0025017919B1A168097829
S3150000131079B905710268511C01601278402A0CD116
S315000013200F78412F09D1A3600671491C0160197815
S3150000133029B1A06810F8012BA0601046F0BD057118
S31500001340E2E7000040F1FF1FC40000207D480000D6
S315000013504947000078E0FF1F254810B54CF22051A0
S31500001360C1814DF62811C181018821F0010101805A
S31500001370214820494FF4003201600021C0E90112E2
S31500001380D202C2604FF0A05242614FF40062826105
S3150000139080F82010491E416200F042FB002800D070
S315000013A0012010BD0020704710B51449124800F006
S315000013B0E7FA002800D0012010BD10B501460F4BFA
S315000013C04FF480620C4800F0E4FA002800D00120B7
S315000013D010BD38B50C460949009113460146224610
S315000013E0054800F07BFB002800D0012038BD000036
S315000013F0002005400000024018110020771B000065
S315000014001E48816B41F4A05181631D498015086116
S315000014101C481021016041611B4940F213104860CD
S3150000142070471849C03908B1C83100E0C4310868AE
S3150000143040F0100008607047F3E7F2E70F498A6B47
S3150000144042F001028A6311498860052048600868F5
S3150000145040F00100086008680006FCD5086820F026
S3150000146001000860704700B50220FFF7E7FF054856
S31500001470C038006D00F0020000BD0000008004408E
S3150000148000C00440C0F00F4000A00440000004402B
S3150000149004490A6ECB6D5A408B6D496D4B405A40DC
S315000014A00260704700800440FE49082008607047CB
S315000014B0FD4908200870FD48416841F4A0214160BB
S315000014C0816C21F00F01816400218164416B41F43C
S315000014D08021416301DFF64890F80C1141F080014C
S315000014E080F80C1190F80C110906FBD4F149090A91
S315000014F000F89C1FEF49090C0175EE49090E0176AB
S31500001500FF2100F81C1CEC499C38096811B1042124
S31500001510022201E000210A461143ED3041F0190193
S3150000152000F8691C4021C174C17F41F04001C177B8
S315000015307047E2490028087806D040F0010008709C
S31500001540102081F87400704720F0010001F8740B38
S31500001550087820F01000087070470120D449002256
S3150000156001EB800383F8C020401C1028F8D3D14833
S315000015700823438000F160034360C82303700272AE
S3150000158000F1E0034361C2610D20803181F8400023
S31500001590C54B4FF055305860087D40F00200087585
S315000015A0FF200870087208730A767047C34810381F
S315000015B0017841F0200101707047C0481038017869
S315000015C021F0200101707047BD494CF25030097876
S315000015D089070ED5B94A117841F0040102F8941929
S315000015E000E000BF401EFCD212F8940F20F0040069
S315000015F0107070477047002904D1B04900F07F0091
S31500001600091D087070477047F0B5A74BA94DA94E44
S315000016105A685FEA006C4FF000044FF0010705F1CD
S31500001620600500F00F010CD507EB4100874017431A
S3150000163006EB411005EB01225F608032C461426116
S31500001640F0BD4FEA400C07FA0CF7BA435A60964AC7
S31500001650125C06EB411005EB0121428041608821B6
S3150000166001700472F0BD014680788988020601D4B3
S315000016708D4A1154C8E770478D49020608D500F017
S315000016800F0001EB800010F8C01F41F0050105E0D6
S3150000169001EB800010F8C01F41F00901017070478E
S315000016A08349020608D500F00F0001EB800010F810
S315000016B0C01F21F0050105E001EB800010F8C01FF6
S315000016C021F0090101707047794900F00F0001EB24
S315000016D0800010F8C01F41F0020101707047744984
S315000016E000F00F0201EB820111F8C02F22F0020276
S315000016F00A7089E77047F0B505004FEA0070DFF819
S31500001700B4C14FEA90630CEBC30E4FF00006BEF86F
S31500001710020006D11CF83320C2F383020D2A00D141
S315000017200126644C0022603404EB831702E0BC5CA3
S315000017308C54521C8242FAD35B4A525DAEF80220A8
S31500001740594D5A081CF833E06C68CEF3801E24FA13
S3150000175002F707F00107774501D0696806E00EB188
S31500001760897941B10121914061406960D140C90741
S3150000177004D0C82103E024F00101F6E788210CF823
S3150000178033104E490A7822F020020A70F0BD70B577
S3150000179000F00F000223474D03EB800405EBC40065
S315000017A00023428005F1600000EB841002E0CE5C6D
S315000017B0C6545B1C9342FAD33B4E6108706820FA0C
S315000017C001F3DB0701D0882300E0C82305F8343095
S315000017D001238B4043401046736070BD37490C317E
S315000017E00878097940F2FF7202EA0121084370473E
S315000017F02D48806870472DE9F041304D143D2C7816
S315000018002879803D04402C4FE0070BD0FFF7A5FE5A
S3150000181000F022FA396811B1042001F075F90120AF
S3150000182085F88000E00609D5FFF7C0FE396811B1DA
S31500001830102001F069F9302085F88000A00609D54E
S31500001840FFF7BBFE396811B1202001F05DF92020B9
S3150000185085F88000600707D5396811B1402001F08E
S3150000186053F9042085F880000F4E022C0DD195F80F
S315000018708800B060396811B1802001F045F9FF2079
S3150000188085F88800022085F88000200759D505F1E3
S315000018909000A84601780C0901780078C1F3C001D0
S315000018A010E0000004E100E010E0FF1F00800440AB
S315000018B0002007400012002044E0FF1F942007404C
S315000018C022E0FF1F204F214DC0F3800009D10022E6
S315000018D002EB4102024417F83220C2F383020D2ABA
S315000018E00AD0A20002EB41010E1817F83600C0F329
S315000018F08300012810D015E0706820F002007060A7
S31500001900387E20F080003876387C20F080003874ED
S31500001910296899B102200FE055F8241011B104206E
S3150000192001F0F2F817F83600C0F38300092805D154
S3150000193055F8241011B1082001F0E6F8082188F8BE
S315000019408010BDE8F08100000012002094F1FF1F16
S3150000195030B5094C2068094B98420BD04FF4A04291
S315000019601946002052F8205041F82050401C3E28CD
S31500001970F8D3236030BD000008ED00E000E0FF1F53
S3150000198008B544220B468DF800206A460021984788
S3150000199008BD2DE9F8430746984616467B680020A1
S315000019A08A194FF480658B4203D8BC681C44944264
S315000019B00DD2FB688B4203D83C691C44944202D288
S315000019C00220BDE8F883CC1A04F5000400E0CC1A26
S315000019D0B4FBF5F105FB114111B14FF48070F0E74E
S315000019E0B6FBF5F105FB1161A9B10120E9E78DF818
S315000019F00090200C8DF80100200A8DF802008DF869
S31500001A0003406A4603213846434698470028D8D102
S31500001A10761B2C4401E04FF00909002EE7D1D0E7F0
S31500001A20F0B5016800240A781206FCD570220A7007
S31500001A3002680321D171016880258D710268002139
S31500001A4051710368FC221A710268D173026815701D
S31500001A50026813781B06FCD5567A127A02F00F0C30
S31500001A604FF400425710BCF1100F11D2DFE80CF012
S31500001A70080A0D0F080808080F1E0D0808080808B0
S31500001A80026105E04FF4C042FAE7076100E0016138
S31500001A9006F00F02102A1BD2DFE802F00B0B0B0D2B
S31500001AA0101316191C1E0B0B0B0B0B0B4FF40052CD
S31500001AB0E6E7C1610CE04FF40061FAE74FF480619C
S31500001AC0F7E74FF40071F4E74FF48071F1E7C56171
S31500001AD02046F0BD4021ECE72021EAE72DE9FC474E
S31500001AE0164607461D4600208A19DDF828808B0712
S31500001AF003D04FF48070BDE8FC87B30701D0012006
S31500001B00F9E77B688B4203D8BC681C4494420CD22C
S31500001B10FB688B4203D83C691C44944201D20220E4
S31500001B20E9E7CC1A04F5000400E0CC1A4FF00609E8
S31500001B30002EE0D08DF80090200C8DF80100200AD0
S31500001B408DF802008DF80340E8788DF80400A87837
S31500001B508DF8050068788DF8060028788DF807005E
S31500001B606A4607213846434698470028C3D1241DB4
S31500001B70361F2D1DDCE770B5044600680025037886
S31500001B801B06FCD57023037000203AE00C2836D2E1
S31500001B90DFE800F0060A0E12161A1E22262A2E3238
S31500001BA026681378F3712AE026685378B37126E025
S31500001BB026689378737122E02668D37833711EE025
S31500001BC026681379F3721AE026685379B37216E021
S31500001BD026689379737212E02668D37933720EE021
S31500001BE02668137AF3730AE02668537AB37306E01D
S31500001BF02668937A737302E02668D37A3373401C9F
S31500001C00C0B28842C2D921688020087003E0606AA9
S31500001C10411C00D08047206800780006F7D5206870
S31500001C200078810601D5042506E0C10601D5082500
S31500001C3002E0C00700D01025284670BDB24910B595
S31500001C400020C870FEF7E3FEFEF7E3FEBDE8104095
S31500001C50FFF72EBCFFF76DBCAC484FF001120178C0
S31500001C60A948C180002101704170C0E902210161CB
S31500001C707047A5484078002800D001207047A24947
S31500001C8020310020FFF737BD10B59F4CA04818340F
S31500001C90A28801788A4200D9CAB212B99A490020AC
S31500001CA0087180202168FFF772FD216801442160D8
S31500001CB0A188081AA08010BD10B5934C00201834D6
S31500001CC02168FFF718FD216801442160A188081AE0
S31500001CD0A08010BD002211468020FFF758BD8D4917
S31500001CE00020FFF708BD2DE9F047DFF81C82044607
S31500001CF008F12008844D80074FF0000AA8F1080675
S31500001D0024D5FFF7BCFF98F800004746C009FFF747
S31500001D10B2FCF888B0803878C0F3411111B10129BE
S31500001D205AD17CE098F801207B4FDFF8F0910C2A1D
S31500001D3052D2DFE802F0060C821C822A3A823E4426
S31500001D40526101F0F7FF32E0FFF79EFF83E00020CB
S31500001D5002F02EF8002870D0FFF7BCFF386820B1DB
S31500001D606969002977D0082050E0484652E00120F2
S31500001D7002F01EF880B3FFF7ADFF38680028F4D0F4
S31500001D806969002967D0042040E010F01F0F54D184
S31500001D9098F80200012140F08000287000F07F00D2
S31500001DA0FFF729FCFFF796FF55E001F01FFF98B1FA
S31500001DB0CAE710F01F0F40D15348401C1AE002F04A
S31500001DC047F848B1FFF786FF386818B16969F9B175
S31500001DD001201BE052481DE02FE000F01F00012803
S31500001DE02BD1687848B398F80400A978884224D2A1
S31500001DF04C4908443060A7E702F0EEF8E8B1FFF777
S31500001E0069FF386828B1696911B10220FEF7F0FD53
S31500001E1021E045480168F1B1084680471BE010F013
S31500001E201F000AD0012808D1FEF7C6FD98B900F0B8
S31500001E307FF880B9FEF7CCFD68B998F8001009065E
S31500001E4004D4B8F8060008B1002000E08020FFF7AF
S31500001E503BFCA6F804A0600723D598F80000474687
S31500001E6000061CD4B088E0B1FFF726FFB088C0B9E1
S31500001E703878C0F3411161B101290AD110F01F0071
S31500001E8007D0012805D1FEF799FD50B9FEF7A2FD4E
S31500001E9038B98020FFF718FCA6F804A001E0FFF788
S31500001EA01EFF200713D598F80000000606D5B08857
S31500001EB0297908430BD0FFF7E7FE08E028780106EA
S31500001EC005D500F07F0028700021FFF794FB60061F
S31500001ED002D50020FFF703FC200604D5BDE8F04735
S31500001EE08020FFF7FCBBBDE8F0870B48006850B1C7
S31500001EF04FF6FF7420462146FEF784FDFEF77EFD71
S31500001F00FFF7F1FEF6E700001CE0FF1F244100008A
S31500001F1028410000090000203C4100003841000033
S31500001F2030410000080000203441000000F045B8B0
S31500001F3010B51248124A0179127891421BD14278A3
S31500001F404188C088FE2A09D0FF2A14D199B990B9D0
S31500001F5000F055F878B1FFF7BDFE0AE059B901283F
S31500001F6009D100F055F830B1074906480860FFF777
S31500001F708BFE012010BD002010BD00003CE0FF1FBD
S31500001F80294100000900002034E0FF1F7047704718
S31500001F907047704710B50446FFF796FB200605D537
S31500001FA004F00F014FF48030884001E00120A0408A
S31500001FB0FB490A681043086010BDFA48007900F032
S31500001FC08F01080605D501F00F004FF480328240DC
S31500001FD001E001228A40F448007840F080008842FF
S31500001FE00CD1EF490968114208D0F049F04A096856
S31500001FF0914203D10D22ED49FFF7C9BB7047ED4968
S3150000200000200860E9490860EB4908700120704724
S31500002010EA490020087001207047E44910B5E448F9
S315000020200860E1480D22007840F08000FFF7AFFB22
S31500002030E1490520087010BDDF4910B54868C86041
S3150000204008B1012010BDD9481F38816859B1007BFD
S31500002050000604D5D448007840F0800001E0D84856
S315000020600078FFF797FFD14901200873FFF7D5FFE6
S31500002070002010BD2DE9F041CF4DCB480026AA69BE
S315000020800078696AC94F40F080008046914206D3C5
S315000020900024FFF77FFF3E73FFF7BFFF08E0CA4843
S315000020A0C849007831F81040E86A844200D30446F3
S315000020B0FFF7C2FF00B90024A86A20B364B1A96A79
S315000020C0E869224601444046FFF761FBA86A2044BE
S315000020D0A862E86A001BE862D5E90410AA6A4143CF
S315000020E0914203D1AE62696A08446862B868001B0F
S315000020F0B860002C05D0E86AB0B12878022800D074
S315000021003E73BDE8F081002CE6D0E96A28690144F7
S31500002110491EB1FBF0F26869824200D90246E969BC
S31500002120686AFEF725FECAE703202870E8E72DE96E
S31500002130F041A14D00269D4FA969686A884207D3E0
S315000021409F482E630078FFF725FF3E73FFF765FF74
S31500002150FFF772FF00B92E6300209C4905E0AB6AC9
S31500002160EC690A5C0344401CE2542A6B9042F6D3A5
S31500002170A86A11000844A862EA6AA2EB0102EA62B0
S3150000218022D092B988B129690844401EB0FBF1F407
S315000021906869844200D904462246E969686AFEF7FE
S315000021A042FEAE62686A20440DE0D5E9041202FBE5
S315000021B001F3834208D1E969686AFEF734FEAE622C
S315000021C06969686A08446862B968286B091AB9605F
S315000021D0002896D0E86A10B12878052891D13E7378
S315000021E0BDE8F04119E78CE72DE9F041724C002576
S315000021F06E4EA169606A884207D3714825630078EC
S31500002200FFF7C8FE3573FFF708FFFFF715FF20B18C
S31500002210206B08B3A06A10B10FE0256320E0E16AE5
S3150000222020690144491EB1FBF0F26069824200D97F
S315000022300246E169606AFEF79BFD00206349A36AD6
S31500002240226B0BE0D4F81CC01F181CF8077011F89D
S3150000225000C0674501D0256202E0401C9042F1D3E0
S31500002260A16A206B0A18A262E16A0B1AE362D4E93A
S3150000227004714F43974203D1A562626A11446162B9
S31500002280B168091AB16000280CD013B1207805286E
S3150000229008D1206A20B100203073BDE8F041BCE6C9
S315000022A00120F9E72DE770B5404C434D1F3CD4F8AB
S315000022B0110000BA20F0FF01207D01430020C5E98E
S315000022C00910E07B2F280AD004DC28280BD02A2806
S315000022D017D104E0A8280DD0AA2812D106E0FFF7EE
S315000022E0ABFE002826D0E08A41BA0AE0FFF7A4FE3A
S315000022F000281FD0D4F8150000BA20F0FF01207E78
S3150000230001432869294E4143E962A068012568B165
S31500002310884210D0207B000604D52348007840F080
S31500002320800001E026480078FFF734FE3573FFF79A
S3150000233074FE002070BD012070BD70B51B481B4D9A
S315000023401F380224816831B1007B000608D41C487E
S315000023500078FFF71FFE2C73FFF75FFE002070BDAD
S31500002360012070BD10B51148134C1F388068216BD1
S31500002370884202D82063032000E0042020700A4827
S315000023801249226B007840F08000FFF700FA0748F8
S31500002390226B8168891A81600021017310BD0000DB
S315000023A028E0FF1F3CE0FF1F2A410000F3F1FF1F5A
S315000023B0555342532CE0FF1FD8000020090000208F
S315000023C02B4100002C4100001FE0FF1FD810002009
S315000023D0F74810B5816800F11F0469B1007B00065B
S315000023E004D5F448007840F0800001E0F248007817
S315000023F0FFF7D0FD012004E0FFF71EFE0028CDD038
S3150000240000202073BDE8104007E6C7E710B5FFF7C8
S3150000241094FF0028C2D0E9487021E94B01700021E1
S315000024204170DC685A6832EA040406D006248470D7
S31500002430282404734173DA6009E0DAB1DC4A1F32FA
S31500002440127BDAB105228270202202734173C170B9
S315000024500171417181710A22C271017241728172E8
S31500002460C1728173C1730174417412201863BDE88F
S31500002470104077E7022282703A22E6E78170017304
S31500002480E4E78BE710B5FFF758FF002886D0CB4B63
S31500002490002080211870597002219970D97020246B
S315000024A01C7158719871D871C648016808200A785D
S315000024B012B11A54491C00E01C54401CC0B2242816
S315000024C0F5D3BF4924200863BDE810404AE765E715
S315000024D0B74810B5817C00F11F0421B1012020739B
S315000024E0BDE8104099E5C07CB54900F001004860A0
S315000024F0FFF74FFD0020F2E7AD48C07CC107AC48AE
S3150000250000F11F0000D00121017386E510B5FFF729
S3150000251014FF00281AD0FFF78FFD002816D0A74811
S31500002520032100220170A64942700B7ADB018370F9
S31500002530C270042008639E491F318A68042A02D9A2
S315000025409B4A90608860BDE810400BE726E710B50F
S31500002550FFF7F3FE00281ED0FFF76EFD00281AD005
S315000025609648002106220170954B427081701A7AB6
S31500002570D201C270017141718171C1718C4908200B
S315000025801F3118638A68082A02D9894A90608860D0
S31500002590BDE81040E6E601E710B5FFF7CEFE0028DD
S315000025A01BD0FFF749FD002817D0854A834891695B
S315000025B0491E0B0E03700B0C43700B0A8370C1701F
S315000025C011690B0E03710B0C43710B0A8371C171F8
S315000025D008201063BDE81040C4E6DFE610B5FFF73B
S315000025E0ACFE002828D0FFF727FD002824D073482A
S315000025F00021734A0170417081700821C170916990
S315000026000B0E03710B0C43710B0A8371C17102210E
S31500002610017211690B0C43720B0A8372C172644911
S315000026200C201F3110638A680C2A02D9604A906018
S315000026308860BDE8104095E6B0E65D4900201F3190
S315000026400873EAE470B5FFF778FE00281CD05B48F3
S3150000265002225B4D02704270554C03202A631F34E0
S315000026602870A068022802D951488260A2605148A9
S315000026705249007840F08000FFF789F8A068296B7E
S31500002680401AA0600120207370BD10B5FFF755FEFB
S31500002690002818D049482022002102704170484C79
S315000026A0C17703202263207042484449007840F0F5
S315000026B08000FFF76CF83E48226B1F308168891A4C
S315000026C081600121017369E62DE9F0473C4E002047
S315000026D0374D3A4A316B02E0135C2B54401C88425A
S315000026E0FAD3344C0127DFF8D09020781F2940F028
S315000026F0800A6BD128683449884267D12C4C6868B7
S315000027001F346060A868A060687B18B9A87B08B110
S31500002710102801D9277381E0E87B4FF002082828AA
S315000027206AD01BDC1A285BD00DDC0428F2D005DC4D
S31500002730E8B30328EED1BDE8F04767E61228E9D1F1
S31500002740BDE8F0479EE61B2844D01E2845D0232826
S3150000275049D02528DED1BDE8F0471DE791286DD088
S3150000276013DC35286AD009DC2A2816D02F28D1D1C7
S31500002770287C800756D4002020734FE05528C9D006
S315000027805A28C7D1BDE8F047E1E69E2831D0A128F6
S315000027902CD0A82830D0AA28BCD1FFF784FD002869
S315000027A003D0287B000647D43770BDE8F0870EE0DB
S315000027B0D4F1FF1F2A4100002B410000D810002051
S315000027C0D8000020040000205553424339E0BDE8FC
S315000027D0F047FDE5BDE8F0477AE6BDE8F0478BE651
S315000027E0BDE8F04792E6BDE8F047F7E6BDE8F047FA
S315000027F028E7BDE8F04748E7FFF755FD0028D4D0A5
S31500002800287B000604D586F80080BDE8F04731E451
S3150000281099F80000FFF7BEFB84F80C80BDE8F0478E
S31500002820FFF7FBBBFFF73FFD0028BED0287B000665
S3150000283002D437703762B8E75046EBE7BDE8F04799
S31500002840FBE65046FFF7A6FB2078534C00F00F013D
S315000028504FF48030884021684D460843206099F83F
S315000028600000FFF797FB287887402068074306207B
S315000028702760307099E7494910B50878022808D0D2
S31500002880032810D0042812D0052801D10020087092
S3150000289084E54348C07B282801D0A828F8D1BDE8A4
S315000028A01040FFF7E7BBBDE81040FFF7B6BB3D4859
S315000028B0007840F08000FFF76DFBF4E7374810B56D
S315000028C0007878B1012810D005281CD03648007849
S315000028D0FFF760FB324902201F310873BDE8104044
S315000028E0FFF79BBBBDE81040EEE62D48C07B2A28CB
S315000028F003D02F2804D0AA2805D1BDE8104016E43D
S31500002900BDE8104070E449E5B5E7274810B527490A
S315000029100078FEF7F0FE21490863BDE81040CDE7D8
S3150000292010B50446400702D50020FFF7EEFF20074A
S3150000293002D5BDE810409EE730E51D48006860B14D
S315000029404FF6FF7420462146FEF75CF8FEF756F870
S315000029500007F7D5FFF78FFFF4E71548006868B161
S315000029604FF6FF7420462146FEF74CF8FEF746F870
S315000029704007F7D50020FFF7C8FFF3E70C480068CB
S3150000298050B14FF6FF7420462146FEF73BF8FEF79E
S3150000299035F8FFF7C5FFF6E72CE0FF1FD80000204B
S315000029A0D4F1FF1F2A4100002B410000D81000205F
S315000029B03C41000010B5428C920803D1234A12888C
S315000029C0C2F38D02836A03EB82035A0700D51B1FED
S315000029D0403B4FF08072C3E90E120022144643F8C2
S315000029E02240521C0E2AFAD3C2691A624362C1629D
S315000029F0806A1749016010BD16480068C0010BD5F2
S31500002A0015480068C00707D01348803800680028BA
S31500002A1002DA12490120087070474FF06042D36F06
S31500002A20002BFCD0C36AD367D36F002BFCD0C078D1
S31500002A3040EA0120A2F87C0070474FF06041CA6F5F
S31500002A40002AFCD081F87C00704700000441000099
S31500002A50A52E5AE2FCED00E0800E00E048E0FF1FE4
S31500002A6070B5034645480D460468208B42B133EAEB
S31500002A70000101D0062109E098432083022070BDA1
S31500002A8010EA030101D06183F6E705216383284636
S31500002A9000F084FD012070BD024670B5384800EB99
S31500002AA0810050F8044C002C22D0208B1043208348
S31500002AB06178658B062918D0052919D1284217D0C7
S31500002AC005EA00016183A8432083204600F023F92C
S31500002AD0208BA843208301206070022084F8200008
S31500002AE02046BDE8704000F03CBD35EA0001EAD062
S31500002AF070BD234A02EB810151F8041C002902D063
S31500002B000A8B82430A83704702461D4810B500EBC4
S31500002B10810050F8040C002806D0114600F00FF989
S31500002B20BDE8104000F067BC10BD14480068408B3B
S31500002B30704710B50446008B084320836278618B8A
S31500002B40062A16D0052A17D1084215D001EA000236
S31500002B50628388432083204600F0DDF80120607000
S31500002B60022084F820002146BDE81040054800F008
S31500002B700BB831EA0002ECD010BD000054E0FF1F94
S31500002B8060E0FF1F00F2FF1F30B502780024022A22
S31500002B9003D0012A01D0032A00D101248B7800E05A
S31500002BA01046426812B195789D42F9D24A6041605A
S31500002BB01CB102B19160886030BD0020FBE7014680
S31500002BC04068002342684A600A78022A05D0012A32
S31500002BD003D0032A01D04360704742680AB191606E
S31500002BE04360836070476A494A6842600022826097
S31500002BF0486070476649674B48681B6882789B78CF
S31500002C009A4202D142684A60704700207047816844
S31500002C1039B142684A604168002901D080688860FD
S31500002C2070475B4906E04A68824202D140684860C4
S31500002C30704711460029F6D1704710B583680446DF
S31500002C402BB9607801280DD1514B03E09B681878A9
S31500002C500028FBD02046FFF7DAFF2146BDE81040EA
S31500002C60184691E710BD4A4A10B51832D368ABB181
S31500002C7013469B8A03E08CB12246A48A2344D46877
S31500002C808B42F8D3C460D0600261C46804B120618D
S31500002C90591A8182908A401A908210BD0024C4601D
S31500002CA0D060C91A02619182848210BD70B5384E17
S31500002CB01836F06800282DD0B08A401EB082002554
S31500002CC022E0A06838B161684160606810B1A1680F
S31500002CD081606560A56021462D48FFF755FFA08AF3
S31500002CE0B0826078042804D12B49E08A0988084418
S31500002CF0A0820120607084F82000E068F060E0683F
S31500002D0008B10661E5602561B08A002802D1F46841
S31500002D10002CD6D170BD10B5016900290ED0C2684D
S31500002D20CA60C36800223BB18B8A848A23448B82A3
S31500002D30C3681961C26000E08A82026110BDF0B406
S31500002D40164FBC1CFE783D46D4E84F3FB34202D135
S31500002D50BFF32F8F0EE05B1CC4E8423F002AF3D17D
S31500002D60D5E84F3F5A1CB24200D10022C5E8442F95
S31500002D70002CF5D1FA789A4205D907EBC302C2E9CD
S31500002D800101F0BC7047F0BC0220FDF7D1BD000088
S31500002D9000F2FF1F54E0FF1F5CE0FF1F680E0020DB
S31500002DA00122027000224270426002814281103983
S31500002DB08281C1F38F01C18170472DE9F041174629
S31500002DC00C468189994D4268002602B149B1C389F2
S31500002DD0994229D1BFB195490968BAB1FFF7D4FE26
S31500002DE01BE0FFF7ECFE0746C0690460042087F885
S31500002DF020003846FFF78FFF384600F0B2FB286800
S31500002E0080F8206025E00120BDE8F0814160296856
S31500002E104E60296888600121417028680821C461D4
S31500002E20384600F0BBFBEEE7018900EB81010C613F
S31500002E3000F10C01D1E85F2F521CC1E8532F002B83
S31500002E40F8D10189491C89B20181C289914200D118
S31500002E5006810020D8E72DE9F04104468089734FAA
S31500002E6090460D460026A8B3608904EB80000069F1
S31500002E7008606089401C80B26081E189884200D187
S31500002E8066816068E0B12046FFF799FE80F8206011
S31500002E902189054604EB8101C06908612089401C2F
S31500002EA080B22081E189884200D126812846FFF739
S31500002EB032FF284600F055FB386880F8206007E0AE
S31500002EC00C34D4E85F0F401EC4E8510F0029F8D136
S31500002ED0002099E7FFE7B8F1000F07D05349606873
S31500002EE0096828B12046FFF74FFE06E001208BE770
S31500002EF0616038684660386884600821404600F0A2
S31500002F004DFB3868C561F1E7C1898089081A7047A9
S31500002F1010B5FFF714FFBDE8104000F06CBA10B50D
S31500002F2004468089002822D0608904EB800000696D
S31500002F3008606078012807D10220607000212046D1
S31500002F40FFF7FDFE00F057FA04F10C00D0E85F1F12
S31500002F50491EC0E8521F002AF8D16089401C80B281
S31500002F606081E189884201D100206081042010BD82
S31500002F702DE9F041044640680F46002204F10C0595
S31500002F8020B16078022819D0A089A0B3A089E18970
S31500002F90884245D2208904EB80000761D5E85F0F9F
S31500002FA0401CC5E8510F0029F8D12089401C80B289
S31500002FB02081E189884200D1228125E71746627087
S31500002FC02046FFF7FCFD80F820702189064604EBB9
S31500002FD08101C0690861D5E85F0F401CC5E8510F43
S31500002FE00029F8D12089401C80B22081E1898842DD
S31500002FF00BD1278109E0FFE72046FFF7E0FD0646F3
S31500003000C0690421076086F82010012070703046E0
S31500003010FFF781FE3146BDE8F0410548FFF7B4BD34
S31500003020BDE8F0410320FDF783BC000054E0FF1F1C
S3150000303000F2FF1F10B5002A06DA22F00042D21D68
S3150000304022F00703102203E0D21C22F003030C2215
S3150000305013B19C188C4201D9012010BD02440144D1
S315000030608360C0E90021C91AD018884202D81060CE
S315000030700246F9E70020106010BD014651E8000F36
S3150000308028B1036841E80032002AF7D17047BFF340
S315000030902F8F704710B50446FDF74CFA002807D06D
S315000030A0A1680246002903D0002308C2091FFCD1EB
S315000030B010BD814202D342688A4201D8012070477E
S315000030C050E8002F0A6040E80012002AF8D10020DC
S315000030D0704700000321017000214170418041606A
S315000030E0816070472DE9F0470446408820B13F4E85
S315000030F0A1683268914202D0FF20BDE8F087401EE9
S315000031000004000C60803ED131686078DFF8E08012
S31500003110887061684FF00009012739B32046FFF730
S315000031204EFD0546052085F820002846FFF7F3FDED
S315000031306780A560A87860703168D8F804008A783E
S315000031408078824201D328460AE02948FFF71CFD11
S3150000315029462748FFF718FD306847706F7010E062
S3150000316000F0FFF9316881F820900CE0D8F80410DF
S315000031708A783168824206D91D48FFF705FD306816
S3150000318047700020ECE70020B7E770B5174D0E46F4
S3150000319004464188286839B1A168814208D160880F
S315000031A0401C6080002070BDA06080786070F6E7EB
S315000031B076B162788078824203D28870A068FFF781
S315000031C03CFD606830B120462968FFF7DDFC08E069
S315000031D0012070BD28686060296800204860286862
S315000031E084600921304600F0D9F9F1E754E0FF1F69
S315000031F000F2FF1F022202700022426041807047E7
S3150000320010B5416889B1FFF7DAFC0446032084F85B
S3150000321020002046FFF77FFD204600F0A2F9234953
S315000032200020096881F8200002E04188491C41809D
S31500003230002010BD10B50C46418819B1491E4180C9
S31500003240002010BD34B1194A4368116823B1FFF755
S315000032509BFC07E0012010BD416013680021596006
S31500003260116888600721204600F098F9F2E710B54A
S315000032700021FFF764FDBDE8104000F0BCB810B5B2
S31500003280416879B1FFF79BFC0446FFF744FD012036
S315000032906070032084F820002146BDE810400448F1
S315000032A0FFF772BC4188491C418010BD54E0FF1FE6
S315000032B000F2FF1F30B58D4901228D4C48684FF052
S315000032C0E023002808DA052018610A70226800EA5F
S315000032D09260887040060EE000F01F0502FA05F5C0
S315000032E0401103EB8000C0F880510A702068C0F3DB
S315000032F000708870C006206030BD10B54FF6FF74B0
S31500003300FFF7D8FF7B48C16801B1848A7A48016813
S3150000331019B18088A04200D20446204610BDF0B5FF
S31500003320724A002310465168714C80784FF0E026AF
S31500003330002907DA072131611370517840EA8100CC
S3150000334080060CE001F01F070125BD40491106EB80
S315000033508101C1F8005113705178084300072060BD
S315000033605370F0BD2DE9F041054664480126016819
S315000033704E700068FFF737FC61490020614F086016
S315000033805C49C868D0B1888AA84211D83A682C1A14
S31500003390104438608E828846FFF788FC8CB1386806
S315000033A0641E401C3860D8F80C000028F4D108E0F0
S315000033B03B685A19401B3A60888202E03868284404
S315000033C038604D4F386870B1B888A84209D82C1AB1
S315000033D0BE8000F08FFA34B13868641E0028F8D138
S315000033E001E0401BB8804848FFF7E9FB00F0B4F85D
S315000033F0BDE8F04193E73D48017811B101214170E4
S3150000340070473B494FF080500860704770B53B48A5
S315000034100121026851700068FFF7E5FB3B4D6C78AF
S3150000342016E005EBC40148680278E2B1012A1FD014
S31500003430FFF725FFE878641C844200D10024334856
S31500003440801CD0E84F1F491EC0E8421F002AF8D151
S31500003450A8780028E5D16C702B48FFF7B0FBBDE8D3
S31500003460704000F079B8098989B2FFF762FBE1E79D
S315000034708968FFF77DFDDDE7254801684FF0E0200C
S315000034804161002181610721016119481C300168F1
S3150000349041F07F410160401770477047174810B5EB
S315000034A00268012151700068FFF79DFBFDF742FAA3
S315000034B014480168491C0160FFF7F8FB00F01AFA8E
S315000034C01148FFF77CFBBDE8104000F045B80B48FB
S315000034D00068D0E90910814203D300680D4988428B
S315000034E002D00120FDF724BA704700001001002029
S315000034F004ED00E018F2FF1F1801002054E0FF1F42
S315000035004CE0FF1F5CE0FF1F00F2FF1F680E00206B
S3150000351008410000A52E5AE270B504460020154663
S31500003520207001226270A1706060A060E06020617E
S31500003530A082E0822083608384F8200084F8210042
S31500003540608C18B9C648FFF798FDA0622946204648
S31500003550BDE87040FFF72EBAC249486002214170AB
S31500003560704770B504000ED0BE4DA17801262868BC
S31500003570827891420BD9FFF736FB286846702046C1
S31500003580BDE87040E8E7B848FFF719FBF8E7667052
S315000035902146BDE87040B448FFF7F6BA70B50D464F
S315000035A0002811D04FF6FF71AE4C884204D2226833
S315000035B001461046FFF757FB20684570AA48FFF7FB
S315000035C0FEFABDE87040C7E770BD70B5FFF712FBA5
S315000035D004000BD0A34DA4482968FFF7D5FA296843
S315000035E0012048702046BDE87040B5E770BD9D4893
S315000035F00068002800D0C078704770B5994D002645
S3150000360070B19A4A128890421DD8994A02EB8000FE
S3150000361050F8044CBCB1A1702868A04202D014E056
S315000036202868817090484068807888421BD98E4807
S315000036302968FFF7A9FA296801204870286880F8E8
S31500003640206000200DE0FF2070BD2046FFF7F5FA50
S315000036506078012807D18448FFF7B1FA296881F814
S315000036602060FFF77EFF002070BD2DE9F0411E4669
S31500003670174680460C4611F0FF0F00D14C1C7D48C2
S31500003680FFF7FBFC050024D0C4F30F20AF6268846B
S31500003690E1B242462846EE61FFF73EFF0124744838
S315000036A0724905E000EB840252F8042C22B1641C36
S315000036B00A889442F6D9002400EB840040F8045CA2
S315000036C0EC702846FFF74DFF6648006880F82040FA
S315000036D02046BDE8F08170B5624C654E0025216834
S315000036E010B1CA7882421AD14D70FCF712FF2168D8
S315000036F04862FFF7ECFE2068C17806EB810141F8CD
S31500003700045C816A5648FFF7D4FC216859488D62EB
S31500003710FFF7CFFC00202560FFF723FF19E0534990
S315000037200988884217D806EB800656F8044C94B1EF
S315000037302046FFF76CFA2046FFF7EDFA46F8045CE0
S315000037404748A16AFFF7B5FC21464A48A562FFF73C
S31500003750B0FC002070BDFF2070BD2DE9F04781460A
S3150000376016468846002005464149404A02E041F88F
S315000037702050401C13889842F9D33F4830220188D4
S315000037803C48FFF757FC3D48008880B240F00042B5
S315000037903B4801683248FFF74DFC3A480822018849
S315000037A039480068FFF746FC384CFF27384AE7706F
S315000037B0658400212046FFF7AFFE2B4804210170E7
S315000037C0456034480170C56005618582606A2030B5
S315000037D0FCF79CFE234831490460022060702E48A5
S315000037E0057045700978C170FDF7A3F82C4801688B
S315000037F041F47F0101600068390601EA002028498A
S31500003800C0431439B0FA80F00968C0F10800C1F36A
S315000038100221814200DB481C2149091F0B686FF019
S315000038208072824063F317020A60FFF725FE1D4986
S31500003830002808600CDB1C49475400F01F020121D8
S31500003840914040114FF0E02202EB8000C0F80011D9
S31500003850324641464846BDE8F047002305E70000EA
S315000038605002002054E0FF1F00F2FF1F004100003D
S3150000387060E0FF1F20010020184100000441000005
S315000038801C410000224100000000002060150020BD
S315000038902D09000018F2FF1F680E002020410000CD
S315000038A020ED00E01401002000E400E00F4800686D
S315000038B070470321FFF772BE0D490C4A0968C8829A
S315000038C012881044888270470948016807488A8A26
S315000038D00088CB8AA2EB00001A4480B28A820104D7
S315000038E002D40421FFF75ABE704700005CE0FF1FB8
S315000038F054E0FF1F70B52A4D2868002815D0A88807
S31500003900284E401EA8800AE0E088FDF710F8A0883F
S31500003910A8802068286021463068FFF7CAFBA8887F
S31500003920002802D12C68002CEED170BD70B50D4672
S3150000393004000AD01B48006838B1FFF79EFB002838
S3150000394004D01749C5808A8804E0002070BD194656
S315000039509B881A44A24202D20B68002BF7D10B684F
S31500003960121B0360828008608A888388D21A8A8044
S3150000397070BD10B50A4A02E000290FD00A46116848
S315000039808142F9D101681160918883881944918038
S31500003990014604480068FFF78CFB002010BD0000BC
S315000039A018010020000000200048704790150020F4
S315000039B010B5431C02E010F8011B71B18107FAD162
S315000039C04FF0013202C88C1A8C4314EAC211F9D0A6
S315000039D0C01A0A0603D0C01E10BDC01A10BD0A04C4
S315000039E001D0801E10BD0902FCD0401E10BD032A66
S315000039F040F2308010F0030C00F0158011F8013B06
S31500003A00BCF1020F624498BF11F801CB00F8013BEC
S31500003A1038BF11F8013BA2F1040298BF00F801CBB0
S31500003A2038BF00F8013B11F0030300F04A80083A62
S31500003A30C0F0088051F8043B083A51F804CBA0E8DE
S31500003A400810F5E7121D5CBF51F8043B40F8043B33
S31500003A50AFF30080D20724BF11F8013B11F801CB68
S31500003A6048BF11F8012B24BF00F8013B00F801CB39
S31500003A7048BF00F8012B70474FF000020429C0F040
S31500003A80128010F0030C00F05080CCF1040CBCF155
S31500003A90020F18BF00F8012BA8BF20F8022BA1EBDC
S31500003AA00C0100F042B85FEAC17C24BF00F8012B8C
S31500003AB000F8012B48BF00F8012B7047704770478C
S31500003AC0704710B5203AC0F00B80B1E81850203A84
S31500003AD0A0E81850B1E81850A0E81850BFF4F5AFA8
S31500003AE05FEA027C24BFB1E81850A0E8185044BF32
S31500003AF018C918C0BDE810405FEA827C24BF51F89F
S31500003B00043B40F8043B08BF7047D20728BF31F892
S31500003B10023B48BF11F8012B28BF20F8023B48BFE3
S31500003B2000F8012B70474FF0000200B5134694468B
S31500003B309646203922BFA0E80C50A0E80C50B1F1FF
S31500003B402001BFF4F7AF090728BFA0E80C5048BF13
S31500003B500CC05DF804EB890028BF40F8042B08BFB1
S31500003B60704748BF20F8022B11F0804F18BF00F8AD
S31500003B70012B70477546FFF717FFAE4605006946ED
S31500003B80534620F00700854618B020B5FCF776FDB1
S31500003B90BDE820404FF000064FF000074FF0000848
S31500003BA04FF0000B21F00701AC46ACE8C009ACE8C9
S31500003BB0C009ACE8C009ACE8C0098D4670470446A8
S31500003BC0AFF300802046FCF798FC0000014918205E
S31500003BD0ABBEFEE7260002007047000003000000AF
S31500003BE0A914000025080000290800007CB54649F4
S31500003BF0A1F120050878A1F1080410F01F0002D0F9
S31500003C0001287BD168E04048CE7820383F4AC17809
S31500003C102030082E807871D2DFE806F07004134257
S31500003C207070082D3A482060122052E0107808B9CA
S31500003C30012963D019B1374820600A2049E0364887
S31500003C40FAE712780AB9012958D019B13349009117
S31500003C50002108E03249FAE7009A137813B1538835
S31500003C601A440092491C8842F6D10098017891B313
S31500003C70206040882DE012780AB901293ED019B19A
S31500003C8028490091002108E02749FAE7009A1378AD
S31500003C9013B153881A440092491C8842F6D1E4E7CE
S31500003CA022490091032801D000210BE0FDF7C2FA5A
S31500003CB02060FDF7B5FA0CE0009B1A780AB11A44A9
S31500003CC00092491C8842F7D10098017819B120600A
S31500003CD00078019006E011E001A96846FCF76AFE4B
S31500003CE000280CD0A188019881420BD9104980B2D6
S31500003CF0A0800978491E084202D003E000207CBD5E
S31500003D000120287101207CBD3CE0FF1F25410000F9
S31500003D10884100009B4100009A410000BD4100001F
S31500003D209C410000BF410000BE410000C0410000B0
S31500003D302841000070B51C481B4C0078A4F108040B
S31500003D4010F01F000AD0184AA4F11803174D59782D
S31500003D501279012806D0022824D109E012481A381F
S31500003D6020601DE0F1B1987882421BD2002015E058
S31500003D7002F08F00020605D500F00F064FF48032E0
S31500003D80B24001E00122824009B900070AD19868D1
S31500003D90104207D0D868104000D001202880256046
S31500003DA0012070BD002070BD3CE0FF1F090000200F
S31500003DB070B5264B024619461878498810F01F0040
S31500003DC0A3F1200604D0012829D0022827D111E02A
S31500003DD0012924D132B10120FDF70CFCF08840F016
S31500003DE0020005E00020FDF705FCF08820F0020047
S31500003DF0F08029E0187900F08F04200605D504F03C
S31500003E000F004FF48035854001E00125A54070780C
S31500003E1028B1200703D0B068284200D009B100209D
S31500003E2070BD2AB12046FDF74FFCF06828430AE032
S31500003E303069284208D12046FDF751FC2046FEF79E
S31500003E4075F8F068A843F060012070BD3CE0FF1FE4
S31500003E502DE9F05F5A480026017811F01F0F7DD139
S31500003E60574F8078203FB1464FF0010A4FF4803B10
S31500003E70002879D0534801783846C07809B9012816
S31500003E806CD008B1504C68E0504C66E0607802286F
S31500003E9004D0042844D005285DD143E04848617920
S31500003EA0807881423AD178702079B87000204849EC
S31500003EB0484A02E001F80090401C13889842F9D362
S31500003EC00125B8460AFA05F0D8F80810084202D0CB
S31500003ED02846FDF7E5FBD8F808100BFA05F008426E
S31500003EE003D045F08000FDF7DBFB6D1C102DE9D3F8
S31500003EF04FF00110C8E902090120C8F81090FDF73B
S31500003F0082FBE0794006B8F8060002D540F00100D1
S31500003F1001E020F00100A8F806001CE060881BE024
S31500003F20E67818E0BEB9A07800F08F05280604D51B
S31500003F3005F00F010BFA01F001E00AFA05F0B96885
S31500003F4001432046B960FDF78EFB2846FDF794FB3A
S31500003F502846FDF759FB2078044401E02AE003E0F7
S31500003F602078002892D120E04D4687F80190012460
S31500003F705E46B9680AFA04F0084202D02046FDF708
S31500003F808FFBB96806FA04F0084203D044F08000BB
S31500003F90FDF786FB641C102CEBD34FF00110C7E92C
S31500003FA0020500203D61FDF72EFB054879788078F3
S31500003FB0884202D00020BDE8F09F0120FBE7000008
S31500003FC03CE0FF1F25410000BD4100009C41000070
S31500003FD008000020264100002DE9F84F434800273D
S31500003FE03E460078BA4600F01F00B94601287BD14C
S31500003FF03E4920394878002873D0002000903C487C
S3150000400002780846C0780AB901286DD08B4608B1F7
S31500004010384C62E0384C60E06078022804D004280E
S3150000402009D0052857D118E061799BF80100814233
S3150000403051D0608850E02D48A778E67801794FF096
S315000040400009B94247D18078B04244D1012000909E
S315000040502A4810F807A0C6553DE024490879B84219
S3150000406039D1A07800F08F085FEA086005D508F01E
S315000040700F004FF48035854002E0012505FA08F56A
S315000040808878B04215D1DBF8081020462943CBF8D2
S315000040900810DBF80C10A943CBF80C10FDF7E3FA77
S315000040A04046FDF7E9FA4046FDF7AEFA49EA05094A
S315000040B011E056450FD119EA050F0CD1DBF80810AF
S315000040C04046A943CBF80810DBF80C10A943CBF8FF
S315000040D00C10FDF7E5FA20780444207800289BD1DF
S315000040E00098BDE8F88FFFE70020FAE73CE0FF1FE5
S315000040F025410000BD4100009C4100000800002051
S3150000410006000000B8010001FF5207000100000090
S3150000411010270000000000002C010000180C000011
S315000041200400000000000100080002024000000236
S315000041300000000000000000000000000100000078
S315000041400000000000000000EB1E00000000000060
S315000041507D290000000000000000000000000000B3
S315000041600000000000000000000000000000000049
S315000041700000000000000000000000000000000039
S3150000418000000000000000001201100100000008FD
S31500004190280D0402000101020301000009022000AB
S315000041A001010080FA090400000208065004070510
S315000041B082024000000705020240000000000000E5
S315000041C0040309040A034D004200450044001E038F
S315000041D04D00420045004400200043004D005300BE
S315000041E0490053002D004400410050001A033000DE
S315000041F03000300031004100300030003000300027
S3150000420030003000300010035500530042005F00BC
S315000042104D0053004300EB3C904D5357494E342E0E
S315000042203100020801000220003001F00300010005
S3150000423001000000000000000000000029741902BF
S31500004240274D626564205553422020204641543153
S3150000425032202020000000000000000000000000C6
S315000042600000000000000000000000000000000048
S315000042700000000000000000000000000000000038
S315000042800000000000000000000000000000000028
S315000042900000000000000000000000000000000018
S315000042A00000000000000000000000000000000008
S315000042B000000000000000000000000000000000F8
S315000042C000000000000000000000000000000000E8
S315000042D000000000000000000000000000000000D8
S315000042E000000000000000000000000000000000C8
S315000042F000000000000000000000000000000000B8
S3150000430000000000000000000000000000000000A7
S315000043100000000000000000000000000000000097
S315000043200000000000000000000000000000000087
S315000043300000000000000000000000000000000077
S315000043400000000000000000000000000000000067
S315000043500000000000000000000000000000000057
S315000043600000000000000000000000000000000047
S315000043700000000000000000000000000000000037
S315000043800000000000000000000000000000000027
S315000043900000000000000000000000000000000017
S315000043A00000000000000000000000000000000007
S315000043B000000000000000000000000000000000F7
S315000043C000000000000000000000000000000000E7
S315000043D000000000000000000000000000000000D7
S315000043E000000000000000000000000000000000C7
S315000043F000000000000000000000000000000000B7
S3150000440000000000000000000000000000000000A6
S315000044100000000055AAF0FFFFFFFFFFFFFFFF00AF
S3150000442000000000000000004641494C20202020EA
S315000044305458542018B174768E418E4100008E7601
S315000044408E410600070000002E202020202020207C
S315000044502020201000A5858A734373430000868AB6
S3150000446073430300000000002E2E20202020202071
S315000044702020201000A5858A734373430000868A96
S3150000448073430000000000004247007500690064A5
S315000044900000000F00FFFFFFFFFFFFFFFFFFFFFF12
S315000044A0FFFF0000FFFFFFFF0149006E006400658B
S315000044B00078000F00FF6500720056006F006C0068
S315000044C0750000006D006500494E444558457E3133
S315000044D02020202000A7858A734373430000868A24
S315000044E0734304004C0000007B00390036003600A0
S315000044F0310039003800320030002D003700370017
S31500004500440031002D0034004600380038002D00EC
S3150000451038004600350033002D00360032004400D6
S315000045203900370046003500460034004600460094
S3150000453039007D00000000000042494E00000000E6
S315000045400062696E00000000015041520000000048
S3150000455002444F570000000003435244000000008D
S315000045600500000000000000424F4F544C4F4144EC
S31500004570455220280000000000000000000085755C
S315000045808E41000000000000412E006600730065A9
S315000045900076000F00DA65006E0074007300640098
S315000045A000000000FFFFFFFF46534556454E7E3193
S315000045B02020201200477D758E418E4100007D75BA
S315000045C08E4102000000000042650072005F006933
S315000045D0006E000F00A86400650078000000FFFF71
S315000045E0FFFF0000FFFFFFFF012E006D0065007456
S315000045F00061000F00A864006100740061005F00A4
S315000046006E000000650076004D45544144417E3100
S3150000461020202022003285758E418E41000085754E
S315000046208E41000000000000412E0054007200611F
S315000046300073000F00256800650073000000FFFF8F
S31500004640FFFF0000FFFFFFFF5452415348457E31F4
S3150000465020202022003285758E418E41000085750E
S315000046608E4100000000000042200049006E0066F6
S31500004670006F000F007272006D0061007400690027
S315000046806F0000006E000000015300790073007493
S315000046900065000F00726D00200056006F006C0070
S315000046A0750000006D00650053595354454D7E3129
S315000046B02020201600A5858A734373430000868A4E
S315000046C07343030000000000424F4F544C4F4144D7
S315000046D048544D2018B174768E418E4100008E7676
S315000046E08E41050000020000002E20202020202000
S315000046F0202020203200477D758E418E41000088A3
S31500004700758E410200000000002E2E202020202061
S31500004710202020201000477D758E418E4100007DAF
S31500004720758E410000000000004E4F5F4C4F472041
S315000047302020202020083285758E418E410000857C
S31500004740758E410000000000003C212D2D206D6279
S315000047506564204D6963726F636F6E74726F6C6C03
S315000047606572205765627369746520616E642041C5
S31500004770757468656E7469636174696F6E205368D9
S315000047806F7274637574202D2D3E0D0A3C212D2DFC
S315000047902056657273696F6E3A203032303120428E
S315000047A075696C643A2046656220323520323031B4
S315000047B0342031363A35303A3231202D2D3E0D0A2D
S315000047C03C68746D6C3E0D0A3C686561643E0D0A7A
S315000047D03C6D65746120687474702D6571756976B9
S315000047E03D22726566726573682220636F6E74651A
S315000047F06E743D22303B2075726C3D687474703A5D
S315000048002F2F6D6265642E6F72672F6465766963FC
S31500004810652F3F636F64655F626C3D4041222F3EAA
S315000048200D0A3C7469746C653E6D6265642057655B
S3150000483062736974652053686F72746375743C2F74
S315000048407469746C653E0D0A3C2F686561643E0DA3
S315000048500A3C626F64793E3C2F626F64793E0D0AB2
S315000048603C2F68746D6C3E0D0A0D0A0030313233F0
S31500004870343536373839414243444546006B346651
S315000048806C75356673004D424544202020206D69C5
S3150000489063726F6E74726F6C6C6572202020312E9D
S315000048A030200042414420455854454E53494F4E0E
S315000048B02046494C450053574420504F52542049F6
S315000048C04E2055534500535744204552524F5200EF
S315000048D042414420535441525420534543544F526D
S315000048E0004E4F5420434F4E534543555449564569
S315000048F020534543544F5253005245534552564553
S315000049004420424954530054494D454F55540030B4
S31500004910323031005449000000E0FF1F6000000003
S31500004920A8040000B4490000000000202001000097
S31500004930A8040000B449000060E0FF1FD014000086
S31500004940C4040000D44A000020010020D014000056
S31500004950C4040000006CDC0200000000000000003F
S3150000496000000000000000005555555500000000ED
S315000049700000000000000000000000000000000031
S315000049800000000000000000000000000000000021
S315000049900000000000000000000000000000000011
S315000049A00000000000000000000000000000000001
S315000049B00000000000000000864800000000000023
S315000049C000000000000000000101000000000000DF
S315000049D0000000000050000007000000000000007A
S315000049E000000000000000000000000000000000C1
S315000049F000000000000000000000000000000000B1
S31500004A0000000000164200000002000016440000EC
S31500004A1010000000264400000000000026440000AC
S31500004A2000000000264400000000000026440000AC
S31500004A300000000026440000000000006845000059
S31500004A4080010000E846000001000000E946000081
S31500004A506000000078E0FF1F00020000C64800006A
S31500004A60A3480000E1480000B6480000F9480000ED
S31500004A70D048000007490000000000000F49000070
S31500004A800000000000000000000000000000000020
S31500004A900000000000000000000000000000000010
S31500004AA00000000000000000000000000000000000
S31500004AB000000000000000000000000000000000F0
S31500004AC000000000000000000000000000000000E0
S31500004AD000000000FFFFFFFFFFFFFFFFFFFFFFFFDC
S31500004AE0FFFFFFFFFFFFFFFFFFFFFFFFFFFFFFFFD0
S31500004AF0FFFFFFFFFFFFFFFFFFFFFFFFFFFFFFFFC0
S31500004B00FFFFFFFFFFFFFFFFFFFFFFFFFFFFFFFFAF
S31500004B10FFFFFFFFFFFFFFFFFFFFFFFFFFFFFFFF9F
S31500005000701E00202957000031570000335700005A
S3150000501035570000375700003957000000000000E0
S315000050200000000000000000000000008D54000099
S315000050303D570000000000001555000065550000B2
S3150000504043570000435700004357000043570000F2
S3150000505043570000435700004357000043570000E2
S3150000506043570000435700004357000043570000D2
S3150000507043570000435700004357000043570000C2
S315000050804357000043570000598A00004357000069
S3150000509043570000435700004357000043570000A2
S315000050A04357000043570000435700004357000092
S315000050B04357000043570000435700004357000082
S315000050C04357000043570000435700001D8F000060
S315000050D04357000043570000435700004357000062
S315000050E043570000E987000043570000435700007C
S315000050F04357000043570000435700004357000042
S315000051004357000043570000435700004357000031
S315000051104357000043570000435700004357000021
S315000051204357000043570000435700004357000011
S31500005400FFFFFFFFFFFFFFFFFFFFFFFFFEFDFFFFA9
S31500005410DFF80CD006F0F6FF0048004739640000BC
S31500005420701E002080F309887047EFF309807047EB
S31500005430684680F3098804480078C00714BF022034
S31500005440032080F31488704768C50000DFF818C091
S31500005450EFF305831B0618BF6047EFF31483DB07E2
S3150000546008BF604700DF70470DBB0000DFF818C0BB
S31500005470EFF305831B0618BF6047EFF31483DB07C2
S3150000548008BF604700DF70474BBB0000EFF30980A1
S31500005490816911F8021C39BB90E80F10E047EFF361
S315000054A0098C194B93E80600914218D059B10CB4F7
S315000054B04FF0010381F821302CE9F00FC1F824C028
S315000054C006F0D4FC0CBC1A60D2F824C0BCE8F00F7D
S315000054D092F821308CF309881BB192F82000CCF8A1
S315000054E000006FF0020E704710B5084A126891422C
S315000054F009D8074C54F8214090E80F10A047EFF365
S31500005500098C8CE80F0010BDD4E5FF1F84C4000091
S3150000551084C4000006F048FC114B93E80600914253
S315000055201BD00CB44FF0000381F82130EFF3098C47
S315000055302CE9F00FC1F824C006F098FC0CBC1A60E8
S31500005540D2F824C0BCE8F00F8CF3098892F8213019
S315000055501BB192F82030CCF800306FF0020E704785
S31500005560D4E5FF1F06F069FCD6E7000006F064FCF0
S3150000557006F063FCD0E7000063484CF22051C1817D
S315000055804DF62811C1814FF4E97101805F494FF44E
S31500005590881048645E48002101705E480173242229
S315000055A042709A220270C27802F01F02C270032271
S315000055B002714171817911F0020FFBD0817901F0FE
S315000055C00C010829FAD1027140214171817911F04B
S315000055D0200FFBD0817911F0400FFBD01A2101700A
S315000055E00C21827931EA0202FBD1817911F0400F58
S315000055F0FBD049494FF4A04008607047454A1078EF
S315000056004FF0010C10F0C00F444819D0117801F08A
S31500005610C00140296AD0117801F0C001802918BF65
S315000056207047117B11F0010F01D04FF4004037494C
S31500005630496C0CEB1171B0FBF1F039490860704709
S31500005640517911F0400F0AD0117901F01F01491C60
S31500005650B0FBF1F0517901F01F01183140E01178EB
S3150000566011F0040F18BF4FF400400ED0D17801F0AE
S31500005670E00111F01F0FDAD149110829D7D2DFE86E
S3150000568001F0181B1F23272A2D31117B11F0010F62
S3150000569018BF4FF400401178C1F3C2010CFA01F1B2
S315000056A0C9B2B0FBF1F0517811F0300F18BF4009C4
S315000056B0DCE700EB800005E000EB80000002B6E7C7
S315000056C0C0EB0010C001B2E700EB80004002AEE77D
S315000056D04FF4377104E04FF4B76101E040F69501ED
S315000056E04843A4E740F671314843A0E7507810F0EC
S315000056F0010F9AD0107A0B49C0F342000CFA00F061
S31500005700B1FBF0F093E70000002005400080044064
S31500005710005006400040064008ED00E000127A0006
S3150000572000E0FF1F00093D00064880470648004785
S31500005730FEE7FEE7FEE7FEE7FEE7FEE7FEE7FEE73B
S31500005740FEE7FEE779550000115400004FF47A5148
S315000057504843401EFDD17047FF2008700120704766
S315000057602DE9F84F0278A2F180031F2B03D800F031
S3150000577029FCBDE8F88F01F8012B89460178461C03
S31500005780172980F05482DFE801F00C3B4A79FBFAD6
S31500005790F9F8F7969BF8F8F8F8F8A1F6F5F4F3F3AC
S315000057A0F3003078002209F10101052823D007DC37
S315000057B001281CBF022803281DD0042809D01AE09E
S315000057C0062818D0F02809D0FE2811D0FF2809D0C5
S315000057D011E0FC480422006808600CE00120087013
S315000057E0024608E04020087000204870022202E0CD
S315000057F005200870012289F80020901CBDE8F88F6A
S31500005800307820B1012800F00B8100F0F4B87078F0
S31500005810ED4900F00100C043086000F001B934789A
S31500005820002C08BF012400F022FE012C40F0F88075
S31500005830E649012020220870E549CA674022CA6766
S31500005840086410220A600222CA63CB6843F0100380
S31500005850CB600B6843F010030B600B6C43F0010345
S315000058600B64CA63CA6C42F00202CA64D94A40F2A7
S315000058701311516089F8000000F0A0B9D348002543
S3150000588001240570D448446410214160022141641A
S31500005890816C41F02001C0F88810CE48416841F083
S315000058A080714160CD49416000F0E0FD89F800500B
S315000058B0204600F083B930880001401EFDD1AFE0DC
S315000058C0002089F8010089F80000D4E07078737927
S315000058D0D6F80220317863F31F6210F0010F0AD068
S315000058E0DFF8F4C211F0010F4FF020030CBFCCF823
S315000058F08830CCF8843010F0020F0AD0DFF8D8C216
S3150000590011F0020F4FF040030CBFCCF88830CCF8F2
S31500005910843010F0800F04D0DFF8C4C2CB09CCF875
S31500005920003072B3AF4B9A4288BF1A4600234FF03D
S31500005930E02CCCF81830AC4C6243AC4CB2FBF4F221
S31500005940CCF814200522CCF81020A34C10F0010F3F
S3150000595018BF002929D110F0020F06D0D4F89020E4
S31500005960C2F3C012B2EB510F1FD110F0040F09E0C1
S315000059704CE163E059E031E044E158E182E071E056
S3150000598066E01AE018BFB3EB910F0ED110F0200FAE
S3150000599018BFB3EB511F08D110F0800F0BD0226D4A
S315000059A0C2F34002B2EBD11F05D0DCF81020C2F3DF
S315000059B00042002ACAD0CCF810308D4900204A6D2A
S315000059C04969C2F3C01240EA4200C1F3400140EA0D
S315000059D0C11089F80000012000F0F0B8F1783068B5
S315000059E061F31F6038B18349814209D877490120A4
S315000059F04870486014E0FF2089F800000120DDE0CF
S31500005A00724900224A707C4A0244B2FBF0F0022836
S31500005A1098BF012003D9794AA2FB002040084860BC
S31500005A20002089F800000120C8E03078711C0028A9
S31500005A3008BF4FF4807000F01BFDF1E7307800F0EE
S31500005A4003014A1C6149C0F380000A754875E7E7FF
S31500005A505E4831780172B6F801104181B6F803103C
S31500005A608181DDE759480078012806D0002089F8B1
S31500005A70000089F801000220A0E04946304600F007
S31500005A802AF99BE0514D2878012808D0002089F892
S31500005A90000089F8010089F8020003208EE0DFF893
S31500005AA060B10024204609F103078BF8004036F860
S31500005AB001AFB61CBAF1000F77D016F8018B18F0BB
S31500005AC0020F08BFAAF1010A45D018F0010F18BF4E
S31500005AD06E890FD00021404600F08FFF022802D0C9
S31500005AE0012807D061E0761E5FD39BF800100029DD
S31500005AF0F0D05AE0AAF10106BAF1000F55D026B946
S31500005B0018F0010F18BF4FF00E08B5F80AA0694645
S31500005B10404600F072FF022802D0012808D044E077
S31500005B20BAF1010A41D39BF800100029EFD03CE0FE
S31500005B30009907F8011B0099641C090A07F8011B64
S31500005B400099090C07F8011B0099090E07F8011BBB
S31500005B50761ED4D229E0F17856F8040B61F31F6063
S31500005B6000901A4845896946404600F046FF0228DB
S31500005B7002D0012807D018E06D1E16D39BF800103E
S31500005B800029F0D011E0641CBAF1010AE3D20F48F3
S31500005B90458900210E2000F030FF022805D16D1E38
S31500005BA003D39BF800100029F3D089F80040210A9E
S31500005BB089F8011089F80200A7EB0900401CBDE82E
S31500005BC0F88F00005AC500001018FE43E8E5FF1FD5
S31500005BD008F00F4000A0044000F00F4013010A0037
S31500005BE00408FE43C0C62D00006CDC0240420F00D4
S31500005BF03CF00F40001BB700FF356E01ABAAAAAA06
S31500005C0004E0FF1FE7480078012805D0FF2089F847
S31500005C1000000220BDE8F88F3179D6F8010061F363
S31500005C201F6000906946002000F0E7FEF8E6FF20BE
S31500005C3009F8010C0120BDE8F88FDA4810B44FF0DE
S31500005C40020C6421C0F804C0418101230375D648C3
S31500005C50816B41F4F0518163D44A81155161D44876
S31500005C602024C466C46F44F02004C46791614024B4
S31500005C70C466C46F44F04004C467CC1CD461C26FD0
S31500005C8022F08002C267CB4A1160C362C36B43F045
S31500005C900103C363C84B1961102140F8141C50F866
S31500005CA0043C43F0100340F8043C40F223135360D5
S31500005CB0C0F82CC0C26B42F00202C263DA1EBF4BB0
S31500005CC01A61C0F8B010D0F8BC1041F01001C0F84D
S31500005CD0BC1010BC70472DE9F04F85B0054600207A
S31500005CE0DFF8DCB2029101908C1C8BF8000015F8ED
S31500005CF0011F6D1C491E039107468146491C00F091
S31500005D00478115F8018B18F0020F00F0BE80002FB6
S31500005D1030D0A448468908F0110001280ED1694602
S31500005D20404600F06AFE022815D1761EC0F030818A
S31500005D309BF800100029F2D000F02AB969460E201F
S31500005D4000F05BFE022805D1761E03D39BF80010F7
S31500005D500029F3D00027012840F01A81009904F8A1
S31500005D60011B0A0A04F8012B0A0C04F8012B090E80
S31500005D7004F8011B18F0100F4AD0E87855F804AB68
S31500005D8018F0010F60F31F6A8648B0F80C901CBF2C
S31500005D908448468912D00021404600F02EFE022893
S31500005DA003D001280AD000F0F3B8761EC0F0F080C8
S31500005DB09BF800100029EED000F0EAB87948468931
S31500005DC06946404600F019FE022802D0012807D095
S31500005DD013E0761E11D39BF800100029F0D00CE0DA
S31500005DE07049009A09691140514506D0B9F1010977
S31500005DF003D39BF800100029E0D06A49009A09698C
S31500005E001140514518BF40F0100001284AD133E037
S31500005E10644918F0010F4E8912D06FBB002140462D
S31500005E2000F0EBFD022804D0012808BF012723D08B
S31500005E30AEE0761E36D39BF800100029EED0A7E020
S31500005E406946404600F0D9FD022802D0012807D055
S31500005E509EE0761E26D39BF800100029F0D097E02E
S31500005E60009904F8011B0A0A04F8012B0A0C04F82D
S31500005E70012B090E04F8011B4FF000090199491C7A
S31500005E8001919BF80010D1BB46E0002F1CBF45488E
S31500005E9046891CD069460E2000F0AFFD022802D0CC
S31500005EA0012807D074E0761E72D39BF800100029F3
S31500005EB0F0D06DE0009804F8010B010A04F8011B0C
S31500005EC0010C04F8011B000E04F8010B0027E97809
S31500005ED055F8040B18F0200F61F31F6000901DBFEA
S31500005EE03049086101202F4808BF4689C6D1694656
S31500005EF0404600F082FD022807D0012800E011E0AC
S31500005F0008BF4FF00109B9D042E0761E40D39BF896
S31500005F1000100029EBD03BE00399491E0391491C70
S31500005F207FF4EFAE012833D1002F1CBF1D484589F1
S31500005F301CD069460E2000F060FD022802D0012820
S31500005F4007D025E06D1E23D39BF800100029F0D062
S31500005F501EE0009904F8011B0A0A04F8012B0A0C3A
S31500005F6004F8012B090E04F8011B11E0B9F1000F2A
S31500005F701CBF0C4845890BD000210E2000F03DFDCA
S31500005F80022805D16D1E03D39BF800100029F3D01B
S31500005F90DDE90112117002994870029805B0201AC5
S31500005FA0BDE8F08FE8E5FF1F0080044000B0044024
S31500005FB018F00F4000A004400090044000C00440C8
S31500005FC004E0FF1F70B500780C46802803D0FF2040
S31500005FD00870012070BD01F0A7FE0646001D06F000
S31500005FE0FBF9C5B28020207065702A46311DA01CC1
S31500005FF006F0CEF9A81C70BD00240320DFF8ECC320
S3150000600000DFFB4DFB4EDFF8F0C300DF0220DFF8B8
S31500006010ECC3B16800DFA5FB04104008A0EB8000CC
S31500006020001904F10101CCB2EDD10120DFF8CCC397
S31500006030B16800DFE7E7EF48DFF8C0C381680420F6
S3150000604000DF7047EB49012200280A7014BF0220C6
S315000060500120C8707047E749012200284A7014BF22
S315000060600220012008717047E249012200288A7047
S3150000607014BF0220012048717047DE4821210161CA
S315000060800121C1717047DB48DFF870C381680820C1
S3150000609000DF7047D748DFF864C38168802000DFDF
S315000060A07047D448DFF854C38168102000DF70477A
S315000060B0D048DFF848C38168202000DF7047CD4C08
S315000060C084B00125002202A9CD48DFF838C300DFDD
S315000060D0C8B9029810F0FF0006D0012807D00228A0
S315000060E008D0032809D00EE002F0A6FB0BE002F070
S315000060F0C8FB08E002F0D3FB05E0684601F08BFF21
S31500006100684602F0DFFB03F0CCF84028CCBF402005
S3150000611000280CD081B2BC4802F070FC38B10146B0
S31500006120B94803F0C6F810B165700120207102F07D
S3150000613008FC01464028CCBF40210029C2D0B24805
S3150000614003F0FAF80028BDD081B2AF4802F002FC95
S315000061500028B7D0657001202071B3E7704782B080
S3150000616000204FF001080090474646466021A448AB
S31500006170DFF898C200DFDFF898C200DFDFF874B2FC
S31500006180CBF8080002F0ECFA012002F003FB012034
S3150000619002F009FB012002F00FFB0421DBF80800E6
S315000061A002F015FBC14602F0C5FF01F0CAFD03F07F
S315000061B097FA002003F09DFA4FF0000A8BF807A02B
S315000061C00125CBF810A08BF80650052400F04DF9F8
S315000061D000F04CF98F4A002346F20B41AFF2E7106C
S315000061E0DFF834C200DF022002F065FF00224FF61E
S315000061F0FF71BF20DFF824C200DFDFF824C200DF12
S31500006200054610F0080F05D005248BF807A00620D8
S315000062108BF8060015F0800F05D000248BF807A038
S3150000622006208BF8060015F0040F0ED08BF804A09C
S31500006230002002F0B8FA022002F03DFF01208BF8A0
S31500006240040002F0B0FA4FF0000915F0100F11D05B
S3150000625000F00DF9042002F02EFF002003F049FAA9
S31500006260002002F097FA002002F09DFA002002F0CA
S31500006270A3FAFEE715F0200F04D000F0F8F804208A
S3150000628002F019FF15F0010F65D0B9F1000F06D124
S315000062900421DBF8080002F09AFA4FF001099BF896
S315000062A00700012808D1DBF8100018B1401ECBF812
S315000062B0100001D18BF807A09BF8060007284AD2E8
S315000062C0DFE800F0491C492849040B009BF8070049
S315000062D0002808BF8BF806A03DE09BF807000028C1
S315000062E039D1002C18BFB4F1010434D101208BF848
S315000062F006004C482124C0F800A02CE0002C18BF52
S31500006300B4F1010427D1012003F0F3F903208BF83F
S31500006310060020E003F0FCF9E8B1009898B90023E4
S31500006320414A42494248DFF8F0C000DF414A0023B3
S315000063304CF60101AFF27920DFF8DCC000DFCBF8C4
S315000063400C000120009002208BF8060001F0CCFE24
S3150000635034480121016015F0020F3FF447AF9BF866
S315000063600000A0B19BF80300012818BF02280ED137
S31500006370B8F1000F18BF4FF0000805D14FF0010823
S31500006380012808BF8BF800A0404602F003FA9BF8EC
S31500006390020088B19BF80500012818BF02280BD11E
S315000063A0002E18BF002604D10126012808BF8BF84D
S315000063B002A0304602F000FA9BF8010000283FF4E4
S315000063C015AF9BF80400012818BF02287FF40EAF12
S315000063D0002F18BF002704D10127012808BF8BF81A
S315000063E001A0384602F0DFF900E7000099C200007C
S315000063F0ABAAAAAA08E0FF1FA9C200006BB400005E
S31500006400B8E9FF1FD3B8000018EAFF1F15B800004F
S315000064105DBF000000E6FF1FDBBF000031B40000D7
S3150000642005B500008CE5FF1F60E6FF1F0F040100A5
S31500006430B777000060E7FF1F10B502F0A8FEFEF771
S31500006440F7FF044A0449AFF2E920DFF810C000DF85
S31500006450002010BD28E8FF1F0A90010001C10000BE
S31500006460FEE77047FEE77047704770477047704712
S31500006470F0B4441EFF4D02004FF040064FF02007D7
S31500006480FD48D0F804C002D1F0BC704712B911F82B
S31500006490013B082213F0010F14BFC5F88460C5F84C
S315000064A08860C5F888706046401EFDD1C5F88470C6
S315000064B06046401EFDD15B08521E641EE6D2F0BC4B
S315000064C070472DE9F003ED4F0122BA61E94D202610
S315000064D0C5F88860C5F88460B861C5F88860C5F8F5
S315000064E084604208BA61C5F88860C5F8846083187C
S315000064F08208BA61C5F88860C5F884601344C2088A
S31500006500BA61C5F88860C5F884601A44BA61C5F8EE
S315000065108860C5F884600022BA61C5F88860C5F84D
S3150000652084600122BA61C5F88860C5F88460914626
S315000065306A64DFF8448398F814305FEA030C05D0E8
S31500006540C5F88860C5F884605B1EF9D1C5F8886017
S31500006550D7F81C22C5F88460C5F88860D7F81C32C5
S31500006560C5F8846042EA4303C5F88860D7F81C2260
S31500006570C5F8846043EA8202012A12D0022A18BFB3
S31500006580042A66D01CF1210005D0C5F88860C5F83C
S315000065908460401EF9D10120B861BDE8F003D0B295
S315000065A0704710F0020F29D000239C462020C5F822
S315000065B08860D7F81C42C5F884605B08A44443EAA7
S315000065C0C473401EF3D1C5F88860D7F81C02C5F81D
S315000065D084608CEA000010F0010F18BF0822002921
S315000065E018BF0B6098F8140028B1C5F88860C5F884
S315000065F08460401EF9D1C5F848901CE0BCF1000F3C
S3150000660006D0C5F88860C5F88460BCF1010CF8D1E5
S31500006610C5F84890002308682021B861C5F888604D
S31500006620C5F8846003444008491EF6D1BB61C5F82D
S315000066308860C5F8846098F8080000281CBF00210F
S31500006640B961A8D0C5F88860C5F88460401EF9D144
S31500006650A1E798F81530002B1CBF10F0020F21217E
S3150000666005D0C5F88860C5F88460491EF9D1BCF12B
S31500006670000F06D0C5F88860C5F88460BCF1010C2F
S31500006680F8D1C5F84890002B85D010F0020F82D1C2
S315000066900020B8612120C5F88860C5F88460401ED6
S315000066A0F9D178E72DE9F04FDFF8D08101224FF0DC
S315000066B0000CC8F818206F4E2027C6F88870DFF83F
S315000066C0B8A1DAF8042013465B1EFDD1C6F8847023
S315000066D013465B1EFDD1C8F81800C6F8887013462D
S315000066E05B1EFDD1C6F8847013465B1EFDD10CEB14
S315000066F000044FEA500CC8F818C0C6F88870134654
S315000067005B1EFDD1C6F8847013465B1EFDD1644442
S315000067104FEA900CC8F818C0C6F8887013465B1E7E
S31500006720FDD1C6F8847013465B1EFDD164444FEA62
S31500006730D00CC8F818C0C6F8887013465B1EFDD189
S31500006740C6F8847013465B1EFDD104EB0C03C8F833
S315000067501830C6F8887013465B1EFDD1C6F88470E3
S3150000676013465B1EFDD1C8F81830C6F8887013466C
S315000067705B1EFDD1C6F8847013465B1EFDD1012356
S31500006780C8F81830C6F8887013465B1EFDD1C6F8E7
S31500006790847013465B1EFDD14FF00109C6F8449084
S315000067A09AF814405FEA040C0BD0C6F888701346BA
S315000067B05B1EFDD1C6F8847013465B1EFDD1641EB8
S315000067C0F3D1C6F8887013465B1EFDD1D8F81C328B
S315000067D0C6F884701446641EFDD1C6F88870144647
S315000067E0641EFDD1D8F81C42C6F8847015466D1E8D
S315000067F0FDD143EA4403C6F888701446641EFDD1F1
S31500006800D8F81C42C6F8847015466D1EFDD143EAC1
S315000068108403012B18D0022B18BF042B7ED01CF149
S3150000682021010BD0C6F888701046401EFDD1C6F86F
S3150000683084701046401EFDD1491EF3D10120C8F8D0
S315000068401800D8B2BDE8F08F10F0020F4AD000242D
S3150000685025464FF0200CC6F888701046401EFDD124
S31500006860D8F81C02C6F884709346BBF1010BFCD124
S31500006870054405E000F00F40E8E5FF1F0010FE4369
S31500006880640844EAC074BCF1010CE4D1BC46B346CA
S31500006890C6F88870D6461046401EFDD1D8F81C02B0
S315000068A0CBF884C0521EFDD1684010F0010F18BF0E
S315000068B00823002918BF0C609EF81410002918BF81
S315000068C0DAF804200BD0CBF888C01046401EFDD164
S315000068D0CBF884C01046401EFDD1491EF3D1CBF83B
S315000068E0489035E0BCF1000F0CD0C6F88870104611
S315000068F0401EFDD1C6F884701046401EFDD1BCF185
S31500006900010CF2D1C6F84890096800244FF0200C1B
S31500006910C8F81810C6F88870104600E02FE0401E30
S31500006920FBD1C6F884701046401EFDD10C444908C0
S31500006930BCF1010CECD1C8F818403946B446C6F88B
S3150000694088701046401EFDD1CCF88410521EFDD131
S315000069509AF8081000293FF471AF0020C8F8180013
S31500006960DAF80420C6F888701046401EFDD1C6F835
S3150000697084701046401EFDD1491EF3D15EE79AF899
S315000069801550002D1CBF10F0020F21240BD0C6F8A5
S3150000699088701146491EFDD1C6F884701146491EFD
S315000069A0FDD1641EF3D1BCF1000F0CD0C6F888707F
S315000069B01146491EFDD1C6F884701146491EFDD107
S315000069C0BCF1010CF2D1C6F84890002D3FF436AF69
S315000069D010F0020F7FF432AF0020C8F81800212112
S315000069E0C6F888701046401EFDD1C6F88470104661
S315000069F0401EFDD1491EF3D120E7024A527802B16A
S31500006A005FE54FE6E8E5FF1F10B5FFF716F9FF480B
S31500006A102021C1674021C167012101641021016065
S31500006A200221C163C26842F01002C260026842F0ED
S31500006A3010020260026C42F001020264C163C16C82
S31500006A4041F00201C164F24940F21310486001208E
S31500006A5010BD38B50C4600F00C0040F00200694647
S31500006A6000F049FC9DF80020DDF80130012842EADB
S31500006A700322226018BF002038BD082806D1E54A47
S31500006A8013688B4212BF11600120704738B500F0C1
S31500006A900C040422684600F01FFC6946204600F0FC
S31500006AA02AFC012818BF002038BD00F07F4238B507
S31500006AB004460D4600F0F00042EA00010820FFF708
S31500006AC0DCFF002808BF38BD04F00C0040F00304CA
S31500006AD06946204600F00FFC6946204600F00BFC94
S31500006AE09DF80010DDF80120012841EA0221296005
S31500006AF018BF002038BD38B50D46044600F07F416A
S31500006B0000F0F00001430820FFF7B7FF002808BF98
S31500006B1038BD7CB104F00C0040F001040422294683
S31500006B20684600F0D9FB6946204600F0E4FB0128E0
S31500006B300FD107E0B7484168A94214BF456001205C
S31500006B40E8D138BD0E20002100F0D5FB012808BF92
S31500006B5038BD002038BD30B50C46054683B0AE4979
S31500006B600020FFF7C8FF002804BF03B030BD042291
S31500006B70294601A800F0B0FB052001A900F0BBFBE7
S31500006B80012818D10F20694600F0B5FB012812D163
S31500006B900E20694600F0AFFB9DF80010DDF80120DD
S31500006BA0012841EA0221216018BF002000281EBFEB
S31500006BB0012003B030BD002003B030BD38B50C460F
S31500006BC0054695490020FFF796FF002808BF38BD07
S31500006BD004222946684600F07FFB0520694600F03E
S31500006BE08AFB012815D104222146684600F074FB71
S31500006BF00D20694600F07FFB01280AD10E200021F6
S31500006C0000F079FB012818BF002000281CBF0120D6
S31500006C1038BD002038BD2DE9F04F83B015460F462C
S31500006C2006462EE07D490020FFF765FF002800F0AC
S31500006C30B7803146042201A800F04EFB052001A9C9
S31500006C4000F059FB01287DD10F20694600F053FB67
S31500006C50012877D10E20694600F04DFB9DF8001003
S31500006C60DDF80120012841EA022118BF0020002892
S31500006C7068D0B007C00E21FA00F0761C07F8010BA9
S31500006C806D1E002D7ED016F0030FCBD1032D4ED9ED
S31500006C90C6F30B00C0F58058454538BF25F00308FC
S31500006CA0B946B8F1000F7BD04FEA980B5A4900203D
S31500006CB0FFF721FF002873D005240422314601A8DE
S31500006CC000F00AFB01A9204600F015FB012867D158
S31500006CD00F204946009000F00EFB012860D14FF0CE
S31500006CE0000ABBF1000F14D900980024029049460F
S31500006CF00298FFF782FE022803D1611CCCB2642CF5
S31500006D00F5D301284CD10AF1010A09F10409DA4543
S31500006D10EAD30E20002100F0EEFA012818BF002069
S31500006D2080B14644A5EB08054744032DB0D8002D95
S31500006D3018BF3A4C30D021460020FFF7DCFE08B1E0
S31500006D40314600E02CE0042201A800F0C5FA052037
S31500006D5001A900F0D0FA012822D10F20694600F0DF
S31500006D60CAFA01281CD10E20694600F0C4FA9DF823
S31500006D700010DDF80120012841EA022118BF002099
S31500006D8070B100E008E0B007C00E21FA00F0761CF2
S31500006D9007F8010B6D1ECED103B00120BDE8F08FC0
S31500006DA003B00020BDE8F08F2DE9F84315460E46E6
S31500006DB00446DFF8688036E0377841460020FFF762
S31500006DC09AFE002874D0A007C00E874021460422F0
S31500006DD0684600F081FA0520694600F08CFA012821
S31500006DE066D104223946684600F076FA0D206946D7
S31500006DF000F081FA01285BD10E20002100F07BFA19
S31500006E00012818BF0020002852D009E008F00F40E2
S31500006E1000A0044020E0FF1F520000235000002382
S31500006E20641C761C6D1E002D18BF14F0030FC3D111
S31500006E3025F003094A463146204600F06CFA002840
S31500006E4008BFBDE8F88304EB09074E44B5EB090417
S31500006E502AD0357841460020FFF74DFE38B3B807F3
S31500006E60C00E854039460422684600F035FA0520F2
S31500006E70694600F040FA01281AD1042229466846DC
S31500006E8000F02AFA0D20694600F035FA01280FD1E4
S31500006E900E20002100F02FFA012818BF002030B183
S31500006EA07F1C761C641ED4D10120BDE8F883FFE761
S31500006EB00020BDE8F88373B5064600246425FA4829
S31500006EC00199FFF77BFE002804BF02B070BD46F4AF
S31500006ED08031F648FFF772FE002812BFF44E02B06A
S31500006EE070BD01A93046FFF736FE002804BF02B088
S31500006EF070BD019810F4803F02D002B0012070BD31
S31500006F00641CAC42EDDB02B0002070BD38B50D4606
S31500006F1004466946E648FFF71EFE002808BF38BD4E
S31500006F20009810F4003008BF38BD2146002000F05C
S31500006F3030FA002808BF38BD2946012000F029FA9A
S31500006F40002818BF012038BD014608B50020FFF70C
S31500006F50B2FF002808BF08BD69460F2000F019FAE5
S31500006F60002808BF08BD0098811C0F20FFF7A3FF6B
S31500006F70002808BF08BDCF49CD48FFF71FFE0028EF
S31500006F8018BF012008BD2DE9F04393B08946DDE91D
S31500006F901A7804461E4615464421684605F011FA3D
S31500006FA08DE8E00160680990A0680D902068CDE941
S31500006FB00E094FF0807010906D4600210820FFF7F3
S31500006FC05CFD002818BF00245AD055F8241020462E
S31500006FD0FFF771FF002853D0641C042CF5D3092059
S31500006FE0696AFFF768FF002818BF0D2448D055F8D6
S31500006FF024102046FFF75FFF002841D0641C102CA8
S31500007000F5D31020296CFFF756FF002838D04FF42F
S315000070109362A9494FF0005000F07DF980B3A44E69
S31500007020A4493046FFF7CAFD50B3062011A900F067
S3150000703062F99DF84410DDF84520012841EA022155
S3150000704002BF11F0A00F42F21075002418D111A949
S315000070503046FFF780FD98B1119810F4003F13D029
S315000070606946002000F095F9002804BF13B0BDE87A
S31500007070F0830098002802BF012013B0BDE8F0831A
S31500007080002013B0BDE8F083641CAC42DFD3F7E701
S3150000709038B58A484FF0FF3101604160FFF7B4FC14
S315000070A002F006F800F0A0F9002808BF38BD1E213E
S315000070B00020FFF7E2FC002808BF38BD00210820A9
S315000070C0FFF7DBFC002808BF38BD4FF0A0410420C5
S315000070D0FFF7D3FC002814BF4FF0204438BD06202C
S315000070E0694600F008F99DF80010DDF80120012836
S315000070F041EA022101D0002038BD34EA0100EED178
S315000071006F490420FFF7B9FC002808BF38BD01F01D
S31500007110D4FF00210820FFF7B0FC002818BF01208B
S3150000712038BD0028674914BF002001200860704759
S31500007130F8B50446FFF768FC5E4E5D4D062C7DD221
S31500007140DFE804F0033F0716848C0120FFF7E9FF10
S31500007150A8E00120FFF7E5FF0220DFF86CC100DFA1
S315000071600020FFF7DEFF0220DFF85CC100DF99E0B8
S315000071700120FFF7D6FF0120DFF84CC100DF002019
S31500007180FFF7CFFF0120DFF840C100DFFFF780FFE8
S31500007190002808BFF8BD31462846FFF70FFD002836
S315000071A008BFF8BD0120FFF7BCFF0120DFF818C1BA
S315000071B000DF0020FFF7B5FF0120DFF80CC100DF7C
S315000071C070E00120FFF7ADFF0220DFF8FCC000DF12
S315000071D00020FFF7A6FF0220DFF8ECC000DFFFF774
S315000071E057FF002808BFF8BD31462846FFF7E6FCE2
S315000071F0002808BFF8BD0121344C2046FFF7DEFC0D
S31500007200002808BFF8BD0120FFF78BFF0220DFF83A
S31500007210B8C000DF0020FFF784FF0220DFF8A8C017
S3150000722000DF69462846FFF796FC002808BFF8BD30
S31500007230009810F4003FF4D0002100E04AE0204618
S31500007240FFF7BCFC002808BFF8BD2BE02049284604
S31500007250FFF7B4FC002808BFF8BD23E0FFF7D4FB16
S3150000726000F0C2F8002808BFF8BD1E210020FFF775
S3150000727004FC002808BFF8BD00210820FFF7FDFB2D
S31500007280002808BFF8BD4FF0A0410420FFF7F5FB2A
S31500007290002808BFF8BD31462846FFF78FFC0028B6
S315000072A008BFF8BD0120F8BDF8ED00E0F4ED00E000
S315000072B0F0ED00E001005FA080C5000020E0FF1FA8
S315000072C0000F00500408FE4393C20000FCED00E0EE
S315000072D000005FA00020E6E70023002A98BF704761
S315000072E04FEAC30C21FA0CFC00F803C05B1CDBB2AE
S315000072F09A42F5D8704770B50D46064600242946D1
S315000073003046FFF77AFB022818BF70BD611CCCB26D
S31500007310642CF4D370BD002A04BF002070472DE909
S31500007320F8430E46054697084B490020FFF7E3FB56
S31500007330002808BFBDE8F8830524042229466846CC
S31500007340FFF7CAFF69462046FFF7D5FF01281DD182
S3150000735000254FF00D08002F10D900243146404675
S31500007360FFF74BFB022803D1611CCCB2642CF5D38A
S3150000737001280BD1361D6D1CBD42EED30E20002117
S31500007380FFF7B9FF012808BFBDE8F8830020BDE874
S31500007390F8832DE9F0410E460146002464252F4866
S315000073A0FFF70CFC002814BF2D4FBDE8F0813146D5
S315000073B03846FFF7D0FB002808BFBDE8F0813068EB
S315000073C010F4803F02D1641CAC42F0DBAC4204BF37
S315000073D00020BDE8F08131462248FFF7BCFB0028BB
S315000073E018BF0120BDE8F081002010B584B06946C1
S315000073F0FF240C54401CC0B20828FAD33320FFF7F0
S3150000740037F89E208DF80000E7208DF801006946C8
S315000074101020FFF72DF8002069460C54401CC0B21E
S315000074200828FAD33320FFF723F800208DF804004C
S3150000743001A90820FFF71CF802206946FFF75BFF49
S315000074409DF80010DDF80120012841EA0221029191
S3150000745018BF002004B010BD52000023F4ED00E078
S31500007460F0ED00E0F8ED00E00020704700207047E6
S3150000747000207047002070470020704700207047AA
S31500007480002070470020704700207047002070479A
S315000074904FF6FF7100220846DFF804C100DFDFF86F
S315000074A004C100DF044610F0040F18BF01F09AFF74
S315000074B014F0400FECD002F0CEFF01F0E5FFE7E755
S315000074C04FF6FF7100220846DFF8D4C000DFDFF870
S315000074D0D4C000DF10F0010F18BF02F09EFFEFE7E7
S315000074E000291CBFDFF8C0C000DF7047DFF8B4C05A
S315000074F000DF70470022DFF8A8C000DF704710B534
S3150000750000F0B0F800F07AF9BDE8104001F070BE66
S315000075102DE9F00F254CDFF8988000262660D8F874
S31500007520000038B100231A4603212248DFF888C03C
S3150000753000DF2060DFF88490214D224FDFF888A01D
S31500007540002400BF45F8246057F8240080B1484560
S315000075504FF0000305D000220221DFF85CC000DFF7
S3150000756004E01A4A5146DFF850C000DF45F824000F
S31500007570641C0F2CE6D9164C2660D8F804000028A7
S3150000758004BFBDE8F00F704700231A4602211148D8
S31500007590DFF824C000DF2060BDE8F00F7047000070
S315000075A031B4000005B500006BB4000060E5FF1FB4
S315000075B054CA000091740000DBBF000025B3000030
S315000075C0A01B00205CCA00000258020090080020A0
S315000075D04CE5FF1FC174000000F0F8BC00F0FEBCD3
S315000075E000F004BD1C4902680A6082790A7142797A
S315000075F04A71007988710020C871084600F0FEBC07
S3150000760010B50446144800F006FD002808BF10BD5A
S315000076101148016821600179A17141796171807910
S315000076202071012010BD10B50C4CDFF834C030B10C
S3150000763000DF2060002001F03EFD012010BD00DFCC
S315000076402168401AB0F5967F2CBF01200020FEF776
S31500007650F2FCF2E70120704744E0FF1F40E0FF1F05
S315000076608DC200005D4800210170416081600122E9
S3150000767042708170C1600161704710B5944601285F
S3150000768002D10BB1012B01D0002010BD534C206953
S31500007690E168884201BFA078002801206070F3D01D
S315000076A04F482169402200EB8111604604F070FECC
S315000076B02069401C206121690020052908BF20613E
S315000076C02169E268914208BFA070402010BD0228DF
S315000076D018BF7047002B08BF704770B5107801259A
S315000076E01146072802BF3F48057070BD3B4C207805
S315000076F020B16068A268904208BF70BD3A486268CF
S3150000770000EB82101A4604F043FE6068401C60607D
S315000077106068052804BF002060606068A168884230
S3150000772008BF25700120DFF8C4C0616900DF70BDA5
S315000077302DE9F0472A4E0025284CA6F5A077DFF85C
S31500007740B0804FF0010920E0E06806EB8011A068E8
S3150000775007EB8010FEF704F8A068401CA8FB002188
S315000077608908494201EB81010844A060A06861686C
S31500007770884208BF2570607880B16570E068402255
S3150000778006EB8011002002F05FFFA0686168884266
S3150000779004BF20780028D7D1BDE8F087E068401CF8
S315000077A0052808BF0020E060E0682169884208BF1C
S315000077B084F80290E9E7DFF83CC000DF074948613A
S315000077C000224FF6FF710120DFF82CC000DFFFF723
S315000077D0AFFF0020FEF736FCF2E700004CE0FF1F8B
S315000077E0280C002004E0FF1FE80A00206BB400000C
S315000077F0CDCCCCCC5DBF000031B4000010B500F09C
S315000078004AFCD249D24AD44BB1F80B00B1F8131056
S3150000781041431160CF4A1060B1FBF0F0CF4901221D
S315000078201A600860CF49CE480860CF48026010BD94
S315000078302DE9F74F8346C74800269246006835462D
S315000078400BFB00F8C8483746344600684FF001097C
S31500007850002804BF03B0BDE8F08F0020FEF704FC4B
S31500007860C2490DE00544A84508D2A5EB080251F827
S315000078703460871A042F28BF4FF00009601CC4B279
S3150000788001EBC400406810B1002EEBD000E016B149
S31500007890B9F1010F23D0AF4800680AFB00F1019847
S315000078A004F08FFDA948B0F81110B0F80B2049017B
S315000078B0B1FBF2F1C289C38A007C03FB00200844B5
S315000078C058451CBF03B0BDE8F08FA24800680AFB0C
S315000078D000F1019803B0BDE8F04F00F0E2BA9D4810
S315000078E0F11900680AFB00F2019804F051FDD9E78E
S315000078F02DE9F04F0646002095B007460490059006
S3150000790006900790089009900A9005460B909648B5
S31500007910934689460068002804BF15B0BDE8F08F7D
S31500007920DFF84CA2DAF8140038B192A28E2197A0A3
S3150000793000F009F915B0BDE8F08F314696A000F0C9
S3150000794002F90020FEF790FBDAF81000002848D074
S315000079507E48017CC08A4843411CB1421CBF801C42
S31500007960B04240F09A807B480168B5EB511F38BFA2
S31500007970DFF8308280F0918009EB4511202204A8BF
S3150000798004F006FDBDF82A00BDF82230BDF8262019
S315000079909DF81D108DE80F009DF81B2004A982A0FC
S315000079A00B9B00F0D0F804AC0DF1400C0FCC0CACE6
S315000079B00FC408AC0FCCACE80F00D8F800000024C8
S315000079C0002863D09DF8302086A00178914255D1D9
S315000079D058F8240003220EA904F005FD002850D112
S315000079E064E0484600F09EFB012808BF012406D04B
S315000079F0484600F0B2FB01280CBF02240024002CEC
S31500007A004BD082A185A000F09EF84FF0FF30514D7B
S31500007A10CAE900602868CAE902060120CAF810000F
S31500007A208AF81840204600F0BAFB07000DD0002067
S31500007A30CAF810000120CAF81400384600F0F8FA17
S31500007A40FEF728FB15B0BDE8F08F75A2AD2178A032
S31500007A5000F079F82868DAF8001000FB0BF2711ACA
S31500007A604843494600F02BFC0746014672A000F049
S31500007A706AF8002F18BF0F2FD9D14AE0401C002901
S31500007A80A3D1641C58F8240000289BD131486D1CF2
S31500007A900068B5EB501FFFF46FAFDAF80000B04294
S31500007AA09CBFDAF81000012833D109E013980028AA
S31500007AB018BF0120012804BF0B98CAF80400E5E7A7
S31500007AC0DAF80C00401CB04204D05DA153A000F0CF
S31500007AD03AF81EE052A2D12155A000F034F81D4C10
S31500007AE0DAF800102068711A00FB0BF24843494689
S31500007AF000F0E5FB074601464FA000F024F8002FF2
S31500007B0018BF0F2F93D1DAF8080021680844CAE994
S31500007B100206DAE90101814224BFDAF810000128E1
S31500007B201EBF0F2F15B0BDE8F08F4BA13BA000F094
S31500007B300AF80020CAF8100000F07AFAFEF7A3FA55
S31500007B4015B0BDE8F08F0120704700007CE0FF1FF4
S31500007B50BCE5FF1F98E5FF1F9CE5FF1FA0E5FF1F83
S31500007B60680D0020A4E5FF1F8CE5FF1F7CE4FF1FC6
S31500007B70481000205472616E736665725F666169B3
S31500007B806C6564202D2065786974000025643A20B0
S31500007B9025730D0A00000000626C6F636B3A2025A6
S31500007BA0640D0A00ECCB00006E613A252E3131736C
S31500007BB009617472623A25386409737A3A25386421
S31500007BC00973743A2538640963723A253864096D75
S31500007BD06F643A25386409616363643A2538640D35
S31500007BE00A000000303132333435363738394142F5
S31500007BF0434445464748494A4B4C4D4E4F505152D7
S31500007C00535455565758595A00000000464C415394
S31500007C104820494E49540D0A000000002573000013
S31500007C20464C415348205752495445202D200000C8
S31500007C3025643A202573000025640D0A0000000023
S31500007C40424C4F434B204F5554204F46204F5244F1
S31500007C5045520D0A00000000464C41534820454E4F
S31500007C60440D0A002DE9F00300210A460B46DFF811
S31500007C7034C31825CC4C01E0042916D250F82360F1
S31500007C804F4205EBC707FE40F6B202EB410704EB95
S31500007C901619674499F8009006F00F0687F80090C9
S31500007CA0A65D491C7E700429E8D300215B1C0832BE
S31500007CB0202AE1D300208CF82000BDE8F0037047AD
S31500007CC0F0B40021B94CB84D08264B42426806EB89
S31500007CD0C303DA40D2B204EB410305EB121702F0FC
S31500007CE00F023F781F70AA5C491C5A700229ECD318
S31500007CF0062938BF182613D2C1F10203026806EB23
S31500007D00C303DA40D2B204EB410305EB121702F0CB
S31500007D100F023F781F70AA5C491C5A700629EBD3E4
S31500007D200020E073F0BC7047A148704710B5A14829
S31500007D3004F052FB022101EB4000C0B210BD9E4888
S31500007D4070472DE9F05F9D4800F06AFD102204217E
S31500007D509B4800F000F99B4C054610220421606800
S31500007D6000F0F9F8954E45EA0040954F316810222B
S31500007D704840E0600821381D00F0EDF8E16806F1A2
S31500007D80100581EA000E2421C4F80CE02970697000
S31500007D90A97018210020E97004213A5C6A54491C34
S31500007DA0401CC0B2C9B20428F7D362680020135C35
S31500007DB06B54491C401CC0B2C9B20428F7D3DFF883
S31500007DC0E8810023C3F1030201EB430A00204FEAD6
S31500007DD0C20B0AEB050956F820200AEBC00C22FA62
S31500007DE00BF20CEB0504D2B208EB121709EBC00C30
S31500007DF03F7802F00F022770401C18F80220C0B22C
S31500007E008CF801200428E6D3581CC3B2042BD9D31E
S31500007E1001F1200000F0FF0C0020C0F10301C900B1
S31500007E202EFA01F10CEB4002C9B208EB11142A44F8
S31500007E30247801F00F011470401C18F80110C0B22C
S31500007E4051700428E9D30CF10800C0B200262E5464
S31500007E503446281D04F0C0FA574AC0B2022101EB8D
S31500007E6040011170032151700221B6EB400F0AD276
S31500007E7014F0010F1CBF0B19D6540AD0631CDCB2D8
S31500007E80B4EB400FF4D301EB4000C0B21654BDE88A
S31500007E90F09F05EB540301EB040C1B7902F80C3040
S31500007EA0ECE72DE9F047474D07460024287882B0D5
S31500007EB08A46012610B9FFF744FF2E70424800900B
S31500007EC03C484FF0000C8DF804C0A0F14808A0F122
S31500007ED038099DF8042032B1AA681278002A08BF32
S31500007EE08DF804C025D1009A531C00931378402BBB
S31500007EF023D1009A1278412A04BFA8608DF8046045
S31500007F000DD04D2A04BF8DF80460C5F8088006D050
S31500007F10552A04BF8DF80460C5F808900DD1009A63
S31500007F20521C0092AA681278002A08BF8DF804C075
S31500007F30CFD0A96811F8013BA960002B1CBF3B55A7
S31500007F40641CC6D1AAEB04013819202204F032FAC7
S31500007F5002B0BDE8F08770B400252C462B460029F8
S31500007F601DD990F800C0ACF13006092E98BF302319
S31500007F700AD9ACF14106052E98BF372304D9ACF1D6
S31500007F806106052E98BF572305FB02CCACEB030513
S31500007F9004F1010C401C0CF0FF048C42E1D328468E
S31500007FA070BC7047780F002000CC0000680F0020DE
S31500007FB0AC0F0020B00F0020E10F00209C0F002026
S31500007FC078DF000064E0FF1FACD0000000221146FD
S31500007FD01448DFF854C000DF012070470022012159
S31500007FE01048DFF844C000DF01207047002202215C
S31500007FF00C48DFF834C000DF012070470B49D0E998
S315000080000020C1E90020002203210648DFF818C03D
S3150000801000DF012070470549D1E90021C0E90021B0
S3150000802001207047B8E9FF1F2FB8000074E0FF1F5A
S3150000803070B5364A364904001CD001F50F7002F5BA
S31500008040187690E82910A6E82910D1E99303D1E91A
S3150000805095C1C2E99C03C2E99EC12D4D55F8240085
S3150000806004F0BAF92B49C86701F5007155F82400E8
S31500008070886470BD01F5177002F5187690E829102E
S31500008080A6E82910D1E99B03D1E99DC1C2E99C0369
S31500008090C2E99EC1E1E710B51F481C4C406AB4F81E
S315000080A00B1000F58030B0FBF1F080B2A4F813009D
S315000080B0617BB0FBF1F000F2FF30800A00EB40007C
S315000080C0E082164804F088F904F50071C865E08A74
S315000080D001F500714002C8604861607B4002A0F56E
S315000080E000704863486410BD094910B401F51F7259
S315000080F00B4892E81C1080E81C10D1E9A323D1F8A4
S3150000810094120261C0E9053110BC70477CE0FF1F84
S3150000811014CC00007CE2FF1F78DF000050CC00008A
S315000081204810002010B4CF4C02680421D4E907C3DC
S31500008130624528BF93420DD34218D4E9053C126824
S315000081409A4228BF944505D3091D0C29F4D910BCC1
S315000081500120704710BC0020704701783A2901D0F1
S3150000816000207047007A302818BF322804D0332800
S315000081701CBF34283528F3D10120704700B50020F4
S3150000818083B00346009002460190B749B748FEF710
S31500008190FAFE00280CBF0820002003B000BDF0B591
S315000081A0044683B0012000F086FF002802BF0120AC
S315000081B003B0F0BD4FF49362AD494FF00050FEF7A7
S315000081C0F3FD002802BF022003B0F0BD0025A5483C
S315000081D000950195A84F42692B46A64907F1140060
S315000081E0FEF7D1FE002802BF042003B0F0BDA34E67
S315000081F0022C347006D100F04BF9E101A04804F0DE
S31500008200E0F87560002300951A46974907F11400B7
S315000082100195FEF7B8FE00280CBF0820002003B029
S31500008220F0BD002070472DE9F0416FF3080082B0E1
S3150000823014460F46054600F0ABFF012802BF052095
S3150000824002B0BDE8F08122468C4E3946706800F1D6
S31500008250005000F54050FEF7A7FD60B3706820445B
S3150000826070607068B0F5007F21D30020DFF81482BB
S31500008270CDE900807B484FF4007383494069421979
S315000082807A48FEF780FE002802BF092002B0BDE84A
S31500008290F0817068A0F500707060706838B1706821
S315000082A07268201AC1194046FEF77EFD18B102B069
S315000082B00020BDE8F08102B00320BDE8F0812DE981
S315000082C0F04F6E4E002787B033780546022B36D026
S315000082D0012B1EBF0B2007B0BDE8F08F8846144661
S315000082E0B2F5007F27D35F48664EDFF89CA1406950
S315000082F0DFF8849100EB050B22464146284600F044
S3150000830047FF01287AD0224641463046FEF74CFD0B
S31500008310002874D05A464FF40073514609F11400F0
S31500008320CDE90067FEF72FFE002869D0A4F500749A
S31500008330B4F5007FE0D207B00020BDE8F08F0D460F
S315000083401446039704970DF110080DF10C094FF42C
S31500008350807A0597CDF800A0CDE90198484B05AA8B
S315000083602146284600F0A5F868B1022825D0012844
S3150000837047D0042866D0052818BF0628EAD107B0DA
S315000083800D20BDE8F08F0498002802BF384607B0DC
S31500008390BDE8F08F03987268C0F30801914204D9D2
S315000083A072688A1A3949FFF73EFFDDE9030234494C
S315000083B0FFF739FF07B0BDE8F08F049878B103984E
S315000083C07268C0F30801914204D972688A1A2F496B
S315000083D0FFF729FFDDE903022949FFF724FF70684B
S315000083E040B17068C0F50072DDE903010844274911
S315000083F0FFF719FF0598241A0544ABE726E029E0A4
S315000084002CE0049878B103987268C0F30801914291
S3150000841004D972688A1A1D49FFF705FFDDE90302D0
S315000084201749FFF700FF706840B17068C0F5007229
S31500008430DDE9030108441549FFF7F5FE07B00F20F3
S31500008440BDE8F08F07B00C20BDE8F08F07B005201F
S31500008450BDE8F08F07B00320BDE8F08F07B0092014
S31500008460BDE8F08F78DF00005900002058DD0000DD
S31500008470ACD800002100002044DD0000D4E4FF1F3A
S315000084806410002000300020AB00002078DD0000E2
S3150000849010B52521894803F094FF2521884803F06B
S315000084A090FF884800214160017041708170C17061
S315000084B010BD2DE9FF4F81B0DFF808A2109D894657
S315000084C04FF00008044600EB0907C5F800809AF84B
S315000084D00300DFF8E8B11E46D0B18AF803809BF8A6
S315000084E000200BF10401184603F052FF9BF8000030
S315000084F02968064408442860DAF80400BBF801102D
S315000085006FF30F0008439BF800100844CAF80400F4
S31500008510BC4279D020780A2818BF0D2819D03A28ED
S3150000852073D09AF80010002970D010F0100F00F0E8
S315000085300F0008BF093000F00F019AF801001BF880
S31500008540002011430BF80010401C8AF8010000209F
S3150000855096E05A4A002108461378009303F1050C69
S31500008560BCF1000F88BF5B1D0BD912F800C0401C80
S315000085706144C0B2C9B28342F7D811B14FF00408C2
S3150000858086E09AF8020000287CD101208AF80200D1
S31500008590BBF8010090FA90F8ABF801809BF8030055
S315000085A020B1012833D0042834D06BE0434925227A
S315000085B001F1250003F0ECFEDAF8040001466FF342
S315000085C00F0141EA0801814205D001208AF8030023
S315000085D04FF002085CE00BF104013046009A03F00C
S315000085E0D7FE9BF800002968064408442860DAF89C
S315000085F00400BBF801106FF30F0008439BF800104E
S315000086000844CAF804003DE040E01FE02AE04FF0CD
S3150000861001083DE029680E98FF22411A304603F012
S31500008620C9FE2868DAF80410091A0F980160381B89
S31500008630A9EB000103980160BBF8040040BA0004EE
S31500008640CAF8040005B00220BDE8F08F25211B48BA
S3150000865003F0B7FE00208AF800008AF801008AF8C5
S3150000866002000FE09AF80110252908D210F0100F29
S3150000867000F00F0008BF093000010BF801000120CF
S315000086808AF80000641CBC427FF444AF4FF0000837
S3150000869029680E98FF22411A304603F08BFE28689F
S315000086A0DAF80410091A0F980160381BA9EB0001CB
S315000086B00398016005B04046BDE8F08F64110020C4
S315000086C089110020DCE4FF1F2DE9F00700220127B5
S315000086D016460029C4BF48F205084FF6FF7928DD83
S315000086E0082510F806C0002423461CF0010F07D009
S315000086F0A5EB030AAAF1010A07FA0AFA4AEA0404F0
S315000087005B1CDBB24FEA5C0CAB42EED3E3B282EA0F
S315000087100322082312F4004F1ABF88EA420292B2DB
S3150000872009EA42025B1E13F0FF03F3D1761C8E4268
S31500008730D6DB10230021084612F0010F07D0A3EB69
S31500008740000CACF1010C07FA0CFC4CEA0101401CD0
S315000087505208C0B29842EFD3BDE8F00788B270471E
S315000087602848816B41F4A0518163274982150A612B
S315000087702648102303604361836843F01003836037
S315000087808A61016841F040010160416941F04001A0
S315000087904161704710221E49002814BFC1F8C82045
S315000087A0C1F8C420704710210028194A14BFC2F826
S315000087B0C810C2F8C410704710210028144A14BF0C
S315000087C0C2F8C810C2F8C41070470020704711489C
S315000087D0416841F0807141600F49416041150F4881
S315000087E0C0F8FC11C16770470A48D0F8A0100229EA
S315000087F018BF7047416841F08071416040F2131123
S31500008800416070470080044000C00440C0F00F4043
S3150000881000F00F4000A0044013010A0088E000E0C9
S3150000882004490A6ECB6D5A408B6D496D59405140D3
S31500008830016070470080044070B5BF4D4FF480243E
S315000088402C6000F057F9BD48816B41F400618163EB
S31500008850416B41F4006141632C60B948C17841F035
S315000088600C01C170B7494FF44072CA600A61C17801
S3150000887041F02001C170C5F8004145F8804C012047
S3150000888070BDAF4810B5C17821F00C01C170C17838
S3150000889021F0A001C17000F02DF9012010BD70B5C6
S315000088A0A54C4FF480250026256000F023F9A44846
S315000088B0C17821F08001C170A348066044F8805C4D
S315000088C0012070BD2DE9F0474FF0E02800244FF459
S315000088D0802905462746C8F88091994EF07820F001
S315000088E00C00F07000F006F968790021012804BF39
S315000088F00124274603D0022808BF012400D1012104
S31500008900080140EA44003843B07090492868096875
S315000089100001B1FBF0F03178C0F3042221F01F0111
S315000089201143317071787070F07840F00C00F0707F
S31500008930C8F88092C8F800910120BDE8F0870120B0
S3150000894070478348D0F80812D0F80C02081AC0F510
S3150000895000707047002904BF0020704730B4491EDC
S315000089607B4A4FF0000C89B2D2F80832D2F80C429A
S315000089701B1B1BB2B3F5007F15DA10F8014BD2F8BA
S315000089800032D5185B1CC2F800322C70D2F80032C7
S31500008990C3F30803C2F80032D2F808325B1CC2F8EF
S315000089A008320CF1010C0B00A1F1010189B2DBD1F7
S315000089B0654B1868002808BF61481CD1017911F081
S315000089C0800FFBD001211960D2F804125318491CFC
S315000089D0C2F804121978C171D2F80412C1F3080161
S315000089E0C2F80412D2F80C12491CC2F80C12C17853
S315000089F041F08001C17030BC60467047002904BF59
S31500008A000020704710B4491E524A4FF0000C89B23C
S31500008A10D2F80832D2F80C42A3421AD0D2F8043265
S31500008A20D4185B1CC2F80432237800F8013BD2F854
S31500008A300432C3F30803C2F80432D2F80C325B1CCA
S31500008A40C2F80C320B00A1F101010CF1010C89B244
S31500008A50DED110BC6046704718B4394B18793C49D2
S31500008A60D1F80822D1F80C42DFF8DCC0A2423BD094
S31500008A7010F0800F15D0D1F804228C18521CC1F8C2
S31500008A8004222278DA71D1F80422C2F30802C1F86E
S31500008A900422D1F80C22521CC1F80C220121CCF878
S31500008AA0001010F0200F04BF18BC704710F0060F1E
S31500008AB01FBFD8798DF8000018BC7047DA792548B1
S31500008AC0D0F800124318491CC0F800121A70D0F8EA
S31500008AD00012C1F30801C0F80012D0F80812491CB0
S31500008AE0C0F8081218BC7047D97821F08001D970F7
S31500008AF00021D4E710B5BB224FF40071154803F0EE
S31500008B0059FC14480024C0F80042C0F80442C0F8DA
S31500008B100842C0F80C42BB224FF40071A0F5047065
S31500008B2003F048FC0A48C0F80042C0F80442C0F806
S31500008B300842C0F80C4210BD80E100E0008004400D
S31500008B4000B0064000B00440E4E4FF1F00E0FF1F51
S31500008B50B0110020C0130020FE49082008607047AD
S31500008B60FD4908200870FD48416841F4A021416094
S31500008B70816C21F00F01816400218164416B41F415
S31500008B808021416301DFF64890F80C1141F0800125
S31500008B9080F80C1190F80C1111F0800FFAD1F14900
S31500008BA0090A80F89C10EF49090C80F8B010ED49CD
S31500008BB0090E80F8B410FF2180F88010EA49096890
S31500008BC0002919BF0421022200210A46114341F05F
S31500008BD0190180F88410402180F8001190F80C11DA
S31500008BE041F0400180F80C117047DD49002891F8EA
S31500008BF0940014BF40F0010020F0010081F89400B9
S31500008C0012BF102091F8080120F0100081F8080129
S31500008C1070470120D249002201EB800383F8C0206F
S31500008C20401C1028F8D3CF480823438000F1A00346
S31500008C304360C8230370027200F590734361C261FA
S31500008C400D2081F8C000C94B4FF05530186091F8DF
S31500008C50940040F0020081F89400FF2081F8800023
S31500008C6081F8880081F88C0081F898207047C04808
S31500008C70017841F0200101707047BD48017821F06C
S31500008C80200101707047BB48007810F0020F08BF42
S31500008C907047B34A92F8940040F0040082F89400BA
S31500008CA04CF24F3000BF401EFCD292F8940020F0E8
S31500008CB0040082F8940070477047002918BF704777
S31500008CC000F07F00AC4908707047704770B4AB4C39
S31500008CD010F0800F4FF0000CA4F1A0054FF0010238
S31500008CE018D000F00F06A14802EB460102FA01F186
S31500008CF050E8002F0A4340E80023002BF8D104EB8C
S31500008D00062000F1800105EB4610C0F81CC0416149
S31500008D1070BC7047430095499A40D24351E8003FE2
S31500008D2003EA020641E80063002BF7D18A490A5C90
S31500008D3000F00F0105EB411004EB01214280416078
S31500008D408821017080F808C070BC704701468078A1
S31500008D50898810F0800F04BF7F4A1154B6E7704728
S31500008D607F4910F0800F18BF00F00F0001EB800064
S31500008D7090F8C01014BF41F0050141F0090180F8D8
S31500008D80C0107047764910F0800F18BF00F00F0032
S31500008D9001EB800090F8C01014BF21F0050121F00E
S31500008DA0090180F8C01070476D4900F00F0001EB13
S31500008DB0800090F8C01041F0020180F8C0107047A2
S31500008DC0674900F00F0201EB820191F8C02022F002
S31500008DD0020281F8C02079E770472DE9F00105000D
S31500008DE04FEA00705F4C4FEA906304EBC3074FF005
S31500008DF00006788806D114F83320C2F383020D2AC0
S31500008E0008BF01260022002884BFDFF870C10CEBE2
S31500008E10831C06D91CF8028001F80280521C90427D
S31500008E20F8D84D4A4FEA530C525D504D7A8014F8EB
S31500008E3033702A68C7F3801722FA0CF202F0010297
S31500008E40BA4213D136B18979002904BF47496FF078
S31500008E5001021DD04549012202FA0CF251E8006FC9
S31500008E6086EA020741E80076002EF7D1296821FA42
S31500008E700CF111F0010F14BFC821882104F833103A
S31500008E803F490A7822F020020A70BDE8F0017047D7
S31500008E9051E8006F06EA020741E80076002EF7D196
S31500008EA0E4E730B400F00F00022303EB800C2D4DF5
S31500008EB0002305EBCC00002A428084BF2F4800EB3C
S31500008EC08C1004D9CC5CC4545B1C9A42FAD827494E
S31500008ED04FEA5C000968C14011F0010F14BF8821F8
S31500008EE0C82105F83C102149012303FA00F051E896
S31500008EF0003F83EA000C41E800C3002BF7D130BCE9
S31500008F00104670471F480178007940F2FF7202EA66
S31500008F100020084370471548406870472DE9F04126
S31500008F200F4E96F8800096F8905086F8800096F8D6
S31500008F3084100D4F01EA000414F0010F09D0FFF769
S31500008F4068FE00F0D8FB396800291CBF042002F037
S31500008F50C8FA19E004E100E0F0E4FF1F00800440D5
S31500008F60002007400016002060E5FF1FE8E4FF1F11
S31500008F70842007403EE5FF1F98200740A0160020EA
S31500008F8094200740A020074014F0100F0BD096F84D
S31500008F90840040F0200086F88400396800291CBF50
S31500008FA0102002F09EFA14F0200F0BD096F88400E1
S31500008FB020F0200086F88400396800291CBF202094
S31500008FC002F08FFA14F0040F1FBF39680029402001
S31500008FD002F087FADFF8CC80022C0ED014F0080FCE
S31500008FE008BFBDE8F081C5F303142F4E2F4FC5F31C
S31500008FF0C000C5F3800174B117E096F88800C8F880
S315000090000400396800291CBF802002F06AFAFF209C
S3150000901086F88800E2E7002202EB40020A4416F8CE
S315000090203220C2F383020D2A0AD0A20002EB4000CE
S31500009030451816F83500C0F3830001281FD117E044
S31500009040D8F8000020F00200C8F80000307E20F0BA
S3150000905080003076307C20F080003074396800293A
S3150000906008BFBDE8F0810220BDE8F04102F039BA40
S3150000907057F8241000291CBF042002F032FA16F813
S315000090803500C0F38300092818BFBDE8F08157F802
S315000090902410002908BFBDE8F0810820BDE8F04192
S315000090A002F01FBAE8E4FF1F00160020A01B0020F4
S315000090B00120FEF736B8FEF73BB838B569463C489E
S315000090C0FDF7F3FC002808BF38BD0098B0F5E01F97
S315000090D01CBF002038BD69464FF08070FDF7E5FCE7
S315000090E0002808BF38BD009810F0040F20D00020DB
S315000090F0FEF71EF82F4C01212046FDF7FCFC002848
S3150000910008BF38BD69464FF08070FDF7CEFC0028D9
S3150000911008BF38BD009810F0010FF3D0694620460D
S31500009120FDF7C3FC002808BF38BD00980028F5D11C
S31500009130012038BD10B586B0002000900190029045
S3150000914003901D4C0120FDF7F3FFFFF7B6FF102239
S3150000915069462046FDF75FFD10216846FFF7B4FA21
S31500009160ADF810000C216846FFF7AEFAADF8120014
S3150000917008216846FFF7A8FA20F4807040F40070D2
S31500009180ADF8140004A8FEF79BFD06B010BD7047AD
S31500009190B0F5806F0AD1087B00F03001202903D09A
S315000091A000F00300022801D001207047002070471C
S315000091B0FC000001040000015480044000207047B8
S315000091C0002070470020704700207047002070473D
S315000091D0002070470020704700207047002070472D
S315000091E0002070470020704700207047002070471D
S315000091F010B5FEF7F1F910BD10B5FEF7EFF910BD89
S3150000920010B5FE480024FE4944608460C4600461D1
S31500009210C0E90541C0E907144462FA498462C0E91D
S315000092200B4141630480FEF7DBF9F7484FF4165112
S3150000923001600471447108218171FEF7D3F910BDF4
S31500009240F24810B5C178026861F31F62EE490A6000
S3150000925002790A7142794A71807988710846FEF767
S31500009260C1F910BD10B5E848FEF7CAF9002808BFD5
S3150000927010BDE54AE54910680870030A4B70030CF7
S315000092808B70000EC870107908715079487190790A
S315000092908871012010BDD94910B50880FEF7DAF9AA
S315000092A010BDD648D0E90410081AD9490988081A09
S315000092B070472DE9F041D14F0C460646D7E9040127
S315000092C0D34A401A1188091A0029DCBF0020BDE8DC
S315000092D0F0818C42C8BF0C460025D7E906018842BA
S315000092E00FD3DFF81C831188031941448B4208D33E
S315000092F00D1A2A46314603F04BF82E44641BC7F874
S3150000930018803CB122463146B86903F041F8B86985
S315000093102044B8613969601901443961BDE8F081BA
S3150000932001B501216846FFF7C4FF01280CBF9DF86F
S3150000933000004FF0FF3008BD034670B5AF4D0C4638
S31500009340D5E90C01884298BF00240AD9401A844204
S31500009350C8BF04462246184603F01AF8686B204434
S315000093606863204670BD38B5A44D01246846D5E92A
S315000093700C218A420ED9521A012AB8BF1446224637
S3150000938003F006F8686B012C2044686304BF9DF85F
S31500009390000038BD4FF0FF3038BD9848D0E90C10BA
S315000093A0081A70479B4910B50978002904BF0020A8
S315000093B010BDA122984902230A7020224A70002279
S315000093C08A70CA700A714A718B71CA710872000A72
S315000093D0487292480A22007840F08000FFF761FD4B
S315000093E0012010BD10B5FFF70BFF10BD2DE9F047AA
S315000093F0824DA868002808BFBDE8F087D5E90401BA
S31500009400421AE8684FF0000652EA000104BFAE6057
S31500009410BDE8F0877E49DFF8E891814F0988DFF8DB
S31500009420048209EB01047549C96962B1A8698142E0
S3150000943022BF8818A042621A98F8000037F8100078
S315000094409042B8BF02467848EE60007840F080004F
S31500009450FFF727FDE9690144E9616A698C42024424
S315000094606A6108BFC5F81C902969914209D198F82C
S31500009470001037F81110814202BF0120E860BDE8F4
S31500009480F087EE60BDE8F08770B55C4C00250126DC
S31500009490206A002804BFD4E90C01884206D1594944
S315000094A0884203D02163E56225626163A06A80B1C8
S315000094B0206A002804BFE06A00280AD1266200F06C
S315000094C0D7F82562D4E90C0188421CBF401AFFF781
S315000094D081FED4E90101084318BF70BDD4E9040137
S315000094E0884208BF70BD6660A660FFF77FFF6560B3
S315000094F070BD704710B5414C206A18B1A06A401C77
S31500009500A06210BD01202062606200F0B1F8002068
S3150000951060622062D4E90C0188421CBF401AFFF742
S3150000952059FE10BD10B5354C6068002818BF10BD37
S3150000953001206060FFF75AFF0020606010BD10B583
S31500009540044610F0040F1CBF2046FFF7D3FF14F0AB
S31500009550080F08BF10BD294C6068002818BF10BD51
S3150000956001206060FFF742FF0020606010BD2F48B9
S31500009570006838B14FF6FF710846FDF7BBFFFDF7EF
S31500009580B5FFF7E729480068A0B100261B4C012566
S315000095904FF6FF710846FDF7ADFFFDF7A7FF10F088
S315000095A0080FF5D060680028F2D16560FFF71EFF4E
S315000095B06660EDE71D480068D0B300250F4C012614
S315000095C04FF6FF710846FDF795FFFDF78FFF10F088
S315000095D0040FF5D0206A18B1A06A401CA062EFE71C
S315000095E02662666200F044F865622562D4E90C01E1
S315000095F088421CBF401AFFF7EDFDE1E7F8E4FF1FC4
S31500009600460600204608002030E5FF1F30E0FF1F19
S315000096103CCA000039E5FF1F8608002038CA000052
S3150000962040CA00003BE5FF1F39CA000050CA0000CF
S31500009630FFE724480068D8B10027234D01264FF6DE
S31500009640FF710846FDF756FFFDF750FF044610F080
S31500009650040F1CBF2046FFF74DFF14F0080FEED095
S3150000966068680028EBD16E60FFF7C0FE6F60E6E722
S3150000967010B5154C164A1548216B1288164B081A58
S31500009680101A144A1B7832F81320904210DB134844
S315000096900078FFF7A2FB216B08442063A06A00282C
S315000096A008BF10BD616A002908BF401E08D010BD62
S315000096B00120E062606A00281ABFA06A401C10BD43
S315000096C0A06210BD50CA0000F8E4FF1F4608002043
S315000096D03ECA000040CA00003BE5FF1F3ACA000030
S315000096E010B5FDF70CFFFDF713FFBDE81040FFF7BF
S315000096F037BAFFF77ABAFE484FF001120178FD48F3
S31500009700C180002101704170C0E9022101617047EA
S31500009710F8484078002818BF012070470020F64915
S31500009720FFF75BBB10B5F54CF548A28801788A4275
S3150000973088BFCAB212B90020EE490871802021689C
S31500009740FFF7AFFB216801442160A188081AA080B9
S3150000975010BD10B5E94C00202168FFF73EFB2168DB
S3150000976001442160A188081AA08010BD002211467C
S315000097708020FFF796BBE3490020FFF72EBB2DE9BB
S31500009780F14F82B0DD4F0298A7F1180610F0020FD4
S3150000979000F0278306F120010020FFF71EFB06F1EB
S315000097A020042078C009FFF7DAFAE088B88020782C
S315000097B0C0F3411121B1012900F0F68200F002BB8D
S315000097C0CD4949780C2980F0FD82DFE801F0064397
S315000097D0FB62FB7E93FBFAF9F8F7C74910F01F000E
S315000097E008BFC94811D0012803D0022810D000F0C4
S315000097F0E9BA7078002800F0E5820879B1788842E5
S3150000980080F0E082BF4800210180386000F00FB987
S31500009810087900F08F0010F0800F1DBF00F00F01D7
S315000098204FF4803202FA01F1012108BF81407278BB
S315000098301AB910F00F0F40F0C582B068084200F068
S31500009840C182F068084018BF0120AE49088039601F
S3150000985000F0EDB8002002F01BFE002800F0B282F6
S31500009860002211468020FFF71CFBA848006848B17B
S315000098707169002918BF082000F0B382FDF730FE99
S3150000988000F0AFBAA2480168002940F08A8200F0D1
S31500009890A8BA012002F0FCFD002800F09382002205
S315000098A011468020FFF7FDFA9848006830B17169CB
S315000098B0002918BF042000F09482DFE7944801686D
S315000098C0002940F06E8200F08CBA8B4910F01F0F11
S315000098D040F078828878012140F08000307000F0F6
S315000098E07F00FFF7EAF9002211468020FFF7D9FA38
S315000098F000F077BA804910F01F0003D001287BD012
S3150000990000F060BAC878082880F05C82DFE800F0D2
S315000099105A04165B5A5A09367E483860122001905E
S3150000992078E07D480078002800F04C82F078002826
S315000099300CBF7A487A4838600A203DE076480078BD
S31500009940002804BFF078012800F03C82F078002857
S315000099500CBF7448744800908A78002042B1009980
S315000099600B7813B14B8819440091401C8242F6D102
S3150000997000980178002900F025821BE066480078EF
S31500009980002800F01F82F07800280CBF674868485E
S3150000999000908A78002042B100990B7813B14B8869
S315000099A019440091401C8242F6D1009801780029A2
S315000099B000F008823860408801902BE05AE147E1C8
S315000099C043E038E0B0E15B4800908B78032B14D07D
S315000099D0002043B100990A78002A1CBF1144009167
S315000099E0401C8342F6D10098017800291CBF3860DC
S315000099F0007800F0E781DFE705E0FEF7A0F93860C0
S31500009A00FEF794F9D8E701A9684600F0E3FA0028C2
S31500009A1000F0D881B9880198814208D9384980B2C6
S31500009A20B8800978491E084204BF01203071FFF74B
S31500009A3079FE00F0D6B910F01F0F40F0C3813E4802
S31500009A403860FFF76FFE00F0CCB94FF0000810F059
S31500009A501F0F40F0B78128488078002872D02E4822
S31500009A600078002804BFF078012800F0AB81F07878
S31500009A7000280CBF2B4C2C4C207800281CBF4FF420
S31500009A80803A4FF0010B7BD0607802280AD0042878
S31500009A9008BF94F8038074D0052808BFB8F1000FFA
S31500009AA07AD091E0144861798078814218BF608845
S31500009AB069D17070214B2079B07019880020002977
S31500009AC084BF1F4A002105D91154B3F800C0401CB9
S31500009AD08445F9D80125B1460BFA05F0D9F80810E6
S31500009AE008421CBF2846FFF74DF90AFA05F02AE09E
S31500009AF018CA000038E5FF1F58E5FF1F50E5FF1F95
S31500009B001CCA000030E0FF1F3EE5FF1F50CA0000E0
S31500009B104CCA0000C2CA000019CA0000D4CA00001C
S31500009B20D5CA0000D6CA000051CB000052CB0000B7
S31500009B3053CB000054CB000039E5FF1F1ACA0000C2
S31500009B402CE0FF1F47E0D9F8081008421CBF45F07B
S31500009B508000FFF717F96D1C102DBDD34FF00110D3
S31500009B60C9F808000020C9F80C00C9F81000012047
S31500009B70FFF7ABF8E07910F0400FB9F8060003E004
S31500009B804EE021E008E020E014BF40F0010020F0A4
S31500009B900100A9F8060017E0A07800F08F0515F07F
S31500009BA0800F1ABF05F00F000AFA00F00BFA05F055
S31500009BB0B1680843B0602046FFF7C8F82846FFF7AB
S31500009BC0CFF82846FFF782F820780444207800284A
S31500009BD07FF45AAF24E04FF00008012486F8018094
S31500009BE04FF480392546B16805FA04F008421CBFD7
S31500009BF02046FFF7C7F809FA04F0B16808421CBF0F
S31500009C0044F08000FFF7BEF8641C102CEBD34FF035
S31500009C100110C6E902080020C6F81080FFF755F8C3
S31500009C20A8487178807888427ED10022114680202B
S31500009C30FFF737F9A448006828B17169002918BFF1
S31500009C40012073D01AE6A148016800296FD1C8E047
S31500009C509C4900F01F00012866D17078002863D067
S31500009C600879B17888425FD2994908443860FFF78D
S31500009C7059FDB6E04FF0000900F01F00C846CA467D
S31500009C80CDF8049001284FD1707800284CD00020E0
S31500009C90009090480078002804BFF078012843D04F
S31500009CA0F07800280CBF8C4C8C4C2078E8B3607898
S31500009CB0022804D0042809D005281DD059E060796F
S31500009CC07178884218BF608854D152E07D4894F874
S31500009CD0029094F8038001794FF0000A494504BFC9
S31500009CE08078404545D101200090794810F8091048
S31500009CF0019100F809803CE072480179494538D164
S31500009D00A17801F08F0B1BF0800F1DBF0BF00F0227
S31500009D104FF4803101FA02F5012108BF01FA0BF573
S31500009D208078404516D103E04CE027E059E038E062
S31500009D30B0682843B060F068A843F0602046FFF79B
S31500009D4005F85846FFF70CF85846FEF7BFFF4AEAF3
S31500009D50050A0EE00198804508BF1AEA050F08D1EA
S31500009D60B068A843B060F068A843F0605846FFF7B3
S31500009D7009F8207804442078002898D1009808B380
S31500009D80002211468020FFF78CF84F48006828B162
S31500009D907169002918BF022023D06FE55048016879
S31500009DA0F9B1084680471CE010F01F000AD00128D0
S31500009DB008D100F042F9A0B900F0C0F988B900F066
S31500009DC093F870B93F48017811F0800F04D1C0882C
S31500009DD0002818BF002000D18020FEF7E5FF0020F4
S31500009DE0B880029810F0040F08D0364C207810F096
S31500009DF0800F13D03B490020FEF7EFFF029810F0CA
S31500009E00080F3ED02F48007810F0800F2FD0B8886A
S31500009E103179084318BFFFF785FC32E0B88800287F
S31500009E20ECD000203968FEF7D8FF39680144396064
S31500009E30B988081A0004000CB880DFD12078C0F376
S31500009E40411171B101290CD110F01F0009D0012870
S31500009E5007D100F042F90028D0D100F08DF8002893
S31500009E60CCD18020FEF7A0FF0020B880C6E730786E
S31500009E7010F0800F05D000F07F0030700021FEF753
S31500009E801CFF029810F0400F1CBF0020FEF798FF41
S31500009E90029810F0800F04BF03B0BDE8F08F802059
S31500009EA003B0BDE8F04FFEF78BBF0748006848B126
S31500009EB04FF6FF710846FDF71DFBFDF717FBFFF791
S31500009EC05EFCF5E758E5FF1F50CA000044CA0000D3
S31500009ED02CE0FF1F19CA0000D6CA000051CB0000B3
S31500009EE048CA000030E0FF1F70B53549354A087989
S31500009EF01278904203D0344A127890423AD13048D0
S31500009F004978324C324D4088042920D007DCA9B16B
S31500009F1001290DD0022911D0032911D02AE02029C8
S31500009F200CD0212917D022291AD023291CD021E0B0
S31500009F30FFF754F938B91DE0012070BD2C60FBE72E
S31500009F40FFF750F9B0B12C60FFF7ECFBF4E7FFF731
S31500009F504BF960B90EE0FFF785F90028F3D109E067
S31500009F60FFF799F918B905E0FDF75DFB10B1FFF7AA
S31500009F70FDFBE1E7002070BD10B51149114A0879D3
S31500009F801278904203D0104A1278904216D148783F
S31500009F9020B1022806D0202809D00FE0FFF71CF9CF
S31500009FA040B90BE04888FFF71BF918B906E0FFF740
S31500009FB047F918B1FFF7DAFB012010BD002010BDEC
S31500009FC058E5FF1F36CA000037CA000030E0FF1F01
S31500009FD050E5FF1F10B44A4A494BDFF828C1D27832
S31500009FE0494C1B79212A0DD0222A04BF9CF8000077
S31500009FF083421FD14548206045480088086010BC50
S3150000A000012070479CF80020934213D1414A1378EF
S3150000A010414A002B127808BF012A0BD0002A0CBF38
S3150000A0203E4A3F4A026010463E4A1288104420606B
S3150000A0300920E3E710BC0020704710B5304C3149C9
S3150000A04020790978884246D160780C2843D2DFE827
S3150000A05000F04206293342424242421B2D3C00F0A8
S3150000A060A4F8002837D0E078012802D0032804D0CD
S3150000A07006E025492C48086002E023492B48086081
S3150000A080FFF750FB012010BDE078022802D003281C
S3150000A09004D00FE01C49264808600BE01A49234803
S3150000A0A0086007E000F0B1F848B914E000F0B5F830
S3150000A0B070B910E0012010BD00F0C7F858B1124980
S3150000A0C01C480860FFF72EFBF4E700F0C5F810B156
S3150000A0D0FFF74CFBEEE7002010BD10B50848094A13
S3150000A0E001791278914204BF4078092806D100F020
S3150000A0F073F818B1FFF73AFB012010BD002010BD20
S3150000A10058E5FF1F1DCA000050E5FF1F9CCA00004E
S3150000A110BECA000019CA00003BE5FF1FD6CA0000F0
S3150000A12051CB0000C0CA0000850500203EE0FF1F9D
S3150000A130C605002030E0FF1F00F0F1BA10B5134845
S3150000A140134A0179127891421DD142784188C0881C
S3150000A150FE2A0AD0FF2A04BF0029002813D100F0E6
S3150000A16007FB80B1FFF702FB0BE0002908BF0128BF
S3150000A17009D100F006FB30B1074906480860FFF731
S3150000A180D1FA012010BD002010BD000058E5FF1FC8
S3150000A1902ECA000030E0FF1F50E5FF1F7047002069
S3150000A1A070477047002070477047FC490022C87806
S3150000A1B0012808BFFA4A07D0022804BF00207047CA
S3150000A1C0032808BFF74A00D1521C10B5897800232E
S3150000A1D0FDF753FA012010BDF0490022C878012886
S3150000A1E004BF00207047022808BFEF4A03D00328A7
S3150000A1F008BFEC4A00D1521C08B500230093CB8857
S3150000A2008978FDF764FA012008BDE448E7498078BB
S3150000A210085CE749087001207047E048DF4980780C
S3150000A220C97810B1E34A81540DE0E34A002013785F
S3150000A230002B88BFDD4B06D91954401C92F800C08C
S3150000A240C0B28445F8D80120704710B5FFF7AAFFC1
S3150000A250D7490870012010BDD04810B58078FFF7A7
S3150000A260A3FF012010BD2DE9F047D44EB0887188B8
S3150000A270DFF82C83DFF84093002508F101048842BB
S3150000A28024BFB069002816D17561B580012398F8FE
S3150000A290001022461846FDF7F0F97080708850B11C
S3150000A2A0C6F8148099F80000012898BF746102D995
S3150000A2B07088401C708070880127002842D1F068A1
S3150000A2C0002818BFF5603DD1306900283AD099F8CA
S3150000A2D00010012988BF98F8004010D888F800506F
S3150000A2E0B580022308F1010200210120FDF7C5F91E
S3150000A2F070807088002818BF7461356122E0202CB8
S3150000A30028BF002407FA04F1014204BF611CCCB245
S3150000A310F5D0601CC1B288F80010B580022308F1A0
S3150000A32001020120FDF7A9F97080708820B1C6F8F6
S3150000A33014807088401C7080316907FA04F021EAA5
S3150000A340000030617088B169084308BFBDE8F08736
S3150000A3507088B188DFF86C92401A84B2DFF86082A8
S3150000A36099F8000038F81000A04238BF0446964815
S3150000A37022467169007840F08000FEF792FD706910
S3150000A380924920447061B088204480B2B080098828
S3150000A390884208D299F8000038F81000A04204BF9D
S3150000A3A0B761BDE8F087B561BDE8F087F8B5834CC5
S3150000A3B000267D4DE088002808BFE5618448E169F4
S3150000A3C00078FEF70AFD0004E169000C0144E16132
S3150000A3D0E18801448BB2E3800BD07E4909888B4229
S3150000A3E007D2784A7649127831F81210884228BF87
S3150000A3F0F8BD7948017801200129009005D86A4AFC
S3150000A40000210220FDF763F905E029785B1E6A1C2E
S3150000A4100220FDF75CF9E680F8BD6848002141702E
S3150000A420C16001614161418081808161C161C180FA
S3150000A43001620181704710B5044610F0080F1CBF79
S3150000A4402046FFF710FF14F0040F08BF10BD20468A
S3150000A450BDE81040AAE761480078002808BF7047A9
S3150000A4602DE9F05F554F042300243978481C3870D5
S3150000A4705448007800EB400293405B1E994202DB91
S3150000A480002139700124564B4FF0000C1988FF2922
S3150000A4903CBF491C1980534931F810905048008838
S3150000A4A0814508BF4FF0010C0020434B1978002965
S3150000A4B04FD90221DFF830E1DFF830A101FA02F8C6
S3150000A4C04FF0010B002274B11AF80010FF293CBFAF
S3150000A4D0491C0AF800101EF8001021B11AF80030C5
S3150000A4E08B4228BF01221EF8005005FA08F14945A3
S3150000A4F003DA002D18BF012300D10023BCF1000FA1
S3150000A50018BF002B04D03E690BFA00F131433961C4
S3150000A5102649095C8D420CD01AF800508D4206D3AC
S3150000A5203E690BFA00F535433D6100253D700EF896
S3150000A530001042B123B93A690BFA00F111433961AF
S3150000A54000210AF800101C49401CC0B20978884254
S3150000A550B8D3BCF1000F02D0214900200880386929
S3150000A560002808BFBDE8F09F7888002818BFBDE81E
S3150000A570F09F0020BDE8F05F75E61D480068C8B38F
S3150000A5804FF6FF710846FCF7B5FFFCF7AFFF10F07A
S3150000A590080F1CBF0020FFF766FEF1E758E5FF1F16
S3150000A5A0840500203DE0FF1FC50500203CE0FF1F9D
S3150000A5B030E0FF1F3BE0FF1F28CA000064E5FF1FD5
S3150000A5C024CA00003BE5FF1F1ECA00002ACA00007D
S3150000A5D01FCA00002CCA000029CA000039E5FF1F67
S3150000A5E038E0FF1F20CA00003BE0FF1F3AE0FF1FD4
S3150000A5F050CA0000FFE73648006868B14FF6FF71A1
S3150000A6000846FCF777FFFCF771FF10F0040F1CBF3C
S3150000A6100020FFF7CBFEF1E72D480068A0B14FF60A
S3150000A620FF710846FCF766FFFCF760FF044610F072
S3150000A630080F1CBF2046FFF716FE14F0040F1CBFC0
S3150000A6402046FFF7B3FEEAE72DE9F0410746214829
S3150000A65016460088824238DC1F480378002B34D027
S3150000A6601E4C0120E06060884FF0000830B100E029
S3150000A67003B3B4F802C0BCF1000FF9D1184D681C41
S3150000A6802F7001F085FE6561A4F804806680154888
S3150000A6900078012899BF681C60616088401C88BFEB
S3150000A6A060800020FFF7DFFD0F4800F807800120DB
S3150000A6B0BDE8F081C4F80C80C4F81480A4F80480C6
S3150000A6C0A4F802800020BDE8F0810020BDE8F081FA
S3150000A6D050CA00002ACA000039E5FF1F64E5FF1FC3
S3150000A6E08405002028CA00003AE0FF1F7047704723
S3150000A6F07047704710B50446FEF756FB14F0800FFE
S3150000A7001DBF04F00F004FF4803101FA00F0012064
S3150000A71008BFA040FC490A681043086010BDFB480A
S3150000A720007900F08F0010F0800F1DBF00F00F01C0
S3150000A7304FF4803202FA01F1012108BF8140F44A48
S3150000A740137843F08003834218BF7047EE480068D1
S3150000A750084208BF7047EF48EF490068884218BFB3
S3150000A760704710780D2240F08000EA49FEF799BB49
S3150000A770EA4900200860E7490860E94908700120B5
S3150000A7807047E8490020087001207047E14910B57C
S3150000A790E1480860DE480D22007840F08000FEF7B0
S3150000A7A080FBDF490520087010BDDD4910B54868FB
S3150000A7B0C86000281CBF012010BDDB48816859B164
S3150000A7C0007B10F0800F0CBFD848D148007818BF26
S3150000A7D040F08000FFF78EFFCE4901200873FFF797
S3150000A7E0D5FF002010BD2DE9F041CD4DDFF82083C7
S3150000A7F00026A969686AC74F88420AD398F80000FC
S3150000A800002440F08000FFF775FF3E73FFF7BEFFA0
S3150000A81008E0C849C648097830F81140E86A844219
S3150000A82028BF0446FFF7C1FF002808BF0024A86A16
S3150000A83000282FD07CB1A96AE8692246014498F81D
S3150000A840000040F08000FEF72CFBA86A2044A862B6
S3150000A850E86A001BE862D5E90410AA6A41439142FE
S3150000A86003D1AE62696A08446862B868001BB860C2
S3150000A870002C08BFBDE8F081E86A002804BF032069
S3150000A880287004D02878022808BFBDE8F0813E73FE
S3150000A890BDE8F081002CDED0E96A28690144491E32
S3150000A8A0B1FBF0F26869824288BF0246E969686ACC
S3150000A8B0FCF7BEFFBFE72DE9F041994D0026954F05
S3150000A8C0A969686A884207D398482E630078FFF71B
S3150000A8D011FF3E73FFF75AFFFFF767FF002808BF17
S3150000A8E02E630020296B002984BF9349EA6909D9A0
S3150000A8F0D5F828C00B5C8444401C02F80C302B6B46
S3150000A9008342F5D8296BA86A0844A862EA6A521AF3
S3150000A910EA6209B392B988B129690844401EB0FBBE
S3150000A920F1F46869844288BF04462246E969686A88
S3150000A930FCF7DEFFAE62686A20440CE0D5E904123B
S3150000A9405143814208D1E969686AFCF7D1FFAE62DA
S3150000A9506969686A08446862B968286B091AB96047
S3150000A960002808BFBDE8F081E86A00281EBF2878E5
S3150000A9700528BDE8F0813E73BDE8F04106E72DE904
S3150000A980F041674C0025634EA169606A884207D38F
S3150000A990664825630078FFF7ADFE3573FFF7F6FED0
S3150000A9A0FFF703FF002816BF206B2563002823D07E
S3150000A9B0A06A68B9E16A20690144491EB1FBF0F258
S3150000A9C06069824288BF0246E169606AFCF730FF2F
S3150000A9D0226B0020002A0FD9574BD4F81CC0A16A5D
S3150000A9E013F800800F181CF80770474501D0256240
S3150000A9F002E0401C9042F3D3A16A206B0A18A262BF
S3150000AA00E16A0B1AE362D4E904C101FB0CFC94452C
S3150000AA1003D1A562626A11446162B168091AB16024
S3150000AA20002808BFBDE8F081002B1EBF207805284E
S3150000AA30BDE8F081206A00280CBF01200020307399
S3150000AA40BDE8F041A2E670B5374C354DD4F811009B
S3150000AA50217D00BA20F0FF0001430020C5E909105E
S3150000AA60E07B2F280AD004DC28280CD02A2805D021
S3150000AA7018E0A8280FD0AA2808D013E0FFF795FE03
S3150000AA80002808BF70BDE08A41BA0BE0FFF78DFED3
S3150000AA90002808BF70BDD4F81500217E00BA20F04A
S3150000AAA0FF00014328694143E962A068194D012668
S3150000AAB078B1884204BF012070BD207B10F0800F62
S3150000AAC014BF13481948007818BF40F08000FFF7FC
S3150000AAD011FE2E73FFF75AFE002070BD70B51248A6
S3150000AAE0022500F11F04816849B1007B10F0800F38
S3150000AAF01CBF012070BD0D480078FFF7FBFD2573D4
S3150000AB00FFF744FE002070BD44E5FF1F58E5FF1F18
S3150000AB102FCA0000FF1B00205553425348E5FF1F74
S3150000AB2088E5FF1F30E0FF1FE01B002030CA000051
S3150000AB3032CA00003BE5FF1F0606002010B5F948A3
S3150000AB40F94C8068216B88429ABF20630320042059
S3150000AB502070F648F649226B007840F08000FEF738
S3150000AB60A0F9F448226B8168891A8160002101737B
S3150000AB7010BDEC4810B5816800F11F0481B1007B5F
S3150000AB8010F0800F0CBFEC48E848007818BF40F082
S3150000AB908000FFF7AFFD01202073BDE81040F5E50A
S3150000ABA0FFF703FE002808BF10BD00202073BDE894
S3150000ABB01040EBE510B5FFF791FF002808BF10BD68
S3150000ABC07021DB48D84B017000214170D3F80CC0CE
S3150000ABD05A6832EA0C0C0AD04FF0060C80F802C014
S3150000ABE04FF0280C80F80CC04173DA600CE0F2B12B
S3150000ABF0D04A127B002A04BF8170017303D005225C
S3150000AC008270202202734173C1700171417181719A
S3150000AC100A22C271017241728172C1728173C1735B
S3150000AC200174417412201863BDE8104086E70222C1
S3150000AC3082703A2202734173E6E710B5FFF74EFFC2
S3150000AC40002808BF10BD0020B94B80214FF0200C12
S3150000AC501870597002219970D97083F804C0587120
S3150000AC609871D871B548016808200A78002A1ABF79
S3150000AC701A54491C03F800C0401CC0B22428F4D35F
S3150000AC80A94924200863BDE8104057E7A54810B538
S3150000AC90817C00F11F0421B101202073BDE8104022
S3150000ACA074E5C07CA04900F001004860FFF721FD73
S3150000ACB000202073BDE8104068E59A48C07C10F07B
S3150000ACC001019C4818BF012101735FE510B5FFF72C
S3150000ACD005FF002808BF10BDFFF767FD002808BF65
S3150000ACE010BD03219248002201708F4942700B7AF1
S3150000ACF0DB018370C270042008638E498A68042AC7
S3150000AD0003D9A1F11F0290608860BDE8104015E7E5
S3150000AD1010B5FFF7E3FE002808BF10BDFFF745FD9D
S3150000AD20002808BF10BD0021814806227E4B017015
S3150000AD30427081701A7AD201C270017141718171BB
S3150000AD40C1717C49082018638A68082A03D9A1F1D1
S3150000AD501F0290608860BDE81040EFE610B5FFF76F
S3150000AD60BDFE002808BF10BDFFF71FFD002808BF65
S3150000AD7010BD6D4A6E499069401E030E0B70030CA0
S3150000AD804B70030A8B70C8701069030E0B71030CAD
S3150000AD904B71030A8B71C87108201063BDE810401F
S3150000ADA0CCE610B5FFF79AFE002808BF10BDFFF7E6
S3150000ADB0FCFC002808BF10BD00215D485A4A0170FE
S3150000ADC0417081700821C17091690B0E03710B0CE3
S3150000ADD043710B0A8371C1710221017211690B0C57
S3150000ADE043720B0A8372C17252490C2010638A683F
S3150000ADF00C2A03D9A1F11F0290608860BDE81040BB
S3150000AE009CE64C4900200873C0E470B5FFF766FE67
S3150000AE10002808BF70BD02224548434D454C0270CC
S3150000AE20427003202A632870A068022803D9A4F17F
S3150000AE301F008260A2603D483D49007840F08000D6
S3150000AE40FEF72FF8A068296B401AA0600120207336
S3150000AE5070BD10B5FFF742FE002808BF10BD2022C6
S3150000AE6033480021304C02704170C17703202263C1
S3150000AE7020702E482E49007840F08000FEF711F829
S3150000AE802C48226B8168891A81600121017310BDEB
S3150000AE902DE9F05F244F0020224D396B002988BF31
S3150000AEA0234A04D9135C2B54401C8142FAD801264C
S3150000AEB0DFF87880DFF880B01F2970D12868204934
S3150000AEC088426CD11B4C68686060A968A160687B89
S3150000AED000286DD1A87B00286AD0102868D8E87BA6
S3150000AEE04FF000094FF0020A2A287CD02ADC1A28E3
S3150000AEF07AD009DC04285BD003DC90B103284FD05C
S3150000AF0056E0122854D14EE023287AD004DC1B28C0
S3150000AF104CD01E285DD04BE0252875D028287CD043
S3150000AF2046E028E0E01B002088E5FF1F2FCA00004E
S3150000AF3006060020FF1B002030CA000028E0FF1F85
S3150000AF40555342439E2865D00CDC552830D004DC8E
S3150000AF502F287DD0352849D02AE05A284ED091286E
S3150000AF6044D025E0A12852D0A3280CD0A82854D03C
S3150000AF70AA286CD01CE069B1287B10F0800F08BFAE
S3150000AF809BF8000003D098F8000040F08000FFF71F
S3150000AF90B1FB0DE0FFF709FC40BBBDE8F09F8AE07E
S3150000AFA0BDE8F05F06E6BDE8F05F46E6A87C20B1A6
S3150000AFB02673BDE8F05FFFF7E9BBE87C00F001000F
S3150000AFC07860FFF796FB84F80C90BDE8F05FFFF71A
S3150000AFD0DDBBE87C10F0010F14BF267384F80C90DB
S3150000AFE0BDE8F05F05E032E005E00AE05DE00BE079
S3150000AFF013E0FFF7CBBBBDE8F05F67E6BDE8F05FA7
S3150000B00086E6BDE8F05FCCE6BDE8F05FA6E6BDE803
S3150000B010F05FFAE6BDE8F05F1BE7FFF714FD0028D6
S3150000B02008BFBDE8F09F287B10F0800F05D087F899
S3150000B03000A0BDE8F05FFFF7D6BB9BF80000FFF766
S3150000B04059FB84F80CA0BDE8F05FFFF79FBB00E05A
S3150000B0500DE0FFF7F8FC002808BFBDE8F09F287B4D
S3150000B06010F0800F04BF3E70BDE8F09F11E0287C11
S3150000B07010F0020F19D0FFF7E6FC002808BFBDE864
S3150000B080F09F287B10F0800F02BF3E703E62BDE845
S3150000B090F09F98F8000040F08000FFF72BFB84F843
S3150000B0A00CA0BDE8F05FFFF771BB84F80C90BDE81B
S3150000B0B0F05FFFF76BBB98F8000040F08000FFF7E9
S3150000B0C019FB98F80000A34C00F00F004FF48031F4
S3150000B0D001FA00F02168084320609BF80000FFF7A2
S3150000B0E009FB9BF80000216806FA00F0084320607F
S3150000B0F006203870BDE8F09F974910B508780228F9
S3150000B10008D0032810D0042812D0052804BF002038
S3150000B110087010BD9148C07B28281CBFA82810BD08
S3150000B120BDE81040FFF75FBBBDE81040FFF72EBB40
S3150000B1308B48007840F08000FFF7DCFABDE810404D
S3150000B140FFF724BB844810B5007878B1012810D0E9
S3150000B150052808BF10BD83480078FFF7CBFA82495F
S3150000B16002200873BDE81040FFF710BBBDE8104091
S3150000B1708EE67A48C07B2A2804D02F2806D0AA2833
S3150000B18018BF10BDBDE81040FFF795BBBDE81040E5
S3150000B190FFF7F5BB704910B50878022808D00328D8
S3150000B1A010D0042812D0052804BF0020087010BD56
S3150000B1B06A48C07B28281CBFA82810BDBDE81040DF
S3150000B1C0FFF711BBBDE81040FFF7E0BA644800780E
S3150000B1D040F08000FFF78EFABDE81040FFF7D6BAC0
S3150000B1E010B5604C61492078FDF7F7FD5A490863B0
S3150000B1F0087870B101280FD0052808BF10BD207847
S3150000B200FFF778FA584902200873BDE81040FFF7A7
S3150000B210BDBABDE810403BE65048C07B2A2804D0A2
S3150000B2202F2806D0AA2818BF10BDBDE81040FFF78A
S3150000B23042BBBDE81040FFF7A2BB10B5044610F0B4
S3150000B240040F1CBF0020FFF7CBFF14F0080F08BF48
S3150000B25010BD0020BDE810409CE74548006850B38B
S3150000B2603E4E3F4F3C4C00254FF6FF710846FCF71B
S3150000B27041F9FCF73BF910F0080FF5D020780228C9
S3150000B28007D003280CD004280DD0052808BF257048
S3150000B290EAE7F07B282814BFA828FFF7A4FAE3E71B
S3150000B2A0FFF774FAE0E7387840F08000FFF722FAFB
S3150000B2B0FFF76CFAD8E72E48006878B3274E264C7D
S3150000B2C0284D022706F11F084FF6FF710846FCF7C6
S3150000B2D011F9FCF70BF910F0040FF5D02349287883
S3150000B2E0FDF77BFD2063207858B101280CD0052896
S3150000B2F0EAD02878FFF7FEF988F80C70FFF746FACF
S3150000B300E2E7FFF7C5FDDFE7F07B2A2803D02F2809
S3150000B31005D0AA28D8D1FFF7CEFAD5E702E0FFF785
S3150000B3202EFBD1E712480068A0B14FF6FF71084620
S3150000B330FCF7E0F8FCF7DAF8044610F0040F1CBF3F
S3150000B3400020FFF74DFF14F0080F1CBF0020FFF789
S3150000B35021FFEAE748E5FF1F88E5FF1FE01B002005
S3150000B3602FCA000030CA0000FF1B0020060600207E
S3150000B37050CA0000428C920803D1274A1288C2F3B1
S3150000B3808D02836A03EB820212F0040F18BF121FAC
S3150000B390A2F140034FF08072C3E90E1200229446D8
S3150000B3A043F822C0521C0E2AFAD3C2691A624362BB
S3150000B3B0C162806A1949016070471948006810F037
S3150000B3C0807F08BF70471748006810F0010F08BF5C
S3150000B3D070471548006810F0004F08BF70470120FD
S3150000B3E01249087070474FF06042D36F002BFCD0B3
S3150000B3F0C36AD367D36F002BFCD0C07840EA012024
S3150000B400A2F87C0070474FF06041CA6F002AFCD05A
S3150000B41081F87C007047000060C50000A52E5AE246
S3150000B420FCED00E0800E00E0000E00E0C0E5FF1F2E
S3150000B4308C46494910B50B68198B7AB130EA01027E
S3150000B44018BF062105D05883604600F05DFD012037
S3150000B45010BD21EA00001883022010BD11EA000287
S3150000B46014BF5A830521F4D1EDE770B53B4A02EBD0
S3150000B470810151F8044C002C08BF70BD218B084394
S3150000B48020836178658B06291AD0052918BF70BDFF
S3150000B49028421ABF05EA0001618370BDA8432083D4
S3150000B4A0204600F06EF9208BA843208301206070AF
S3150000B4B0022084F820002046BDE8704000F001BD5F
S3150000B4C035EA0001EAD070BD244A02EB810151F849
S3150000B4D0041C002908BF70470A8B22EA0000088373
S3150000B4E0704702461D4810B500EB810050F8040C69
S3150000B4F0002808BF10BD114600F059F9BDE81040FC
S3150000B50000F046BC14480068408B704710B50446EE
S3150000B510008B084320836278618B062A18D0052A9F
S3150000B52018BF10BD08421ABF01EA0002628310BDAF
S3150000B53088432083204600F024F901206070022011
S3150000B54084F820002146BDE81040054800F00AB8FE
S3150000B55031EA0002ECD010BDD4E5FF1F4C050020F7
S3150000B5600C1C002010B402780024022A1ABF012AFB
S3150000B570032A01248B7842682AB192F802C09C45BE
S3150000B58028BF1046F7D24A604160002C01BF002058
S3150000B590886010BC7047002A18BF9160886010BC94
S3150000B5A0704701464068002342684A600A78022ACA
S3150000B5B018BF012A03D0032A1CBF436070474268A4
S3150000B5C0002A1CBF91604360836070478C494A68BB
S3150000B5D0426000228260486070478949894B48680A
S3150000B5E01B6882789B789A4206BF42684A600020B0
S3150000B5F070478168002908BF814907D042684A60C0
S3150000B600416800291CBF8068886070474A6882428A
S3150000B61002D14068486070471100F7D170478368CF
S3150000B62084461BB11978184639B10AE09CF8010026
S3150000B63001280CBF7248704703E080680278002A30
S3150000B640FBD06146002B08BF6D4A08D04A685A6095
S3150000B6504A68002A1CBFDCF80810916008E05368AD
S3150000B6608B4203D1DCF80410516001E01A00F6D1D8
S3150000B670614677E7644AD36813B313469B8A8B42C5
S3150000B6800BD204E0D2F80CC0BCF1000F18D0D2687F
S3150000B690B2F814C063448B42F4D3D2F80CC0C0F89D
S3150000B6A00CC0D0600261D0F80CC0BCF1000F18BF0E
S3150000B6B0CCF81000591A8182908A401A90827047FD
S3150000B6C04FF0000CC0F80CC0D060C91A026191821C
S3150000B6D0A0F814C070472DE9F0014B4DE86800282A
S3150000B6E004BFBDE8F0017047A88A0024401E474FFA
S3150000B6F0A8820126A88A00281CBFBDE8F001704771
S3150000B700E868002804BFBDE8F0017047816839B1D8
S3150000B71042684A60416811B182688A604460846008
S3150000B720374A0023117802291ABF01290329012368
S3150000B73090F802C0516829B191F80280E04528BF0F
S3150000B7400A46F7D241605060002B08BF846003D0E0
S3150000B750002918BF88608260818AA98241780429FD
S3150000B76003D1C18A3A8811448182467080F82060EC
S3150000B770C168E960C16800291CBF0D61C46004612D
S3150000B780B8E70169002908BF7047C268CA60C36884
S3150000B7900022002B08BF8A8207D08B8AB0F814C01B
S3150000B7A063448B82C3681961C26002617047F0B45A
S3150000B7B0174DAA1CEC78AC46D2E84F3FA3420ED1F7
S3150000B7C0BFF32F8FEA789A4281BF05EBC302C2E925
S3150000B7D00101F0BC70470220F0BCFAF743BE5B1CC7
S3150000B7E0C2E8463F002EE7D1DCE84F3F5A1CA24292
S3150000B7F008BF0022CCE8462F002EF5D1E2E7000074
S3150000B8000C1C0020D4E5FF1F241C0020DCE5FF1FD4
S3150000B8102805002001220270002242704260028147
S3150000B820428110398281C1F38F01C18170472DE9B0
S3150000B830F0410D468189A14F43681646002403B1A5
S3150000B84069B1C28991422CD1002E04BF0120BDE806
S3150000B850F0819A490968A3B1FFF784FE18E0FFF763
S3150000B860A0FE0646C0690560042086F82000304622
S3150000B870FFF787FF304600F024FB386880F8204049
S3150000B88024E0416039684C60396888600121417064
S3150000B89038680821C561304600F036FB0120BDE856
S3150000B8A0F081018900EB81010D6100F10C01D1E805
S3150000B8B05F2F531CC1E8523F002AF8D10189491C69
S3150000B8C089B20181C289914208BF04810020BDE886
S3150000B8D0F0812DE9F041044680890026774F904695
S3150000B8E00D46002839D0608904EB800000690860A5
S3150000B8F06089401C80B26081E189884208BF668108
S3150000B9006068002808BF04F10C001CD02046FFF731
S3150000B91048FE80F820602189054604EB8101C06954
S3150000B92008612089401C80B22081E189884208BFD5
S3150000B93026812846FFF725FF284600F0C2FA386818
S3150000B94080F8206006E0D0E85F1F4A1EC0E8512F4D
S3150000B9500029F8D10020BDE8F081B8F1000F04BF3E
S3150000B9600120BDE8F08155496068096818B1204694
S3150000B970FFF7F8FD04E06160386846603868846067
S3150000B9800821404600F0C0FA3868C5610120BDE8CC
S3150000B990F081C1898089081A704710B5FFF707FF43
S3150000B9A0BDE8104000F0F4B910B5044680890028BF
S3150000B9B008BF10BD608904EB8000006908606078EC
S3150000B9C0012807D10220607000212046FFF7EFFE14
S3150000B9D000F0DEF904F10C00D0E85F1F4A1EC0E853
S3150000B9E0512F0029F8D16089401C80B26081E1891D
S3150000B9F0884204BF00206081042010BD2DE9F0417B
S3150000BA00044640688846002704F10C0528B1607892
S3150000BA1002281CD0A089002835D0A089E189884257
S3150000BA2046D2208904EB8000C0F81080D5E85F0F6D
S3150000BA30411CC5E8501F0028F8D12089401C80B25F
S3150000BA402081E189884208BF2781BDE8F081204630
S3150000BA506770FFF7A6FD80F820702189064604EB83
S3150000BA608101C0690861D5E85F0F411CC5E8501F18
S3150000BA700028F8D12089401C80B22081E1898842C3
S3150000BA8008BF278109E02046FFF78BFD0646C069FF
S3150000BA900421C0F8008086F820100120707030461E
S3150000BAA0FFF76FFE3146BDE8F0410548FFF75ABD86
S3150000BAB0BDE8F0410320FAF7D5BC0000D4E5FF1F2E
S3150000BAC00C1C002012F0004F1FBF22F00042D21DB6
S3150000BAD022F00703102202BFD21C22F003030C221D
S3150000BAE01BB103EB020C8C4501D9012070470244BF
S3150000BAF001448360C0E90021C91AD01888429CBF5E
S3150000BB0010600246F9D9002010607047014651E8DE
S3150000BB10000F28B1036841E80032002AF7D17047C8
S3150000BB20BFF32F8F704710B50446F9F78FFC002836
S3150000BB3008BF10BD0246A168002914BF002310BD2E
S3150000BB4042F8043B091FFBD110BD814224BF426865
S3150000BB508A429CBF0120704750E8002F0A6040E8E7
S3150000BB600012002AF8D1002070470000022202705D
S3150000BB70002242604180704710B5416881B1FFF7ED
S3150000BB8010FD0321044680F82010FFF7FAFD204639
S3150000BB9000F097F924490020096881F8200002E0A6
S3150000BBA04188491C4180002010BD10B50C464188D3
S3150000BBB019B1491E4180002010BD002C04BF012090
S3150000BBC010BD194A4368116813B1FFF7CBFC05E0B5
S3150000BBD0416013680021596011688860072120467A
S3150000BBE000F092F9012010BD10B50021FFF7DFFD2E
S3150000BBF0BDE8104000F0CCB810B5416879B1FFF748
S3150000BC00D0FC0446FFF7BDFD01206070032084F8D8
S3150000BC1020002146BDE810400448FFF7A3BC418838
S3150000BC20491C418010BD0000D4E5FF1F0C1C0020FC
S3150000BC3095490123954A48684FF0E02C00280ADA16
S3150000BC400520CCF810000B70136800EA936088702A
S3150000BC5040061060704710B400F01F0403FA04F4A5
S3150000BC6040110CEB8000C0F880410B701068C0F3E7
S3150000BC7000708870C006106010BC704710B54FF693
S3150000BC80FF74FFF7D5FF8248C168002918BF848A70
S3150000BC908048016800291CBF8088A04238BF04463E
S3150000BCA0204610BD70B4784A002310465168774C80
S3150000BCB080784FF0E02C00290BDA0721CCF8101021
S3150000BCC01370517840EA810080062060537070BC82
S3150000BCD0704701F01F05012606FA05F549110CEB20
S3150000BCE08101C1F8005113705178084300072060A4
S3150000BCF0537070BC70472DE9F04105466648012730
S3150000BD0001684F700068FFF761FC6449DFF88081C5
S3150000BD1000200860624ED8F80C00E0B1B8F81410A4
S3150000BD20A94211D830686C1A08443060A8F814701B
S3150000BD30FFF7D1FC94B13068641E401C3060D8F81F
S3150000BD400C000028F4D109E0326850193060481B15
S3150000BD50A8F8140002E03068284430604D4E306880
S3150000BD6070B1B088A84299BF2C1AB780401BB0802A
S3150000BD7006D800F0AFFA1CB13068641E0028F8D16E
S3150000BD804848FFF70EFC00F097F8BDE8F04189E758
S3150000BD903D48017800291EBF0121417070474FF0D0
S3150000BDA080503A490860704770B53B4801210268E7
S3150000BDB051700068FFF70AFC3B4EB0787478002893
S3150000BDC018BFB51C17D006EBC40148680278D2B17B
S3150000BDD0012A1DD0FFF710FFF078641C844208BFCB
S3150000BDE00024D5E84F0F411EC5E8401F0028F8D1B2
S3150000BDF0B0780028E7D174702A48FFF7D2FBBDE877
S3150000BE00704000F059B8098989B2FFF77FFBE3E774
S3150000BE108968FFF7F3FDDFE7244801684FF0E0206B
S3150000BE20416100218161072101612148016841F0DA
S3150000BE307F410160401770477047174810B5026888
S3150000BE40012151700068FFF7C1FBFAF70DFB14489A
S3150000BE500168491C0160FFF73EFC00F03BFA1148FF
S3150000BE60FFF79FFBBDE8104000F026B80A480068BF
S3150000BE70D0E90910814204D300680E49884208BF00
S3150000BE8070470120FAF7EEBACCE5FF1F04ED00E09B
S3150000BE90241C0020E0E5FF1FD4E5FF1FC4E5FF1FBB
S3150000BEA0DCE5FF1F0C1C00202805002064C50000EF
S3150000BEB020ED00E0A52E5AE2DF49486002214170DC
S3150000BEC070472DE9F041DC4D04004FF002060DD01D
S3150000BED02868A1780127827891420ED9FFF776FB70
S3150000BEE0286847706C606670BDE8F081D348FFF73C
S3150000BEF058FB68604670BDE8F08167702146BDE872
S3150000BF00F041CE48FFF72EBB002808BF704770B53A
S3150000BF100C464FF6FF71C84D884204D22A68014686
S3150000BF201046FFF7A7FB28684470C448FFF739FBA3
S3150000BF3002216860417070BD70B5FFF74EFB0400CA
S3150000BF4008BF70BDBC4DBD482968FFF70BFB2968CB
S3150000BF500120487002206C60607070BDB6480068B1
S3150000BF60002818BFC078704770B50026B24D00286B
S3150000BF7004BF286881700DD0B14A128890421AD841
S3150000BF80B04A02EB800050F8044CA4B1A1702868B6
S3150000BF90A04212D1A9484068807888421BD9A74898
S3150000BFA02968FFF7DFFA296801204870286880F8B9
S3150000BFB0206000200DE0FF2070BD2046FFF72FFB1C
S3150000BFC06078012807D19D48FFF7EBFA296881F8C8
S3150000BFD02060FFF776FF002070BD2DE9F0411C467A
S3150000BFE0174680460E4611F0FF0F08BF4E1C9648B6
S3150000BFF0FFF78CFD050008BFBDE8F081C6F30F20F2
S3150000C000AF626884EC6100272F7001216970AE7001
S3150000C0106F60AF60EF602F61AF82EF822F836F8317
S3150000C02085F820702C4685F8217018B98748FFF7E7
S3150000C0306DFDA06241462046FFF79CF98048012429
S3150000C04080490288012A08D301EB840252F8042CA5
S3150000C05022B10288641C9442F6D93C4601EB840066
S3150000C06040F8045CEC702846FFF72BFF7248006826
S3150000C07080F820402046BDE8F08170B56E4C002661
S3150000C080704D216800281CBFCA7882421AD14E70B2
S3150000C090F9F7CBF921684862FFF7E8FE2068C17816
S3150000C0A005EB810141F8046C816A6848FFF74DFD94
S3150000C0B0216865488E62FFF748FD00202660FFF77D
S3150000C0C000FF19E05E490988884217D805EB80050C
S3150000C0D055F8044C94B12046FFF78BFA2046FFF73B
S3150000C0E050FB45F8046C5948A16AFFF72EFD21461E
S3150000C0F05548A662FFF729FD002070BDFF2070BDE0
S3150000C1002DE9F74F8A464E49914600200A88054692
S3150000C110002A88BF4B4A05D942F820500B88401C9C
S3150000C1208342F9D84A48302201884748FFF7CAFCBB
S3150000C1304848008880B240F00042474801684348BA
S3150000C140FFF7C0FC45480822018845480068FFF70C
S3150000C150B9FC444EFF273446F770758425704FF0BE
S3150000C160010884F80180A5706560A560E560256119
S3150000C170A582E5822583658384F82050DFF8E8B040
S3150000C18084F821503148FFF7C1FCA0625946204689
S3150000C190FFF7F0F829480421017045603348017023
S3150000C1A0C56005618582706A2030F9F73BF922483F
S3150000C1B030490660022070702D4805704570097878
S3150000C1C0C170FAF750F92C48016841F47F0101600B
S3150000C1D00068390601EA00202849C043B0FA80F019
S3150000C1E00968C0F10800C1F302218142A8BF481CBA
S3150000C1F023490A686FF0807303FA00F062F31700B0
S3150000C2000860FFF709FE1F49002808600CDB1E497D
S3150000C210475400F01F0108FA01F140114FF0E022E7
S3150000C22002EB8000C0F80011009803B04A46514660
S3150000C230BDE8F04F0023D0E6D4E5FF1F0C1C00201C
S3150000C2405EC500004C05002058EAFF1F08EDFF1FE1
S3150000C25074C5000060C5000078C500007EC50000FA
S3150000C2601CE0FF1F3C1C002061640000241C002011
S3150000C270280500207CC5000020ED00E00CED00E064
S3150000C2801CED00E0D0E5FF1F00E400E00F48006869
S3150000C29070470321FFF738BE0D490C4A0968C8826A
S3150000C2A012881044888270470948016807488A8ABC
S3150000C2B00088CB8A101A80B21A448A8210F4004F82
S3150000C2C018BF70470421FFF71FBE0000DCE5FF1F03
S3150000C2D0D4E5FF1F70B52C4D2868002808BF70BD37
S3150000C2E0A8882A4E401EA8800AE0E088FAF7B9F826
S3150000C2F0A088A8802068286021463068FFF725FCC2
S3150000C300A888002818BF70BD2C68002CEDD170BD20
S3150000C31070B50D4604000BD01C48006840B1FFF70D
S3150000C320F5FB002808BF70BDC58017498A8804E060
S3150000C330002070BD19469B881A44A24202D20B689F
S3150000C340002BF7D10B68121B0360828008608A8875
S3150000C3508388D21A8A8070BD0B4A1168814205D043
S3150000C3600A0008BF704711688142F9D110B501680B
S3150000C37011609188838819449180014603480068BA
S3150000C380FFF7E3FB002010BDE0E5FF1F1CE0FF1FE9
S3150000C39040EA01039B0703D009E008C9121F08C041
S3150000C3A0042AFAD203E011F8013B00F8013B521EC1
S3150000C3B0F9D27047D2B201E000F8012B491EFBD238
S3150000C3C070470022F6E710B513460A46044619469A
S3150000C3D0FFF7F0FF204610BD421C10F8011B002994
S3150000C3E0FBD1801A704730B505460020034600E0B1
S3150000C3F05B1C934205D2EC5CC85C201A01D1002C70
S3150000C400F6D130BD064C074D06E0E06840F001036A
S3150000C41094E8070098471034AC42F6D3F8F7FCFFCF
S3150000C42064E3000084E3000070B501EB020410F839
S3150000C430015B15F0070301D110F8013B2A1106D163
S3150000C44010F8012B03E010F8016B01F8016B5B1E7D
S3150000C450F9D12B0705D40023521E0FD401F8013B56
S3150000C460FAE710F8013B02F10202A1EB030303E035
S3150000C47013F8015B01F8015B521EF9D5A142D6D330
S3150000C480002070BD02000000598B00000000000073
S3150000C49070B5294B024619461878498810F01F00D6
S3150000C4A0A3F1200604D001282ED0022812D02BE0BA
S3150000C4B0012929D132B10120FCF7FEFBF08840F0BA
S3150000C4C0020005E00020FCF7F7FBF08820F00200F0
S3150000C4D0F0802EE0187900F08F0515F0800F1DBF53
S3150000C4E005F00F034FF4803000FA03F4012008BF73
S3150000C4F000FA05F47078002818BF15F00F0F03D066
S3150000C500B068204200D009B1002070BD2AB128468B
S3150000C510FCF74AFCF06820430AE03069204208D163
S3150000C5202846FCF74DFC2846FDF706FEF068A043BA
S3150000C530F060012070BD000058E5FF1F02E008C84A
S3150000C540121F08C1002AFAD170477047002001E087
S3150000C55001C1121F002AFBD17047312E30000E0098
S3150000C56030020401FF5207000100000010270000FE
S3150000C57000000000AC0200002018000004000000CB
S3150000C58000BE0AE00D782D0668400824400000D35E
S3150000C5905840641EFAD1491C521E002AF2D1704737
S3150000C5A070B504460D4616464CF220503249C881F5
S3150000C5B04DF62810C8810846008820F00100088042
S3150000C5C02E48484400F0DCF808B1012070BD002078
S3150000C5D0FCE701460020704710B529492748484422
S3150000C5E000F0B8F804462CB900212448484400F06D
S3150000C5F0A9F9044600F037F8204610BD70B5044688
S3150000C6001E4848441E4B2146C26800F05DF80546A8
S3150000C6103DB91A48484400232146C26800F046F94D
S3150000C620054600F020F8284670BDFEB505460C46C6
S3150000C63016462346324629461048484400F0F8F884
S3150000C640074667B900200122CDE90020334622467D
S3150000C650294602900948484400F084F9074600F04C
S3150000C66002F83846FEBD0748406820F4700000F521
S3150000C670700004494860704700200540040000002F
S3150000C6806B66656B00F0014070200E4A10708020CA
S3150000C690107000BF0B480078C0090028FAD009487E
S3150000C6A0017801F0200008B16720704701F0100002
S3150000C6B008B16820F9E701F0010008B16920F4E744
S3150000C6C00020F2E7000002402DE9F04D04460D4639
S3150000C6D090469A46504600F091F8064616B1304606
S3150000C6E0BDE8F08D102342462946204600F06CF83E
S3150000C6F006460EB13046F3E705EB0800471EE06834
S3150000C700B7FBF0F100FB117040B1E068B7FBF0F049
S3150000C71000F1010BE06800FB0BF0471E11E00B482F
S3150000C72078440068056009200949C871FFF7ACFF25
S3150000C7300646A06908B1A069804706B103E0E06833
S3150000C7400544BD42EBD900BF3046C9E7EC02000004
S3150000C7500000024070B504460D46284600F04EF82B
S3150000C76006460EB1304670BD0CB90420FBE74420E6
S3150000C7700249C871FFF788FFF5E700000000024094
S3150000C780014609B9042070472648C06CC0F303600F
S3150000C790254B7B4433F8100002030AB96420F2E704
S3150000C7A0002008604A6002208860C002C86000203D
S3150000C7B008614861886100BFE5E702460AB90420BE
S3150000C7C0704791610020FBE730B504460CB90420A0
S3150000C7D030BD581E084010B9581E104008B16520DB
S3150000C7E0F6E72068884205D8D4E9000528448D1864
S3150000C7F0A84201D26620EBE70020E9E701460B4894
S3150000C800814201D06B2070470020FCE703460BB93C
S3150000C810042070470F2901D8042A01D00420F8E724
S3150000C8200020F6E7008004405A0200006B66656B44
S3150000C8302DE9F0410746884614461D4614B90420E2
S3150000C840BDE8F08108232A4641463846FFF7BCFF7B
S3150000C85006460EB13046F3E71FE0124878440068FA
S3150000C860C0F8008001CC0F4979440C39096848604A
S3150000C87001CC0C49794418390968886007200A49AF
S3150000C880C871FFF701FF0646B86908B1B869804765
S3150000C89006B104E008F10808083D002DDDD100BF0F
S3150000C8A03046CDE7B0010000000002402DE9FF4D03
S3150000C8B082B082460C46102321465046049AFFF762
S3150000C8C083FF8346BBF1000F03D0584606B0BDE890
S3150000C8D0F08DDAE90101B0FBF1F7604279420840D8
S3150000C8E04542A54200D13D44049E22E0A5EB040842
S3150000C8F0B04500D9B0464FEA181001900F48784469
S3150000C9000068046001200E49C8710198000AC872C7
S3150000C9100198887205984872FFF7B6FE8346BBF108
S3150000C920000F01D05846D1E7A6EB080644443D4423
S3150000C93000BF002EDAD10020C8E700000E0100007B
S3150000C9400000024070B504460D460CB9042070BDC7
S3150000C95040200349C87108468571FFF795FEF6E742
S3150000C960000002402DE9FF4D0C4617461D46DDE945
S3150000C9700CB8DDF838A01DB9042004B0BDE8F08D70
S3150000C98004233A4621460098FFF71EFF06460EB1DD
S3150000C9903046F2E722E0144878440068046002203A
S3150000C9A01249C871084680F80BB00F49794414390A
S3150000C9B0286809688860FFF767FE06465EB1B8F129
S3150000C9C0000F01D0C8F80040BAF1000F02D00020D5
S3150000C9D0CAF8000004E03F1F2D1D241D002FDAD1E8
S3150000C9E000BF3046C9E700007400000000000240A6
S3150000C9F000000000000008000000100000002000F9
S3150000CA00000040000000800000000001000000015E
S3150000CA1004000240000000000000040008030101B9
S3150000CA2001004000400004000101400040000002F7
S3150000CA30020040000002010203040400000240005C
S3150000CA404000400000000000000000000000000060
S3150000CA500100000091740000C1740000AB9E00004C
S3150000CA6019A6000025B300006F950000339600005C
S3150000CA7000000000000000000000000000000000B0
S3150000CA8000000000000000000000000000000000A0
S3150000CA900000000000000000000000000600FF0982
S3150000CAA001A101150026FF007508954009018102C4
S3150000CAB095400901910295010901B102C0002100CA
S3150000CAC063001201100102000008280D0402000193
S3150000CAD001020301000009027A0004010080FA093C
S3150000CAE004000002080650070705820240000007FE
S3150000CAF005020240000009040300020300000609C3
S3150000CB0021000100012221000705810340000107E1
S3150000CB1005010340000109040100010202010405A8
S3150000CB20240010010524010302042402060524063C
S3150000CB3001020705830310002009040200020A000F
S3150000CB4000050705040240000007058402400000B6
S3150000CB5000000000040309040A034D0042004500DA
S3150000CB6044001E034D0042004500440020004300DF
S3150000CB704D005300490053002D0044004100500071
S3150000CB801A03300030003000310041003000300020
S3150000CB9030003000300030003000100355005300E4
S3150000CBA042005F0043004400430012035500530057
S3150000CBB042005F0043004400430031001E034D0065
S3150000CBC0420045004400200043004D005300490048
S3150000CBD053002D004400410050001003550053003F
S3150000CBE042005F004D00530043000000BDDF00001F
S3150000CBF0C5DF0000C1DF0000C9DF00000000000043
S3150000CC0030313233343536373839616263646566BC
S3150000CC1000000000CCDF000005E20000A6E10000F5
S3150000CC2042E2000069E100000EE30000C9E20000F4
S3150000CC303AE100000EE10000E6E0000097E20000A5
S3150000CC4096E000004EE00000D2DF0000CCDF0000DE
S3150000CC5056657273696F6E3A20303232360D0A426B
S3150000CC6075696C643A202020417567203234203281
S3150000CC703031352031373A30363A33300D0A47698C
S3150000CC807420436F6D6D6974205348413A203237E2
S3150000CC906132333662396665333963363734613724
S3150000CCA03033633563383936353566626432366219
S3150000CCB03865323765310D0A476974204C6F6361F8
S3150000CCC06C206D6F64733A205965730D0A0000007D
S3150000CCD0000000000000000000000000000000004E
S3150000CCE0000000000000000000000000000000003E
S3150000CCF0000000000000000000000000000000002E
S3150000CD00000000000000000000000000000000001D
S3150000CD10000000000000000000000000000000000D
S3150000CD2000000000000000000000000000000000FD
S3150000CD3000000000000000000000000000000000ED
S3150000CD4000000000000000000000000000000000DD
S3150000CD5000000000000000000000000000000000CD
S3150000CD6000000000000000000000000000000000BD
S3150000CD7000000000000000000000000000000000AD
S3150000CD80000000000000000000000000000000009D
S3150000CD90000000000000000000000000000000008D
S3150000CDA0000000000000000000000000000000007D
S3150000CDB0000000000000000000000000000000006D
S3150000CDC0000000000000000000000000000000005D
S3150000CDD0000000000000000000000000000000004D
S3150000CDE0000000000000000000000000000000003D
S3150000CDF0000000000000000000000000000000002D
S3150000CE00000000000000000000000000000000001C
S3150000CE10000000000000000000000000000000000C
S3150000CE2000000000000000000000000000000000FC
S3150000CE3000000000000000000000000000000000EC
S3150000CE4000000000000000000000000000000000DC
S3150000CE504641494C2020202054585401000000002F
S3150000CE60210032BB0000DC83BB340400000200005A
S3150000CE7000000000000000000000000000000000AC
S3150000CE80000000000000000000000000000000009C
S3150000CE90000000000000000000000000000000008C
S3150000CEA0000000000000000000000000F8FFFFFF87
S3150000CEB0FFFFFFFFFFFFFFFF000000000000000074
S3150000CEC0000000000000000000000000000000005C
S3150000CED0000000000000000000000000000000004C
S3150000CEE0000000000000000000000000000000003C
S3150000CEF0000000000000000000000000000000002C
S3150000CF00000000000000000000000000000000001B
S3150000CF10000000000000000000000000000000000B
S3150000CF2000000000000000000000000000000000FB
S3150000CF3000000000000000000000000000000000EB
S3150000CF4000000000000000000000000000000000DB
S3150000CF5000000000000000000000000000000000CB
S3150000CF6000000000000000000000000000000000BB
S3150000CF7000000000000000000000000000000000AB
S3150000CF80000000000000000000000000000000009B
S3150000CF90000000000000000000000000000000008B
S3150000CFA0000000000000000000000000000000007B
S3150000CFB0000000000000000000000000000000006B
S3150000CFC0000000000000000000000000000000005B
S3150000CFD0000000000000000000000000000000004B
S3150000CFE0000000000000000000000000000000003B
S3150000CFF0000000000000000000000000000000002B
S3150000D000000000000000000000000000000000001A
S3150000D010000000000000000000000000000000000A
S3150000D02000000000000000000000000000000000FA
S3150000D03000000000000000000000000000000000EA
S3150000D04000000000000000000000000000000000DA
S3150000D05000000000000000000000000000000000CA
S3150000D06000000000000000000000000000000000BA
S3150000D07000000000000000000000000000000000AA
S3150000D080000000000000000000000000000000009A
S3150000D090000000000000000000000000000000008A
S3150000D0A00000000000000000000000003C212D2DC3
S3150000D0B0206D62656420506C6174666F726D2057D6
S3150000D0C065627369746520616E6420417574686574
S3150000D0D06E7469636174696F6E2053686F727463EE
S3150000D0E07574202D2D3E0D0A3C68746D6C3E0D0A3C
S3150000D0F03C686561643E0D0A3C6D65746120687428
S3150000D10074702D65717569763D22726566726573F8
S3150000D110682220636F6E74656E743D22303B207505
S3150000D120726C3D687474703A2F2F6D6265642E6F51
S3150000D13072672F6465766963652F3F636F64653D2B
S3150000D1404041222F3E0D0A3C7469746C653E6D6247
S3150000D150656420576562736974652053686F7274DD
S3150000D1606375743C2F7469746C653E0D0A3C2F68B8
S3150000D1706561643E0D0A3C626F64793E3C2F626FC6
S3150000D18064793E0D0A3C2F68746D6C3E0D0A0D0ADB
S3150000D1900000000000000000000000000000000089
S3150000D1A00000000000000000000000000000000079
S3150000D1B00000000000000000000000000000000069
S3150000D1C00000000000000000000000000000000059
S3150000D1D00000000000000000000000000000000049
S3150000D1E00000000000000000000000000000000039
S3150000D1F00000000000000000000000000000000029
S3150000D2000000000000000000000000000000000018
S3150000D2100000000000000000000000000000000008
S3150000D22000000000000000000000000000000000F8
S3150000D23000000000000000000000000000000000E8
S3150000D24000000000000000000000000000000000D8
S3150000D25000000000000000000000000000000000C8
S3150000D26000000000000000000000000000000000B8
S3150000D27000000000000000000000000000000000A8
S3150000D2800000000000000000000000000000000098
S3150000D2900000000000000000000000000000000088
S3150000D2A0000000000000000000000000506C6163F8
S3150000D2B065686F6C64657220666F72206661696C62
S3150000D2C02E74787420646174610D0A0000000000F9
S3150000D2D00000000000000000000000000000000048
S3150000D2E00000000000000000000000000000000038
S3150000D2F00000000000000000000000000000000028
S3150000D3000000000000000000000000000000000017
S3150000D8A000000000000000000000000000BE0AE0CA
S3150000D8B00D782D0668400824400000D35840641EA9
S3150000D8C0FAD1491C521E002AF2D1704770B504469F
S3150000D8D00D4616464CF220503249C8814DF62810A6
S3150000D8E0C8810846008820F0010008802E48484478
S3150000D8F000F0DCF808B1012070BD0020FCE701460D
S3150000D9000020704710B529492748484400F0B8F868
S3150000D91004462CB900212448484400F0A9F90446DD
S3150000D92000F037F8204610BD70B504461E4848443E
S3150000D9301E4B2146C26800F05DF805463DB91A48FF
S3150000D940484400232146C26800F046F9054600F027
S3150000D95020F8284670BDFEB505460C4616462346F9
S3150000D960324629461048484400F0F8F8074667B999
S3150000D97000200122CDE900203346224629460290A6
S3150000D9800948484400F084F9074600F002F8384692
S3150000D990FEBD0748406820F4700000F57000044999
S3150000D9A04860704700200540040000006B66656B08
S3150000D9B000F0014070200E4A10708020107000BFE9
S3150000D9C00B480078C0090028FAD00948017801F010
S3150000D9D0200008B16720704701F0100008B16820E8
S3150000D9E0F9E701F0010008B16920F4E70020F2E749
S3150000D9F0000002402DE9F04D04460D4690469A4639
S3150000DA00504600F091F8064616B13046BDE8F08D56
S3150000DA10102342462946204600F06CF806460EB111
S3150000DA203046F3E705EB0800471EE068B7FBF0F168
S3150000DA3000FB117040B1E068B7FBF0F000F1010B9C
S3150000DA40E06800FB0BF0471E11E00B4878440068C5
S3150000DA50056009200949C871FFF7ACFF0646A069B1
S3150000DA6008B1A069804706B103E0E0680544BD42FD
S3150000DA70EBD900BF3046C9E7EC02000000000240C7
S3150000DA8070B504460D46284600F04EF806460EB11F
S3150000DA90304670BD0CB90420FBE744200249C8712A
S3150000DAA0FFF788FFF5E7000000000240014609B9CC
S3150000DAB0042070472648C06CC0F30360254B7B44A6
S3150000DAC033F8100002030AB96420F2E70020086068
S3150000DAD04A6002208860C002C86000200861486170
S3150000DAE0886100BFE5E702460AB9042070479161E4
S3150000DAF00020FBE730B504460CB9042030BD581EA3
S3150000DB00084010B9581E104008B16520F6E7206895
S3150000DB10884205D8D4E9000528448D18A84201D2C8
S3150000DB206620EBE70020E9E701460B48814201D079
S3150000DB306B2070470020FCE703460BB904207047B2
S3150000DB400F2901D8042A01D00420F8E70020F6E7BF
S3150000DB50008004405A0200006B66656B2DE9F041B7
S3150000DB600746884614461D4614B90420BDE8F081D0
S3150000DB7008232A4641463846FFF7BCFF06460EB143
S3150000DB803046F3E71FE0124878440068C0F800808A
S3150000DB9001CC0F4979440C390968486001CC0C491D
S3150000DBA0794418390968886007200A49C871FFF75F
S3150000DBB001FF0646B86908B1B869804706B104E0B6
S3150000DBC008F10808083D002DDDD100BF3046CDE73D
S3150000DBD0B0010000000002402DE9FF4D82B08246F0
S3150000DBE00C46102321465046049AFFF783FF8346CE
S3150000DBF0BBF1000F03D0584606B0BDE8F08DDAE958
S3150000DC000101B0FBF1F76042794208404542A54266
S3150000DC1000D13D44049E22E0A5EB0408B04500D99E
S3150000DC20B0464FEA181001900F4878440068046027
S3150000DC3001200E49C8710198000AC87201988872BD
S3150000DC4005984872FFF7B6FE8346BBF1000F01D078
S3150000DC505846D1E7A6EB080644443D4400BF002ED3
S3150000DC60DAD10020C8E700000E01000000000240E3
S3150000DC7070B504460D460CB9042070BD402003491A
S3150000DC80C87108468571FFF795FEF6E70000024069
S3150000DC902DE9FF4D0C4617461D46DDE90CB8DDF8AB
S3150000DCA038A01DB9042004B0BDE8F08D04233A461F
S3150000DCB021460098FFF71EFF06460EB13046F2E7F2
S3150000DCC022E0144878440068046002201249C871B2
S3150000DCD0084680F80BB00F4979441439286809685A
S3150000DCE08860FFF767FE06465EB1B8F1000F01D007
S3150000DCF0C8F80040BAF1000F02D00020CAF80000B0
S3150000DD0004E03F1F2D1D241D002FDAD100BF304631
S3150000DD10C9E7000074000000000002400000000097
S3150000DD200000080000001000000020000000400075
S3150000DD300000800000000001000000010400024015
S3150000DD4000000000210000204900002059000020AA
S3150000DD507D000020AB00002001000020940400207C
S3150000DD600010002000300020000000209804000071
S3150000DD70ACD8000000020000FFFFFFFFFFFFFFFF1F
S3150000DD80FFFFFFFFFFFFFFFFFFFFFFFFFFFFFFFF9D
S3150000DD90FFFFFFFFFFFFFFFFFFFFFFFFFFFFFFFF8D
S3150000DDA0FFFFFFFFFFFFFFFFFFFFFFFFFFFFFFFF7D
S3150000DDB0FFFFFFFFFFFFFFFFFFFFFFFFFFFFFFFF6D
S3150000DDC0FFFFFFFFFFFFFFFFFFFFFFFFFFFFFFFF5D
S3150000DDD0FFFFFFFFFFFFFFFFFFFFFFFFFFFFFFFF4D
S3150000DDE0FFFFFFFFFFFFFFFFFFFFFFFFFFFFFFFF3D
S3150000DDF0FFFFFFFFFFFFFFFFFFFFFFFFFFFFFFFF2D
S3150000DE00FFFFFFFFFFFFFFFFFFFFFFFFFFFFFFFF1C
S3150000DE10FFFFFFFFFFFFFFFFFFFFFFFFFFFFFFFF0C
S3150000DE20FFFFFFFFFFFFFFFFFFFFFFFFFFFFFFFFFC
S3150000DE30FFFFFFFFFFFFFFFFFFFFFFFFFFFFFFFFEC
S3150000DE40FFFFFFFFFFFFFFFFFFFFFFFFFFFFFFFFDC
S3150000DE50FFFFFFFFFFFFFFFFFFFFFFFFFFFFFFFFCC
S3150000DE60FFFFFFFFFFFFFFFFFFFFFFFFFFFFFFFFBC
S3150000DE70FFFFFFFFFFFFFFFFFFFFFFFFFFFFFFFFAC
S3150000DE80FFFFFFFFFFFFFFFFFFFFFFFFFFFFFFFF9C
S3150000DE90FFFFFFFFFFFFFFFFFFFFFFFFFFFFFFFF8C
S3150000DEA0FFFFFFFFFFFFFFFFFFFFFFFFFFFFFFFF7C
S3150000DEB0FFFFFFFFFFFFFFFFFFFFFFFFFFFFFFFF6C
S3150000DEC0FFFFFFFFFFFFFFFFFFFFFFFFFFFFFFFF5C
S3150000DED0FFFFFFFFFFFFFFFFFFFFFFFFFFFFFFFF4C
S3150000DEE0FFFFFFFFFFFFFFFFFFFFFFFFFFFFFFFF3C
S3150000DEF0FFFFFFFFFFFFFFFFFFFFFFFFFFFFFFFF2C
S3150000DF00FFFFFFFFFFFFFFFFFFFFFFFFFFFFFFFF1B
S3150000DF10FFFFFFFFFFFFFFFFFFFFFFFFFFFFFFFF0B
S3150000DF20FFFFFFFFFFFFFFFFFFFFFFFFFFFFFFFFFB
S3150000DF30FFFFFFFFFFFFFFFFFFFFFFFFFFFFFFFFEB
S3150000DF40FFFFFFFFFFFFFFFFFFFFFFFFFFFFFFFFDB
S3150000DF50FFFFFFFFFFFFFFFFFFFFFFFFFFFFFFFFCB
S3150000DF60FFFFFFFFFFFFFFFFFFFFFFFFFFFFFFFFBB
S3150000DF70FFFFFFFFFFFFFFFF3032343078787878FD
S3150000DF80787878780010000000010000000000009A
S3150000DF90000010000000FF1F00000320000010001A
S3150000DFA04D424544202020206D6963726F636F6E79
S3150000DFB074726F6C6C657220312E30200042494EAF
S3150000DFC0004845580062696E006865780030323254
S3150000DFD03600546865206865782066696C6520633C
S3150000DFE0616E6E6F74206265206465636F6465643C
S3150000DFF02E20506172736572206C6F6769632066AC
S3150000E00061696C757265206F6363757265642E0D48
S3150000E0100A546865206865782066696C65206361C6
S3150000E0206E6E6F742062652070726F6772616D6DBF
S3150000E03065642E204C6F676963206661696C757232
S3150000E04065206F636375727265642E0D0A005468ED
S3150000E05065206865782066696C652063616E6E6F01
S3150000E06074206265206465636F6465642E2043686E
S3150000E07065636B73756D2063616C63756C61746940
S3150000E0806F6E206661696C757265206F6363757269
S3150000E09065642E0D0A00546865206170706C6963B2
S3150000E0A06174696F6E2066696C6520666F726D615A
S3150000E0B07420697320756E6B6E6F776E20616E6467
S3150000E0C02063616E6E6F7420626520706172736585
S3150000E0D06420616E642F6F722070726F6365737354
S3150000E0E065642E0D0A00466C61736820616C676F6B
S3150000E0F0726974686D20777269746520636F6D6DDF
S3150000E100616E64204641494C5552450D0A00466CE5
S3150000E11061736820616C676F726974686D206572DF
S3150000E12061736520616C6C20636F6D6D616E642038
S3150000E1304641494C5552450D0A00466C61736820AC
S3150000E140616C676F726974686D20657261736520B2
S3150000E150736563746F7220636F6D6D616E642046C4
S3150000E16041494C5552450D0A0054686520696E7444
S3150000E170657266616365206669726D776172652096
S3150000E1804641494C454420746F20696E6974696143
S3150000E1906C697A652074686520746172676574209D
S3150000E1A04D43550D0A0054686520696E74657266A4
S3150000E1B0616365206669726D7761726520464149C3
S3150000E1C04C454420746F20646F776E6C6F616420D9
S3150000E1D074686520666C6173682070726F6772611F
S3150000E1E06D6D696E6720616C676F726974686D73B7
S3150000E1F020746F2074686520746172676574204DA1
S3150000E20043550D0A0054686520696E74657266612F
S3150000E2106365206669726D77617265204641494C77
S3150000E220454420746F2072657365742F68616C7441
S3150000E2302074686520746172676574204D43550DBE
S3150000E2400A0054686520696E7465726661636520AC
S3150000E2506669726D77617265204641494C45442076
S3150000E260746F20646F776E6C6F61642074686520CC
S3150000E270666C617368206461746120636F6E746597
S3150000E2806E747320746F2062652070726F6772619E
S3150000E2906D6D65640D0A00466C6173682070726F5F
S3150000E2A06772616D206164647265737320616E6468
S3150000E2B020646174612062756666657220756E61A0
S3150000E2C06C69676E65640D0A0054686520696E7432
S3150000E2D0657266616365206669726D776172652035
S3150000E2E04641494C454420746F20756E6C6F636BD4
S3150000E2F0207468652074617267657420666F722089
S3150000E30070726F6772616D6D696E670D0A00546891
S3150000E3106520696E74657266616365206669726DF3
S3150000E320776172652041424F525445442070726FA6
S3150000E3306772616D6D696E672E20496D6167652034
S3150000E340697320747279696E6720746F20736574BF
S3150000E35020736563757269747920626974730D0A36
S3150000E3600000000084E3000000E0FF1FE805000055
S3150000E37028C4000034E40000E8E5FF1F88380000E8
S3150000E3804CC5000011746CDC02041A010101033E45
S3150000E390A0DF0A11CD40100CEB3C904D5344305396
S3150000E3A0342E311402080113022015501FF80129DA
S3150000E3B002A1180B29741902274D42454420011861
S3150000E3C009444E4446415431320B01FF01C148080D
S3150000E3D055AA4D4245442001A22865418EBB3269AB
S3150000E3E0204548544D0112212332BB26DC83BB3421
S3150000E3F0021903C80C44455441494C5320545854FF
S3150000E400203B30032001FF01A1157CE0FF1F220203
S3150000E41033ACCE99085B7CE2185AD4185AD0084A15
S3150000E420D608CB50CC104BACD208011C1A550101B2
S3150000E430FC000000000000000000000000000000DA
S3150000E44000000000000000000000000000000000C6
S3150000E45000000000000000000000000000000000B6
S3150000E46000000000000000000000000000000000A6
S3150000E4700000000000000000000000000000000096
S3150000E4800000000000000000000000000000000086
S3150000E4900000000000000000000000000000000076
S3150000E4A00000000000000000000000000000000066
S3150000E4B00000000000000000000000000000000056
S3150000E4C00000000000000000000000000000000046
S3150000E4D00000000000000000000000000000000036
S3150000E4E00000000000000000000000000000000026
S3150000E4F00000000000000000000000000000000016
S3150000E5000000000000000000000000000000000005
S3150000E51000000000000000000000000000000000F5
S3150000E52000000000000000000000000000000000E5
S3150000E53000000000000000000000000000000000D5
S3150000E54000000000000000000000000000000000C5
S3150000E55000000000000000000000000000000000B5
S3150000E56000000000000000000000000000000000A5
S3150000E5700000000000000000000000000000000095
S3150000E5800000000000000000000000000000000085
S3150000E5900000000000000000000000000000000075
S3150000E5A00000000000000000000000000000000065
S3150000E5B00000000000000000000000000000000055
S3150000E5C00000000000000000000000000000000045
S3150000E5D00000000000000000000000000000000035
S3150000E5E00000000000000000000000000000000025
S3150000E5F00000000000000000000000000000000015
S3150000E60043550D0A0054686520696E74657266612B
S3150000E6106365206669726D77617265204641494C73
S3150000E620454420746F2072657365742F68616C743D
S3150000E6302074686520746172676574204D43550DBA
S3150000E6400A0054686520696E7465726661636520A8
S3150000E6506669726D77617265204641494C45442072
S3150000E660746F20646F776E6C6F61642074686520C8
S3150000E670666C617368206461746120636F6E746593
S3150000E6806E747320746F2062652070726F6772619A
S3150000E6906D6D65640D0A00466C6173682070726F5B
S3150000E6A06772616D206164647265737320616E6464
S3150000E6B020646174612062756666657220756E619C
S3150000E6C06C69676E65640D0A0054686520696E742E
S3150000E6D0657266616365206669726D776172652031
S3150000E6E04641494C454420746F20756E6C6F636BD0
S3150000E6F0207468652074617267657420666F722085
S3150000E70070726F6772616D6D696E670D0A0054688D
S3150000E7106520696E74657266616365206669726DEF
S3150000E720776172652041424F525445442070726FA2
S3150000E7306772616D6D696E672E20496D6167652030
S3150000E740697320747279696E6720746F20736574BB
S3150000E75020736563757269747920626974730D0A32
S3150000E7600000000084E3000000E0FF1FE805000051
S3150000E77028C4000034E40000E8E5FF1F88380000E4
S3150000E7804CC5000011746CDC02041A010101033E41
S3150000E790A0DF0A11CD40100CEB3C904D5344305392
S3150000E7A0342E311402080113022015501FF80129D6
S3150000E7B002A1180B29741902274D4245442001185D
S3150000E7C009444E4446415431320B01FF01C1480809
S3150000E7D055AA4D4245442001A22865418EBB3269A7
S3150000E7E0204548544D0112212332BB26DC83BB341D
S3150000E7F0021903C80C44455441494C5320545854FB
S3150000E800FFFFFFFFFFFFFFFFFFFFFFFFFFFFFFFF12
S3150000E810FFFFFFFFFFFFFFFFFFFFFFFFFFFFFFFF02
S3150000E820FFFFFFFFFFFFFFFFFFFFFFFFFFFFFFFFF2
S3150000E830FFFFFFFFFFFFFFFFFFFFFFFFFFFFFFFFE2
